:020000040800F2
:1000000000C00020FD4301089D440108E52D0108C2
:100010009D4401089D4401089D4401080000000022
:100020000000000000000000000000009D440108E6
:100030009D440108000000009D44010881810008E2
:100040009D4401089D4401089D4401089D44010808
:100050009D4401089D440108D1B40008CDB40008B6
:100060009D4401089D4401089D4401089D440108E8
:100070009D4401089D440108EDB400089D44010819
:1000800061CC00089D4401089D4401089D4401087D
:100090009D4401089D4401089D440108C9B400081D
:1000A0009D440108B9B200089D440108C9B2000886
:1000B000A9B2000899B2000889B20008C55A000820
:1000C000C95A0008BD5A0008C15A00089D440108D9
:1000D0009D440108E1B40008D5B400089D4401081E
:1000E000918100089D4401089D4401089D44010838
:1000F0009D4401089D4401089D4401089D44010858
:100100009D4401089D4401089D4401089D44010847
:100110009D4401089D4401089D4401089D44010837
:100120009D4401089D4401089D4401089D44010827
:1001300000000000000000000000000000000000BF
:1001400000000000000000000000000000000000AF
:10015000000000000000000000000000000000009F
:10016000000000000000000000000000000000008F
:10017000000000000000000000000000000000007F
:10018000000000000000000000000000000000006F
:10019000000000000000000000000000000000005F
:1001A000000000000000000000000000000000004F
:1001B000000000000000000000000000000000003F
:1001C000000000000000000000000000000000002F
:1001D000000000000000000000000000000000001F
:0401E0005FF8E0F1F3
:1001E8002DE9F04F684B694FA1B03B6000237B605D
:1001F80011F012FC18B911F031FC0AF003F90AF0F9
:10020800A7F9634A634C1378634E43F001031370F4
:100218000023089309930A934FF4E0130B93236880
:10022800B07B43F480332360A36943F01003A361D8
:10023800236803F400330993089B01330893099B4F
:100248001BB9089BB3F5A06FF2D12368514913F489
:10025800003301D0022315E00A6842F001020A6067
:100268000893236803F002030993089B013308935A
:10027800099B1BB9089BB3F5A06FF2D123689B07B4
:1002880039D501230A93454B45491A6842F01002B3
:100298001A601A6822F003021A601A6842F0020211
:1002A8001A606368636063686360636843F48063CB
:1002B80063603C4B1A68043B22F070425A603A4A29
:1002C8001160616821F47C116160596841F0004156
:1002D8005960D96821F40041D9609B681D0449BF61
:1002E800324B4FF4E01313604FF480130B930A9BC7
:1002F800012B01D117E0FEE7022B18D168B10B9B47
:10030800B3F5801F02D14FF4A01305E00B9BB3F5A2
:10031800E01F02D14FF400130B930B9963680B4352
:1003280043F4803302E0636843F460136360236836
:1003380043F0807323602168164B8901FBD5596807
:1003480021F003015960596841F00201596063685E
:10035800104903F00C03082BF9D14B68DFF85490CF
:1003680003F00C03042B03D0082B03D00C4B29E01B
:10037800136827E04B684868C3F38343C50303F158
:10038800020319D40A4A1CE0F39B0008C8000020A5
:10039800C030002000100240D4110020002002408C
:1003A80000127A000410014034000020001BB7003E
:1003B80000093D005000002049681268880348BFC2
:1003C80052085343C9F800306368DFF888A2C3F3C2
:1003D800031353441A7ED9F80030DFF87CC2D340A7
:1003E800C9F80030854A864B20ADD360A3690492D2
:1003F80043F00103A361636ADFF86082BB60636A4C
:10040800604643F080736362A3694FF0000B43F0CA
:100418001C03A3614FF6FF7325F82C3D2946CDF840
:100428000CC08DF856B00CF00DFD404629460CF076
:1004380009FD744829460CF005FD734928464B68A8
:1004480043F000734B600EF01BFF159B6F49049A35
:10045800B3FBF1F36E490B606E4B4FF47A71C3F83E
:1004680000B0D9F80030DFF8F891B3FBF1F36A492E
:10047800013B4B60F02382F823300723C1F808B012
:100488000B60B368DFF898B1C9F800300AF12803A7
:100498000FCB85E80F00A369159843F00803A36103
:1004A800A36916A943F00803A3610823C8F810300C
:1004B8001023C8F8103004930CF0C4FC179818A93E
:1004C8000CF0C0FCD9F80020049B12F0080F12D0E1
:1004D8009BF89221012A0ED850499BF893218968EC
:1004E80011F0805B00F0CB8405E04D4B002283F8CF
:1004F80093210AF0F1F9642007F0F1FDA0224948A0
:10050800002116F0F4FAE369002243F00703E361DF
:10051800A36943F4006343F00C03A3613F4B4FF01E
:10052800000B03F10C0102F801B001320E2AF5D1DB
:10053800FF229A76DA761A775A773B4B3B4A594626
:100548001A603B483022D9F8004016F0D0FA5946D4
:10055800C4F380180423374ADFF8D4E0885C0C22FF
:100568004A4302F80E00B8F1000F08D11E380128DE
:100578009FBFFF2003F1FF3302F80E00DBB2013109
:100588000429E8D12C4A96F805B013702B4B2C4956
:1005980083F800B02B4B214A3B62C0330B602A4BD7
:1005A800A10603EBCB035B7848BF0123536200230A
:1005B80040F2DC51254A22F813100133082BF7D1F9
:1005C8000EA800211C2216F092FA14F4007304F409
:1005D800006947D0A2040BD4B9F1000F0AD01C4A15
:1005E80096F88601A2F10C01012808BF0A4602E02C
:1005F800184A00E0164A0492149534E000ED00E031
:100608000005FA05001001400000014040420F00BB
:10061800C81A0020CC1A002010E000E0C800002012
:10062800D4110020B02A0020BC280020C8130020C4
:10063800C0280020FCC00108A9110020040A0020DD
:10064800CC2B0020E8110020E0B60108141100208E
:10065800CC900108C090010800080140000C01403E
:10066800FC2C00200493BBF10E0F04D00BF0EF0B11
:10067800BBF1080F02D101228DF84A200120059311
:1006880007F000FB059B18B14088003018BF012017
:10069800C4F340028DF83E20C4F3403200F001005C
:1006A8008DF83820C4F3C0328DF83D008DF84080B5
:1006B8008DF83B20B9F1000F07D096F8869109F123
:1006C800FF3EDEF1000949EB0E09003318BF012394
:1006D8008DF842307B6AB6F84801003318BF012311
:1006E8008DF84330C4F300538DF84430B6F84A31DE
:1006F800E504ADF84830B6F85631ADF84E0048BFBD
:10070800BA48ADF84630C4F3804348BFB0F850014A
:100718008DF83F30B6F8543148BFADF84E00B3F508
:10072800FA7FADF84C3084BF0023ADF84E3096F810
:10073800D631AF4887F82830002387F8293043702E
:100748009DF84A30C4F30042002B8DF8412004F094
:100758000101C4F3C0028DF83C908DF839108DF872
:100768003A200CBF0023022301B902B101330AEB7E
:10077800830ADAF838304FF00008A3F102091A3377
:1007880005934FF6FF7339F802AF9A4500F0788168
:100798009DF83D205FFA8AF31AB19A1E012A40F2A9
:1007A8006B819DF8402032B192491A018958924ACA
:1007B800914200F061819DF8412032B18D491A01C2
:1007C80089588D4A914200F057819DF83E2052B1D8
:1007D800884A039802EB03125168814203D11289B7
:1007E800102A00F049819DF83B2052B1814A0398B4
:1007F80002EB03125168814203D11289022A00F0E8
:100808003B819DF83C2052B17A4A7C4802EB0312A6
:100818005168814203D11289022A00F02D81149A6D
:100828007AB1744C116804EB03146068884208D1EB
:1008380021899088884200F01F81D2888A4200F07E
:100848001B814FEA1A2ABAF1020F02D19DF838200B
:1008580004E0BAF1010F04D19DF83920002A00F014
:100868000B81DFF890B19DF844101F010BEB0704D2
:100878005A4631B19DF84A1019B9043B032B40F28E
:10088800E380BAF1010F5FFA8AF341D15C4D3A4433
:10089800FF23517B85F8703085F87130506802F17C
:1008A800080312890026ADF854208DF8561002224C
:1008B80015A985F87460C5F8804006938DF857200F
:1008C80085F82C602E636E63AE63EE6685F8726001
:1008D80085F873600CF0B6FA069B5BF80700997808
:1008E80032460CF063F92046314652460AF044FD80
:1008F800444BC5F88C60C5F88430434B2046C5F896
:10090800883005F1840105F188020AF07DFDB3E025
:10091800022B46D15FFA88F21C2101FB02FC384AFF
:10092800002502EB0C06334A4FF0010A3A44517B8A
:10093800506802F1080B128986F875808DF85610F8
:1009480086F8765015A986F87E5086F874A0C6F801
:100958008040CDF818C0ADF854208DF857300CF011
:1009680071FA244B9BF80210D8592A460CF01EF94C
:100978002046294652460AF0FFFC244A204BDDF85F
:1009880018C0C6F8842003EB0C01214A8431C6F84C
:100998008820C6F88C5020460A1D0AF035FDD04440
:1009A8006AE0032B4ED19DF83F30154D194E3BB1EF
:1009B80095F82A70204608214FF6FF72002335E08B
:1009C800BDF84C2095F82A70B2F5FA7FBDF84E3084
:1009D80026D911492046B1FBF2F2082192B20CF057
:1009E80025FB0E4B46F8270025E000BFD411002058
:1009F800F100002070B3010800040040000C014021
:100A0800C800002021CA000801CB0008F1CB00086B
:100A1800F9C90008802A002000127A0021CB0008BA
:100A280067492046B1FBF2F2012192B20CF0FEFABE
:100A3800644B46F82700C36095F82A30013385F8DF
:100A48002A3019E0042B17D1BDF846205C4B5E4DC7
:100A580093FBF2F22046BDF84830012192B295F896
:100A680029600CF0E3FA95F8293005EB8606013386
:100A7800C6F8540185F82930059B99457FF481AE65
:100A8800514D524B95F82920002485F87421504A7D
:100A98001C7017789846A7F11702022A19D82B6AF2
:100AA8000021185903EB040912F054FC10B16B6AC9
:100AB80063BB26E0474E99E80F00264486E80F00FE
:100AC80098F8003010340133C02C88F80030E6D193
:100AD800EDE7414B13F8376003EBC703D3F804E0A5
:100AE80088F80060BEF1000FE1D0B442DFDA394A7D
:100AF800230103EB020C73440FCB01348CE80F0085
:100B0800F3E7364E3368DC0424D41DE0344B354A11
:100B180013F8370003EBC7035C681070002CF0D0A3
:100B280000238342EDDAC3EBC3016218D2F800C098
:100B3800DFF8BCE0013341F80EC001EB0E069188E6
:100B4800B1809279B271ECE707F0EF03082B264BDE
:100B580025D126E098F80030012BF5D9234C04EB79
:100B6800031303F1100810344445EDD054F8100C69
:100B78004FF07C5112F05AFA4FF07C5144F8100CA7
:100B880054F8140C12F052FA4FF07C5144F8140C3B
:100B980054F80C0C12F04AFA44F80C0CE3E70E2F48
:100BA80008D11A78182F42F010021A7022D10FF0CB
:100BB80055FC1FE01A78192F22F010021A70F5E779
:100BC80040420F0011CB0008C80000207F2A0020F7
:100BD800040A002040090020E0B60108FC2C00208F
:100BE800789B0108582B0020C819002048090020CC
:100BF800592B00200FF016FC3368DFF81CB358039C
:100C08005EBFBA4B01221A70B94A0DF15409137824
:100C1800B84F43F004031370B74B4FF0100A93E832
:100C28000300DBF8183089E8030043F00803CBF829
:100C3800183016A915980CF005F901200AF00AFEDB
:100C48003468524604F400430393384604F40063BE
:100C58000021059315F04BFF4FF6FF72ADF83420D5
:100C680002224FF0000814408DF836208DF83780A6
:100C78000DD020A921F84CADA0480EF075FC042336
:100C88003B700124072387F80180BC70FB70039B2D
:100C980073B1022320A921F84C3D98480EF064FC5A
:100CA8000123E2183B71BB7107237C71FB71D4B23D
:100CB800059B7BB1022320A921F84C3D90480EF0FA
:100CC80053FC092301223B73BA73631C07227C730C
:100CD800FA73DCB2DBF804308A4843F44043CBF8BB
:100CE8000430DBF814304FF0000843F00103CBF870
:100CF8001430DBF81830DFF80CA243F40073CBF89B
:100D080018300EF045FA804B012C15937F4B49465D
:100D1800169394BF434680231A934FF480731B9312
:100D28004FF480631C9320231D9350464FF40053C7
:100D380018941E93CDF85C80CDF86480CDF87C8043
:100D48000EF008FADAF80030714A43F00103CAF8E5
:100D580000305368012C23F4702394BF0021012133
:100D680023F4807343EA012353609168694B013C83
:100D78000B4043F4602343F002039360D36AE4B268
:100D880023F4700343EA0454D462012307EB0802F6
:100D9800917800295CD017F80800591C0928C9B2B5
:100DA800D278DFF86CE111D9A0F10A04DEF80CA0C2
:100DB80004EB44044FF0070C0CFA04FC2AEA0C0C70
:100DC800A2404CEA0202CEF80C200EE0DEF81040F9
:100DD80000EB400C4FF0070A0AFA0CFA24EA0A045E
:100DE80002FA0CF22243CEF81020062B484C0ED8FB
:100DF800013B626B03EB83034FF01F0E0EFA03FEF9
:100E080022EA0E0200FA03F3134363631FE00C2B7C
:100E18000ED8073B226B03EB83034FF01F0E0EFA2D
:100E280003FE22EA0E0200FA03F3134323630EE0E3
:100E3800A3F10D02D4F82CC002EB82021F239340C9
:100E48002CEA030E00FA02F34EEA0303E3620B46B0
:100E580008F10408B8F1100F98D12D4B9A6842F4A4
:100E680080729A609A6842F001029A609A6842F029
:100E780008029A609968264A09074FD5FAE7013AA5
:100E8800092A3FF638ABDAF85400C8F81430294676
:100E98002860039804930BF0D5FF039B3C201A4667
:100EA8000823136107F01BF9049BC8F81030D846D3
:100EB80096F893319845BFF618AB114B4FF0080BD5
:100EC800C3F810B00493039B7820C3F814B007F05C
:100ED800FBF8049B7820C3F814B0039B08F10108C1
:100EE800C3F810B007F0F0F8E2E700BF700E00207A
:100EF800C03000201C29002008910108000801408A
:100F0800000C0140080002404C2401402C2900201C
:100F180000240140FDF7F1FF00100240936843F000
:100F280004039360AB4B9A6812F00408FAD1AA4FF5
:100F38009A68B7F85C0142F4A0029A60002841F070
:100F48006882B7F95E31002B41F06382B7F96031EE
:100F5800002B41F05E8233689B031FD5C82007F041
:100F6800BEF8AE200AF071FC08B10CF0B9F99B4C40
:100F780085F87501C82007F0B2F8994B00210C22BA
:100F88002046C5F8783115F0B2FD0223E3700CF065
:100F980040FC07F07DF8934B0344A36097F86B314E
:100FA800B7F864410593904B97F863B11B6897F8BD
:100FB8006C61B3F85630B7F80CA00693FB7B8B4FE7
:100FC80000210C228A48039315F091FD0021142278
:100FD800384615F08CFD874B00221A700793C5F828
:100FE8007C2104F01DFE079BDFF840921A4648B3A7
:100FF800814BB4F5807F3B60804B7B60804BFB600E
:10100800804B3B61804B01D1002116E0BB2C01D9FC
:10101800012112E0612C01D902210EE0292C01D90D
:1010280003210AE0132C01D9042106E0092C01D977
:10103800052102E0002CE7D0062119700123137066
:10104800022322E00790192007F049F815AB682021
:101058000F21012204F0F4F99DF85430DDF81CC08A
:10106800D32B40F01983694B4E2C3B60684B7B6057
:10107800684B3B6100F00A835D2C00F00B83362C33
:1010880000F0028389F880C10123634A634F3B70F3
:10109800136843F0010313600022614BBBF1090F91
:1010A80000F2F680DFE81BF01000F40010000E00DC
:1010B80079000C000E000A000A00EA001A70D3E05A
:1010C8001A70BDE01A7019E01A704FF0000920ABD1
:1010D80003F82C2D53204946012204F0B1F968B1D8
:1010E8009DF85430E52B09D1414B4E4A85F8839140
:1010F8001A604D4A5A60022300F020BC4B4B002274
:10110800C3F87C2104F08CFD002847D006210A464C
:1011180015AB682004F094F99DF8591001F001020C
:101128009DF8571001F001014B0043EA82019DF838
:10113800552002F001030B430BD05BB2012B01D108
:10114800002202E0022B0FD10122384B83F88421C0
:1011580011E00DAB68200C21012204F071F99DF813
:10116800343013F00F0303D1032006F0C2FF02E06E
:10117800042BE9D1E4E71E4B2D4A1A602D4A5A6028
:101188002A4A92F88421002A0CBF6F226E221A7212
:10119800234B01221A700323D0E31A70002220ABDC
:1011A80003F82C2D1C200D21012204F049F90028F8
:1011B80046D09DF854302A2B01D01A2B40D10C4A26
:1011C8001D4911601D495160184A82F88531042370
:1011D800B4E300BF00240140D4110020D41A002039
:1011E8005E130020404B4C0024110020942700205F
:1011F800C82C0020C40700203D5900081B560008D1
:10120800F555000890C1793D00000020095A0008F2
:10121800F9560008325C8F3DC41900204C000020AC
:10122800E4300020655A00087F570008C8000020F5
:10123800E55200085D560008A95900089F560008A5
:10124800002120AB03F82C1D1820012204F0F8F827
:1012580050B19DF85430FB2B06D1C04BC04A1A60E0
:10126800C04A5A60052369E304F02CFC38B1BB4B33
:10127800BD4A1A60BD4A5A6008235FE31A70B74B2B
:10128800BB4A1A60BB4A5A6000221A72092355E306
:10129800BBF1010F3FF618AF1A70042E00F23B8124
:1012A800DFE816F0050042016700050006010A2084
:1012B80006F015FF7720A02101220DAB04F0C0F83D
:1012C800002856D01E210122772004F0BBFA4FF4E3
:1012D8002F6006F0F9FE0025A5F160010026C9B2CD
:1012E800022215AB77208DF854608DF8556004F014
:1012F800A7F89DF854209DF8553043EA02239E4AEA
:1013080002F5C3716B520235102DE5D1B2F8940184
:10131800334600F00F0500F47F40A2F894013246EE
:101328000127954E22F001013144B1F886110029B8
:1013380018BF002712F0010F03D0C9B24B40082193
:1013480002E083EA1123FAE713F4004F18BF83F48D
:10135800C05301394FEA4303F6D10132102AE0D1D4
:101368002843A6F8940127B9C3F303339D4200F03C
:10137800EC82814D95F89631002B41F06A8014205B
:1013880006F0ADFE7720D02101220DAB04F058F80D
:10139800002800F08D809DF834300322552B85F805
:1013A800AF31A5F8B82140F08380D12101220DABDF
:1013B800772004F045F89DF83430772003F00F02C9
:1013C8001B0985F8B02185F8B131162215ABAA2181
:1013D80004F036F89DF854209DF8553043EA02236E
:1013E800A5F898319DF856209DF8573043EA022316
:1013F800A5F89A319DF858209DF8593043EA022300
:10140800A5F89C319DF85A209DF85B3043EA0223E9
:10141800A5F89E319DF85C209DF85D3043EA0223D3
:10142800A5F8A0319DF85E209DF85F3043EA0223BD
:10143800A5F8A2319DF860209DF8613043EA0223A7
:10144800A5F8A4319DF862209DF8633043EA022391
:10145800A5F8A6319DF864209DF8653043EA02237B
:10146800A5F8A8319DF866209DF8673043EA022365
:10147800A5F8AA319DF868209DF8693043EA02234F
:1014880041F27072A5F8AC313C4B1A8046F67812DE
:101498005A803B4A5A603B4A9A603B4ADA603B4A68
:1014A8001A613B4A5A61012385F8963100F0D1BF91
:1014B800314D95F8BC61002E40F05882142006F09A
:1014C8000EFE05F2BD137620D021012203F0B8FFED
:1014D80095F8BD31582B27D105F5E07388211822DE
:1014E800762003F0ADFF31227620F42104F0AAF92A
:1014F8000123284A85F8BC31204B9A60264A1E8071
:101508005A6045F6D8125A80244ADA60244A1A6189
:10151800244A5A612AE2012E06D0234B234A9E70A0
:10152800136843F004031360204D2B689E0702D50F
:101538000A4B1B689847039BE4B20F4E1C4A002BCA
:1015480056D02B68B4BB40F2596113F0020F40F239
:10155800712318BF0B467D2135E000BFC82C002041
:10156800415A000839570008655200089B53000883
:101578000DEE000829EE0008C800002058060020DB
:1015880035590008CD5500081D5900088D5500082B
:10159800895100088551000887510008155900082D
:1015A80041550008214F00084C000020C4190020B4
:1015B800602D0020980759BF4FF47A7319464FF4ED
:1015C800FA634FF47A719A4505DBBAF57A6FA8BFCA
:1015D8004FF47A6A00E09A464B1E5344B3FBF1F38A
:1015E800013BDBB203FB011186F88231116005E093
:1015F8009DF80C30C2F800A086F88231BA4F3B68DB
:101608009847DDF81490B94C0023B9F1020F237004
:1016180006D0B9F1030F1AD0B9F1000F40F0A88134
:10162800002220AB03F82C2DC6F8DC211E200A214D
:10163800012203F005FF50B19DF85430482B06D124
:10164800AB4BAC4A1A60AC4A5A60022395E14FF0A2
:10165800000A20AB03F82CAD0C205146012203F000
:10166800EFFE002800F0F8869DF85430482B08D18A
:101678009F4BA24A1A60A24A5A6007232370032389
:101688007BE1504600F0E8BE402300E0802389F863
:101698008031F9E4C023FAE795F88171002F56D01C
:1016A800984B00221A80002F40F09380964A8021A0
:1016B80013886B2023F040031B041B0C1380138832
:1016C80023F038031B041B0C43F0300313801388EA
:1016D8009BB243F04003138004F092FA962006F080
:1016E800FEFC0321682004F08BFA962006F0F7FC34
:1016F80003216B2004F084FA012006F0E5FC102198
:101708006A2004F07DFA012006F0DEFC39466C20E0
:1017180004F076FA012006F0D7FC3946192004F0C7
:101728006FFA012006F0D0FC10211C2004F068FAA2
:10173800012006F0C9FC1B20182104F061FA0120E1
:1017480006F0C2FC714B012283F8812141E06E4A08
:101758006B201388802123F040031B041B0C13808B
:1017680013884FF0060923F038031B041B0C43F0C1
:101778003003138013889BB243F04003138004F0B6
:101788003FFA962006F0ABFC752015A9012204F05B
:10179800DDF99DF85430682B05D009F1FF3919F0AF
:1017A800FF09EED10FE00C2015A9012204F0CEF9B3
:1017B8009DF85430142B06D3182B7FF671AF543B89
:1017C800062B7FF66DAF04F07DF9474B002860D1FA
:1017D80080E0B4F5807F0ED0BB2C0ED8612C0ED8DB
:1017E800292C0ED8132C0ED8092C0ED8002C14BF77
:1017F800062700270AE0002708E0012706E002275D
:1018080004E0032702E0042700E005273E4A1920E8
:10181800138823F040031B041B0C1380138823F048
:1018280038031B041B0C43F03003138013889BB24E
:1018380043F04003138095F8821104F0E1F9012088
:1018480006F042FC39461A2004F0DAF9012006F0C5
:101858003BFC15A804F0A0F99DF95630294A01333C
:1018680003D19DF95430013302D013889BB213B1D0
:1018780000231380A7E71C4B254A64201A60254AD9
:101888005A60254ADA60254A1A6106F028FCFFF7F3
:10189800FBBB234ABB2C1A60224A5A60224ADA60F0
:1018A8001E4A1A61214B01D901220EE0612C01D98F
:1018B80002220AE0292C01D9032206E0132C01D9BF
:1018C800042202E0092C03D905225A70FFF7DCBB79
:1018D8000622FAE7164A1A60164A5A60164A9A60A9
:1018E8000823FFF7D2BB00BF94270020E530002073
:1018F80034060020A9B6000829B5000839B6000842
:10190800A5B50008EC2C002000380040C8000020D5
:1019180075520008A15B00087D5B000890C1793D05
:10192800F95300085D5300083953000800000020EF
:1019380013EE000837EE00080FEE00082C4A7B7003
:10194800136843F002031360A7E442F21072294BB4
:1019580003261A805A80284A5A60284A9A60284AD8
:10196800DA60284A1A61284A5A61D6E50426D4E57D
:10197800B9F1010F07D9994645E6244AD3702B6877
:1019880043F008032B60224A92F8583191460BB174
:10199800204A137099F859310BB11F4A137099F8FE
:1019A8005A3103B123702B68DFF878A013F0080FC1
:1019B8003AD0BDF918204FF0640B92FBFBF4204697
:1019C800059211F0DFFA059A03900BFB142000B280
:1019D80011F0D8FA114911F029FB039B014618466A
:1019E80011F01CFA0E4911F021FBCAF800001EE0A4
:1019F800C4190020580600200D5900083155000868
:101A08000559000821550008654D00084C000020C4
:101A1800D4110020C4070020E43000208988883CC5
:101A280000002041D82B00200023CAF80030A84C21
:101A3800102223784FF00A0B43F002032370A54BC2
:101A48005A6108221A610394A24C1920E3680BF129
:101A5800FF3B83F01003E360E36883F00803E3606F
:101A680006F03DFB192006F03AFB1BF0FF0BEBD10B
:101A780008234FF0100B2361C4F810B02B68190726
:101A880009D5954BC4F814B01B689847934B0122AD
:101A9800C4F810B01A70924B924C1B68187B11F066
:101AA80071FA914911F0C2FA08F088FB8346208840
:101AB80011F068FA594611F0B9FA15F025FA8B4B6E
:101AC8001880208811F05EFA0146894811F062FBFF
:101AD800884911F05FFB884B83491860386911F019
:101AE800A5FA864911F0A2FA854F864BFF211860A6
:101AF8001B22384614F0FBFF002139702968824BFD
:101B0800012211F0020F1A701FBF7A7003221A7097
:101B1800022218BFBA704A0748BF1A78384641BF30
:101B2800551C1D700325BD5411F00A0F0CD01A78EE
:101B38000421B954511CC9B205257D54D11C023267
:101B48001970D2B20621B954704A11688F0641BF84
:101B58001A78551C1D70072548BF85540D0608D5F1
:101B68001A7809258554951C01321D70D2B20A25B0
:101B7800855499F80550082D01D00E2D04D11A78F6
:101B8800571C1F700B2787541A78CC0302F10107E2
:101B98004FF00C0E48BF5C4C00F802E0FFB248BFA3
:101BA80002321F7041BF2270554A4FF00E0E02F8E4
:101BB80007E04F0748BF1A784FF0120E41BF571C75
:101BC8001F70102787541A784C0502F10107FFB2DD
:101BD8001F7000F802E00AD599F818423CB14A4C47
:101BE80002322270464A4FF0130E02F807E01A78C4
:101BF8008C0502F101074FF0140E48BF424C00F863
:101C080002E0FFB248BF02321F7041BF22703C4A57
:101C18004FF0150E02F807E0182D0DD11A78162787
:101C28008754571CFFB24FF0170E00F807E0D71C77
:101C38000232D2B21F7085540D0341BF1A78551C69
:101C48001D70192548BF8554CC0541BF1A78511C11
:101C580019701A2348BF8354002198222C4814F085
:101C680046FF0DF074F92B4A2B4BB9F852111A6044
:101C78002A4BB9F898011980294900230B808B70E9
:101C880028490A6081B2284A22F813100133122B1E
:101C9800F9D11E4F3B68D9045CBFB9F89E11118079
:101CA8001B0740F1EC8099F89251062D00F2E18073
:101CB800DFE805F004073E6984A2A20045F2F0526D
:101CC80001E042F6F822194B1A800DF0C9F9CFE06D
:101CD800C0300020000C0140340600204C060020D3
:101CE800500800201A00002035FA8E3C6C080020AD
:101CF8000AE81C4100401C4680070020BD37863595
:101D0800ED1000204C080020EC100020FC2C0020D6
:101D1800182800205E130020A40F0020A80F002020
:101D28009430002088300020382D0020AC08002096
:101D380042F6F822784B1A8011F024F9774911F00D
:101D480075F9774911F068F811F05CFB0023754AC2
:101D580042F823000133122BF9D1734A734940200A
:101D68001160734A137006F067F8002800F081804C
:101D780001234FF0070C90F9000040218DE808106E
:101D88006C4A6D4B6FE042F6F822634B40201A8094
:101D98006A4A654B1A60664B10221A7006F04CF8B6
:101DA800002866D001234FF0000E90F90000402172
:101DB8008DE80840624A4FF4E13354E042F6F822D5
:101DC800554B40201A805F4A574B1A60584B0822DF
:101DD8001A7006F031F800284BD00123002590F93D
:101DE800000040218DE82800574A4FF4E13306F0FF
:101DF800D6F9C6F8E00138E042F6F822464B4FF033
:101E08000C0E1A804A4B51485149524A83F800E057
:101E1800062D4FF00003504C03700B7013700AD05E
:101E28001B2323704D4B052283F800E04C4B4FF4E5
:101E3800E1351A7007E021232370484B83F800E04E
:101E4800474B1D70474D484A374B40201A6005F0F4
:101E5800F3FF70B10123002490F900008DE8180009
:101E68002B46424A402106F09AF9003018BF01205B
:101E780028B9082008F094FA3D4A2B4B1A603B68B1
:101E88002B4A13F4804F1FBF082111703948264987
:101E980018BF086042F20101194099B144F6206068
:101EA8001D490880980441BF0821117032481E4915
:101EB80048BF0860D90741BF0C2111702F481A4943
:101EC80048BF086011781D06A1F10401517040F166
:101ED8009480DFF8BC902A4DC6F8E491002631467C
:101EE8001522284C28486E706E60AE6014F0FFFD15
:101EF800A9F105033046236009F057F8234B022067
:101F08001B68A246EB6005F097FF002842D18020AD
:101F180008F046FA69E000BFAC080020CDCCCC3F01
:101F28000000B044982F0020300000204D2A0108FE
:101F3800B4280020F12B0108A0860100392A0108E5
:101F4800452B0108252A0108F92A010884300020B8
:101F5800F1270020F02700201328002083300020DC
:101F68001428002090D0030015EE000845EE000864
:101F7800A92A01087D2A0108992A0108892A010845
:101F88009C070020BC070020B0020020202D002064
:101F9800C813002046796B78BA490C2202FB031259
:101FA8005278B24204D00133DBB2042BF4D90023B7
:101FB8006B70DAF800306A781B7890F90000002B13
:101FC8004FF00C0303FB021314BF03260126002263
:101FD8005B7800960192022106F0E1F8AA4B18609E
:101FE800002894D0012008F0E0FFA84B1868A84BFF
:101FF80000F5C5721A6009F07FF83B689C056CD53E
:10200800A44AA54D049BA5482B6093690DA943F0EC
:1020180001039361049B1B88ADF8343010238DF8BD
:10202800363002238DF837300AF00CFF2B689B48B6
:102038005B880DA9ADF8343004238DF836300AF0EA
:1020480001FF28680F21037A03F0030203F0FC0361
:1020580003F1804303F580339D689200914025EA9F
:10206800010199609968012505FA02F20A439A600C
:1020780042688B4BD1435A611E680E401E605E68F1
:102088000E405E601E6816431E609E680E409E608D
:10209800DE683140D960996811439960D9680A436C
:1020A800DA60437A15A88DF8543003238DF855303B
:1020B80000238DF856308DF8575010F01FF8794BE3
:1020C800794A1B683C3B1360784A136843F0100355
:1020D8001360774B4FF0FF321A60764B764A774D94
:1020E8001360774A803313603B680026D8032E704C
:1020F80040F1AA8040F22A3ADFF8F4B1654C0EF0BC
:10210800EFFA4FF0010952465846314685F80090DB
:1021180014F0EDFCA3696B4843F00403A36140236A
:10212800ADF8303018238DF833300CA903238DF81F
:1021380032300DF019FAE369634943F00203E361B1
:10214800624B634D1B68A4F69474B3FBF1F32988C2
:10215800013B21F45C710904090C29809BB21D2103
:10216800A9852B85A5F814902B8C23F001031B045B
:102178001B0C2B842B8CA888298B23F0020321F0BD
:10218800730109041B04090C1B0C41F0600180B2A7
:1021980043EA0903A8802983AE862B842B8B23F07E
:1021A80008031B041B0C43F008032B83B5F84430C9
:1021B8006FEA43436FEA53439BB2A5F84430D4F81F
:1021C800A83F43EA0903C4F8A83F20460CF0E0FF03
:1021D800404BCDF858B0159380231A934FF4807371
:1021E8004FF0100B1B9320464FF4005315A91E9374
:1021F80019961C961D961F96CDF85CB0CDF860A078
:102208000CF0A8FFAB890DA89BB243F40073AB8117
:10221800236843F0020323608DF834B08DF83590BD
:102228008DF836608DF837900FF068FF2A4B1A68E2
:102238002A4B43F8282008F10108B8F1200FF5D1FE
:102248000AF022FD0AF020FD3B68590540F1908014
:10225800234D244BD5F828A50420C3F800A005F089
:10226800EBFD0421C5F82C0505F0C2FD1E4B85F8D1
:1022780030050820C3F800A005F0DEFD1B4B08213F
:10228800186037E084910108D01A0020241100203A
:10229800001000200010024098070020000C0140A8
:1022A80000040140202D002094070020C4190020BC
:1022B80044110020FC130020181B0020710E002080
:1022C800141B00200008014000366E015000002059
:1022D800000400403404004010910108720E0020F0
:1022E800C8000020B8190020101A00205C1A00202D
:1022F800C502002005F07CFD5C4E85F83105002103
:1023080030462C2214F0F3FB8E2373704FF07C09B7
:10231800E0234FF07D08F37086F8009086F82B8054
:10232800534E2C220021304614F0E1FB8A237370AF
:102338001020A023F37086F8009086F82B80C5F84B
:1023480034A505F079FD1021C5F8380505F050FDD4
:1023580085F83C052020C5F840A505F06DFD202135
:10236800C5F8440505F044FD85F848050BF028F943
:102378003B68404A13F4002318BF0123137005F08B
:1023880087FE3D4B18603D4B5A79052A02BF3C4AEF
:102398004FF4C87111803B4A4FF47A7111803A4A60
:1023A800C821118039490A7842F008020A70384970
:1023B8000A7822F002020A7040F6020239680A40DE
:1023C8006AB13448344A1060344A03201070344AE1
:1023D80001201070334800220280334802808A03AB
:1023E80042BF324A042111719B6848BFD1783B60D3
:1023F80048BF41F001012E4B48BFD17001221A702D
:10240800039B039A1B7863F07F03137021B0BDE828
:10241800F08F284B00221A7000B210F0B3FD264945
:1024280010F004FE1590B7F95E0110F0ABFD2249DB
:1024380010F0FCFD1690B7F9600110F0A3FD1E49DD
:1024480010F0F4FD1D491790484607F0C1FEFEF74D
:1024580082BD0226FFF761B8B9F1010F7FF693AA92
:102468004FF000092070FFF7DBB800BFE01900202B
:10247800151A00205C2D00208C080020D4110020A3
:10248800B60F0020DE300020DC300020C819002004
:10249800E730002050130020B0190020141A002043
:1024A80044000020A0100020A2100020D41A002010
:1024B800700E00203800002035FA8E3CF8280020E5
:1024C800954A2DE9F04F1568944C05F59C43944EB8
:1024D80020332360336889B013F4804F059205D107
:1024E80010F04CFC10B92379013323718D4A13780D
:1024F8004BB18D4909688D4240F2E58003F1FF3800
:1025080082F80080DFE09846884B5FFA88F51F78EC
:10251800DFF83892AF4231D9D9F80030072D98BF8B
:10252800595D834B88BF29461B6880489847032D0F
:102538001ED8D9F8002005F10E0302EB8303998811
:10254800DA88A8B14FF47A73401A5843531A90FBAB
:10255800F3F040F6C90300F57A70984205DC40F2C2
:10256800EE239842B8BF184601E040F6CA0080B290
:1025780004EB4505E88008F10108C5E794F80480F4
:102588000325B8FBF5F50F2384F82A3094F82B308F
:1025980005EB4505019394F82C30C5EB080503932A
:1025A800D9F80030DFF8ACA10293EBB20493002510
:1025B800BD4255DA5F4B4FEA450933F815B0019B28
:1025C80053B910F0DBFB28B1039B002B08BF4FF079
:1025D800000B01E0DDF804B0029B988A584502D848
:1025E800D88A58450ED2E8B210F072FB032D834604
:1025F800DFBF94F82AE00120A8402EEA0000D8BFE7
:1026080084F82A0010F0BAFB18B14B4829F800B03A
:1026180022E0049B94F876002AF813B030B9B8F198
:10262800020F15D93D4B012083F87600BAF8000057
:10263800BAF802300344BAF8040003443F489BB296
:1026480029F800301BB2032093FBF0F39BB200E0A3
:102658005B46394829F8003001350AF1060AA7E730
:1026680094F82A203648A2F10F014A424A4184F8D8
:102678009020344B6AB1344A1268520109D4026876
:10268800D9689A60521AC82A1DD9012283F82120D4
:1026980019E002689868DA605B68121A9A4288BF83
:1026A800284B4FF0000184F82B1088BF83F82110C5
:1026B8000025BD4207DAE8B210F00AFB1E4B23F8EA
:1026C80015000135F5E73368DD0405D51E4B1B6899
:1026D800D80701D410F05AF9059B1F681B4B1A68DC
:1026E800907A002838D01449137B013831F810004B
:1026F8001BB1C0F53B60083080B200B2A0F57A701B
:10270800B0F57A7FA8BF4FF47A7020EAE07010F035
:1027180039FC0F4955E000BFCC300020F80E0020EE
:10272800FC2C0020903000208C300020B4280020A1
:1027380030000020FE0E0020382D0020700F0020F1
:10274800202D002094300020E81000208830002040
:1027580000007A44260F0020336819043AD5D4F8CB
:102768009430934DFB1A002B34DB07F59C43203340
:10277800C5F894308F4BD27A59798F4B33F8113092
:1027880095F898109BB293FBF2F3013101F00F0218
:1027980085F898202A4482F899300346874A825C53
:1027A8000130134410289BB2F8D11BB293FBF0F010
:1027B80000B26428A8BF642020EAE07010F0E2FBB1
:1027C8007F4910F0E7FC7F4910F030FC10F01AFE4A
:1027D8007D4B188033687D4D13F4807F00F00F81A6
:1027E8007B4BDFF8F0919F4205D999F8022012B986
:1027F800012289F8022099F80220002A00F0FF80BF
:10280800744A95F8008092F82170C8F380087A1EFF
:1028180057425741704A002F9246116818BF4FF02F
:10282800000BC1F38063019308BF4FF0030B99F8C5
:102838002020052A00F2DD80DFE802F0034E5379FC
:1028480088A5B8F1000F3AD0D4F8AC00B4F8B010AD
:1028580005F08FFB012809D16049614A09681268AF
:10286800C988642000FB0122C9F81020019B6BB1C4
:102878005A4A126812794AB10CF090FA032289F880
:1028880020204FF47A72C9F81C20D0E7002F40F0BE
:10289800B080534AD9F8101010684E4A88420AD9B5
:1028A80002920CF07BFA029A032182F8201040F67B
:1028B800B831D161BBE7012182F82010B7E7019B4D
:1028C8004FF4806013B107F05BFD01E007F047FDAE
:1028D8000022C9F810208CE0002F49D10CF05EFAD4
:1028E800A5E727B1052289F82020012000E0384615
:1028F800B8F1000F0CD0D4F8AC204FF0020BD189FE
:10290800384A118051809180344909684988D180BA
:10291800334A1168D9F81420914202D8B8F1000F4F
:1029280064D147F23052C9F81C20032221E02A78EA
:1029380042F002022A7010F029F8294AD9F81C102E
:1029480012680A44C9F81820042212E0244A9FB1E8
:102958001168D9F8182091424BD9234A12781AB92C
:10296800DAF80020D30744D42A7822F002022A7029
:10297800052289F820205AE71268D9F81C100A4461
:10298800C9F8182035E01549154A09681268C98838
:10299800642000FB01224FF48060C9F81020002257
:1029A80089F8202089F8032007F0D9FC3FE700BF09
:1029B800F80E00201C2900202C290020910F00204F
:1029C8000000C84200C07F4448110020E7300020C2
:1029D800404B4C0094300020E8100020CC27002009
:1029E800202D0020382D00201800002000287FF41A
:1029F8001EAFBBF1000F02D0584605F00FFB934FF6
:102A080007F5C570B7F8521105F0B3FA0197834678
:102A180068B90CF0B5F98E4B0022C3F800B0C3F8C2
:102A280004B0C3F808B08B4B1A605A609A602B78D0
:102A38005F0736D53368D80633D5874B1B78D90658
:102A48002FD4864B1B789BB1019B93F8E231BBF1E5
:102A5800000F15D17BB1824B1A68D4F8B4309B1A99
:102A6800002B08DA0FF092FF7E4B83F8B8B018E01D
:102A7800BBF1000F0DD1102005F0D0FA01230EE0B4
:102A88003BB1774A4FF47A71126801FB0323C4F80B
:102A9800B43094F8B83023B105F0AEFA002384F8C6
:102AA800B830019B93F8E0A193F8E111B3F89AE1EB
:102AB800B3F89CC1002318466B4F800837F91320E0
:102AC80001337245C4BF60F07F00C0B26245B8BF31
:102AD80040F04000042BB946EED194F8B930614A71
:102AE800834205D192F8BA30F92B04D8013300E0BB
:102AF800002382F8BA30594B84F8B9001A785B4F32
:102B08009846E2B93B68DA0708D5BBF1000F16D141
:102B18002B78DB0713D50FF095FD10E02B785807BD
:102B28000DD5504B93F82B304BB1514BDB7833B963
:102B380011B10FF02BFF02E0BBF1000FF9D094F8B0
:102B4800BA30484A142BDFF83CB140F0AD8098F811
:102B580000301AF1000A18BF4FF0010A6BB392F85F
:102B6800B9305F2B11D12B7803F0040303F0FF0178
:102B780013B10FF00BFF08E00B200391029205F050
:102B88004DFA029A039982F8BA10BAF1000F14D0DC
:102B980094F8B9307D2B10D12B7803F0040303F09F
:102BA800FF0213B10FF0F2FE07E00B20029205F0CE
:102BB80035FA2C4B029A83F8BA202B7803F00403D9
:102BC80003F0FF01002B6FD194F8B930254A572B39
:102BD80015D1284B4FF47A721A803368190601D53B
:102BE80008F0DAFA244B1B685A0742BF234A0A2125
:102BF800118013F0080357D1214A138054E030683C
:102C0800400717D55A2B15D192F8BB302BB10123A9
:102C180082F8BB1082F8BC3046E092F8BD3083F0F1
:102C2800010382F8BD300BB10C2000E00D2005F047
:102C3800F5F939E05D2B00F018855B2B00F017855E
:102C48005E2B21D1032000F013BD00BFD41100205A
:102C5800E02900205C2A0020C81900201800002064
:102C6800202D0020F80E0020382D0020E81000202C
:102C780094300020DE300020C4190020DC30002011
:102C8800C411002024110020562B03D1029307F011
:102C980023FE029B98F80020002A00F0FF846F2B87
:102CA80040F0F6840FF0CEFC3368580736D594F818
:102CB800BD30B64A93B12B7859070FD5019BB9F9A6
:102CC8000610B3F89A31994208DD3B6813F0010306
:102CD80002BF3221A2F8C01082F8BD303B68DA0387
:102CE8000DD594F8C220A94B2AB993F8BB2012B984
:102CF8003222A3F8C020012384F8C2300EE094F8F1
:102D0800BB30A24A53B12B7803F0040303F0FF0150
:102D180023B9012382F8BB1082F8BC30DBF800909D
:102D280000233B6009F17B0809F1CB0A98F80020E1
:102D380098F8013018F8010C9A420BD2414605F078
:102D4800E3F838B118F8022C012303FA02F23B68C1
:102D580013433B6008F10408D045E7D18C4B1B783E
:102D680053B18C4B8C4F1A68984612F0020FDFF85B
:102D7800409240F032832AE309F1CA0709F58978BD
:102D88003A787B7817F8010C9A4225D2394605F033
:102D9800BBF808B397F804E00C21BB7801FB0E419F
:102DA8007E4A013B03EB43031344D1F8C82097F84C
:102DB80003909A4275480FD0C1F8C830002390F8A4
:102DC800F420C1F8CC30012303FA0EF322EA0303FE
:102DD80081F8C49080F8F43006374745D0D1704B5D
:102DE800DFF8D0A1D3F800806E4B4FF0000B1B68C2
:102DF800029394F82B300393DAF80030002B00F09C
:102E0800DD8293F80090B9F1000F00F0D782DAF86C
:102E1800042002998A1A002A0CDB01F5FA72CAF812
:102E2800042094F8F410012202FA0BF221EA0202BB
:102E380084F8F420039A002A00F0C0821AF8042CBF
:102E480059780432D2B2002940F07982564931F9D2
:102E58001210564AB2F8982102F1C800814201DDE9
:102E68009F7814E0C83A914202DA99784F420EE00E
:102E780094F8F420012303FA0BF322EA030384F8FD
:102E8800F430029B03F5FA73CAF8043096E294F81A
:102E9800F43043FA0BF3DB0700F19082002FCCBF2C
:102EA8000220012005F0DCF809F1FF32374B132A24
:102EB80000F27C82DFE812F01400230032004400A4
:102EC80061008000E5004A01AF01E40113027A02C3
:102ED800440055008000E5004A01B7001C0181014B
:102EE80098F8001040460F44FA2FA8BFFA2727EA9F
:102EF800E77788F8007004F0EDFF01201EE098F8ED
:102F0800011040460F44642FA8BF642727EAE777DB
:102F180088F8017004F0DEFF02200FE098F8031033
:102F280040460F44642FA8BF642727EAE77788F84C
:102F38000370D3F8F81004F085FF03203946CBE17D
:102F480098F805100D2039446429A8BF642121EAA6
:102F5800E17188F8051005F03BF8B9F10D0F00F0A4
:102F6800258298F804100E2039446429A8BF6421EA
:102F780021EAE17188F80410AEE198F806100520FE
:102F8800394481F3080188F80610A5E1F80E0020FD
:102F9800E8300020E8100020C4190020C892010879
:102FA8004C110020202D0020382D0020D4110020A5
:102FB8008C1A0020C00F0020D3F8FC301A78022A9F
:102FC80022D1384604930FF0DDFFA94910F0E2F84A
:102FD800049B596A05930FF021FF0021049010F01B
:102FE800C3F9059B48B9049AA249104610F0DAF9CA
:102FF800049A059B10B19F4A00E000225A620F20F4
:10300800114604F0D1FF0AE099780F203944C82905
:10301800A8BFC82121EAE171997004F0D9FFB9F17C
:103028000F0F00F0C381944BD3F8FC9099F800304F
:10303800022B1AD138460FF0A5FF8D4910F0AAF8D7
:10304800D9F820100FF0EAFE0021074610F08CF99D
:1030580030B93846874910F0A5F910B1854F00E01E
:103068000027C9F82070122059E199F801101220A0
:103078003944C829A8BFC82121EAE17189F801109B
:103088002AE1D3F8FC301A78022A22D13846049370
:103098000FF078FF774910F07DF8049B196B0593C2
:1030A8000FF0BCFE0021049010F05EF9059B48B9B2
:1030B800049A7049104610F075F9049A059B10B1EE
:1030C8006C4A00E000221A631020114604F06CFFDD
:1030D8000AE0197B10203944C829A8BFC82121EA71
:1030E800E171197304F074FFB9F1100F00F05E81FB
:1030F800614BD3F8FC9099F80030022B1AD138466E
:103108000FF040FF5B4910F045F8D9F82C100FF08C
:1031180085FE0021074610F027F930B93846554991
:1031280010F040F910B1534F00E00027C9F82C7097
:103138001320F4E099F80B1013203944C829A8BFCC
:10314800C82121EAE17189F80B10C5E0D3F8FC30F9
:103158001A78022A22D1384604930FF013FF474900
:1031680010F018F8049BD96B05930FF057FE002157
:10317800049010F0F9F8059B48B9049A3D491046A7
:1031880010F010F9049A059B10B13A4A00E00022A9
:10319800DA631120114604F007FF0AE0997D112037
:1031A8003944C829A8BFC82121EAE171997504F0FA
:1031B8000FFFB9F1110F00F0F9802F4BD3F8FC90F5
:1031C80099F80030022B1AD138460FF0DBFE2B4954
:1031D8000FF0E0FFD9F838100FF020FE0021074665
:1031E80010F0C2F830B93846224910F0DBF810B1B7
:1031F800204F00E00027C9F8387014208FE099F8B4
:10320800151014203944C829A8BFC82121EAE17142
:1032180089F8151060E0D3F8FC9099F80030022B7B
:103228001AD138460FF0AEFE11490FF0B3FFD9F8A6
:1032380028100FF0F3FD0021074610F095F830B97B
:1032480038460C4910F0AEF810B10A4F00E00027DC
:10325800C9F82870092062E099F803100920394458
:10326800C829A8BFC82121EAE17189F8031033E011
:10327800000020410000C842F80E002000007A44F7
:10328800D3F8FC9099F80030022B1AD138460FF089
:1032980079FEB4490FF07EFFD9F834100FF0BEFD67
:1032A8000021074610F060F830B93846AD4910F0F3
:1032B80079F810B1AB4F00E00027C9F834700A2044
:1032C8002DE099F80D100A203944C829A8BFC82153
:1032D80021EAE17189F80D1004F07AFE66E0D3F86E
:1032E800FC9099F80030022B1DD138460FF04AFEA9
:1032F8009D490FF04FFFD9F840100FF08FFD0021C6
:10330800074610F031F830B93846964910F04AF8B7
:1033180010B1944F00E00027C9F840700B203946DF
:1033280004F042FE42E099F817100B203944C829EE
:10333800A8BFC82121EAE17189F81710CCE7012953
:1033480034D19878894B33F91230B3F5617F05DBB6
:1033580040F633029342A8BF134601E04FF461736D
:10336800B9F10C0F22D14FF4966292FBF0F0A3F55D
:10337800617393FBF0F37E4ADFB21378BB4215D03A
:10338800042F34BF3B4602231370019A09FB032321
:10339800784A03F2B27313600EF01AFB48463946B6
:1033A80004F016FE781CC0B204F05AFE94F8F4201B
:1033B800012303FA0BF3134384F8F4300BF1010BE8
:1033C800BBF1040F0AF10C0A7FF416ADC9E43368A7
:1033D800D80510D5684BDB786BB13B6899070AD5DF
:1033E800B9F8003013F0010A0AD10BF0C9FC01202A
:1033F80006F0C6FF04E0012006F0B1FF012300E05B
:103408000023D8F8002052070DD563B1012006F03B
:10341800A6FFB9F800309B0708D40BF0B1FC0220D6
:1034280006F0AEFF02E0022006F099FFB9F800307E
:10343800524A13F0030F4FF0100114BF516111618C
:103448003A6812F00A0F27D0D8F80020D00609D51C
:1034580059070AD4042006F093FF494B1B88A4F8A7
:10346800003102E0042006F07AFFD8F800309A060E
:1034780007D5B9F800305B0606D4402006F080FF77
:1034880002E0402006F06BFFD8F80030580642BF33
:103498003B4B1B88A4F802313B68990609D4D8F83D
:1034A80000301A0540F1B0804FF4807006F068FFD4
:1034B800AEE0344B1B789B076ED5334B1B78042B3F
:1034C8006AD9D8F8003013F4007A0FD0B9F8003070
:1034D800DF063AD4102006F053FF202006F03FFF05
:1034E8002A48011D07F0C2FD02232AE0B9F800703E
:1034F80007F01007BFB22FB1102006F030FF0127E8
:1035080084F804A1D8F80030580512D5D4F8083149
:103518001F495A89B1F90030002BB8BF5B4293426A
:1035280007DAB1F90230002BB8BF5B429342C0F210
:103538000581B9F80030990608D5202006F00FFF5C
:10354800002384F80431012700E0002794F80C31A7
:103558009BBB0E2004F062FD0E4B012283F80C2168
:103568002BE000BF0000C84200007A44382D00203C
:10357800A82C00204C11002094300020000C0140A1
:10358800C4110020C8190020CE19002054110020B1
:10359800CC110020F80E0020B9F8003003F03003F9
:1035A800002B3FF47CAF102006F0D9FE202006F057
:1035B800D6FE002384F8043102E0002F3FF46FAFF9
:1035C800002214466A4B002023F81400694B191D89
:1035D80003F10A0721F814000021D151174478603B
:1035E800B96023F8140003F132075A33D151D1508E
:1035F800174413447860B960586099601432002CFD
:103608007FF44DAF0124DDE74FF4807006F0A7FE8C
:10361800594B5A791C46082A01D00E2A02D140205B
:1036280006F09DFE33685A0540F19E8094F81832E2
:103638001BB92B7813F0040F03E0D8F8003013F40B
:10364800002F0BD04D4B00221A703C200BF050FD80
:10365800002800F089800DF0C1FEF6E709F0B0FF00
:1036680009B0BDE8F04F0BF072BC012000E0022069
:103678005FFA80F8019A08F1FF3382F8B03706F054
:10368800C1FE06F065FF404604F0EAFCFFF70CBBFC
:10369800BAF1000F02D07E2B3FF404AB972B05D173
:1036A8004FF4C873A4F8BE30FFF7FEBAA72B06D1B3
:1036B800334A137843F004031370FFF7F5BA002276
:1036C800BB2B079201D1022303E0B72B04D14FF69D
:1036D800FE73ADF81E3009E0BE2B01D1022303E0D2
:1036E800BD2B1AD14FF6FE73ADF81C30DBF8003055
:1036F800BDF81C10B3F858200A44A3F85820BDF8A8
:103708001E10B3F85A200A44A3F85A2007F0E4F828
:10371800002384F8BA30FFF7C7BA792B04D1194AC5
:10372800D37823F0010306E07A2B7FF4BDAA154A6B
:10373800D37843F00103D370FFF7B6BAB9F8003075
:103748009B063FF503AF202006F01AFE0E4B0F48EC
:103758001A685B68011D4360026007F087FC0C4B28
:10376800012783F80471F1E609B0BDE8F08F00BFC6
:10377800E030002006100020D4110020B9280020D5
:10378800C8190020D41A0020D01900205C1100208C
:10379800F80E0020B54B2DE9F04FB3F90610B44BE5
:1037A80085B01F6801937A8991420EDBB1F5FA6FF3
:1037B800FC79BFBF8B1A6343A2F5FA6493FBF4F458
:1037C800ACBFC4F16404643400E06424A94BAA4A81
:1037D800B3F898B193F9623112689BB20292154618
:1037E8000393002240F2E630A04B4FEA420C33F933
:1037F80012E0CBEB0E0303F2F316864203D8002B3C
:10380800B8BF5B4201E04FF4FA73022A2ED0029E41
:1038180096F811611EB1B342CCBF9B1B00236420F4
:1038280093FBF0F8954E6FF0630A36F818900AFB90
:10383800083A08F1010836F918600FFA89F8C8EB58
:10384800060606FB0AF696FBF0F68D484E4420F86D
:103858000C60BE183679642073438A4E93FBF6F3E6
:1038680064339BB2634393FBF0F02CE0029890F82A
:1038780012611EB1B342CCBF9B1B0023642093FB93
:10388800F0F0DFF82C926FF0630808FB003A39F982
:103898001060013039F91000002BA0EB060000FB86
:1038A8000AFA9AFBF8FA0398C6EB0A0A0AFB00FA26
:1038B8007348B8BF5B42A0F804A0B8794343714885
:1038C80093FBF0F064306B784FF06408434393FB4C
:1038D800F8F36D4E022AB354EB7A6C4E00FB03F3F7
:1038E80093FBF8F3B3546B7D654E00FB03F090FB3C
:1038F800F8F0674B9854674B0ED1DE4583F8028089
:103908000DDB5C4CB4F89A21914214DBB1F5FA6FE7
:10391800A8BF4FF4FA610FE0DE459C5404DA36F88C
:103928000C305B4226F80C300132032A05F1010500
:103938007FF458AFE5E71146891A4FF47A73594373
:10394800C2F5FA62B1FBF2F1642391FBF3F2DFF8FE
:1039580074E16FF063073EF8120007FB02110132B1
:103968003EF9122007B2D21B514391FBF3F30344F3
:10397800F380494B424D1B885F063BD5474A484B6D
:1039880010881B88181A00B20FF0FCFA45490FF08E
:103998004DFB074606F012FC8046384606F09BFBB6
:1039A8000746B5F902000FF0EDFA8146B5F90000B7
:1039B8000FF0E8FA414682460FF038FB3946834655
:1039C80048460FF033FB014658460FF025FA0FF032
:1039D800F3FC4146288048460FF028FB39468046CC
:1039E80050460FF023FB014640460FF017FA0FF040
:1039F800E3FC68802C4D2B68980740F19E8045F2C7
:103A080007212A4B2A4F1A687B69D31A8B4240F345
:103A180094807A610BF016FF264BDFF8AC901A7889
:103A28009846032AB9F8003050D10A2B58D90023F8
:103A3800282088F8003004F052FB0BF003FF1E4BDF
:103A480018880BF0E9FE1D4B1A68D37890FBF3F049
:103A5800013008281A4BA8BF08201870537980B283
:103A680043433B8313795843788339E0382D00204A
:103A78004C110020D411002024110020AA1A002083
:103A8800CC1100200CFEFFFF682A002096100020B1
:103A98007C2A0020C02900208C1A0020FA0F002060
:103AA800C411002035FA8E3CFC2C0020CC300020BC
:103AB80088100020141A002034290020B019002092
:103AC80044000020921A0020B41900200A2B07D8BD
:103AD8000323964A88F80030002313703B837B83C6
:103AE80098F80030924A012B0CD002D3022B1BD03D
:103AF80023E03A8BB9F800309A421EDD012388F89A
:103B080000300FE0B9F800107B8B8B4202DD0223F6
:103B180013700FE0874B1B8B0133994202DD0023A2
:103B280013700AE0082006E07B8BB9F80020013307
:103B38009A42E3DC072004F071FA2D68290577D54D
:103B48007D4B7C4F1A68FB69C3EB020845F20723DB
:103B580098456DDD794BB6F906B0D3F800904FF46F
:103B68007A7099F80A30FA61012B98FBF0F8B4F8EA
:103B78005211ABF57A7B724E03D042D3022B20D080
:103B880041E0704B396A5A7B6F4B4FF0080E33F89F
:103B9800122091FBFEF392B2C91A8B183B6293FB79
:103BA800FEF3BA8440F6E4429BB25343B9F80820C6
:103BB800C2EB13335843B9F9063090FBF3F0306089
:103BC80021E0624BB9F808A01B78C6F800A05A0794
:103BD80019D55F4804F0CDF920B915F0100F18BFBA
:103BE8004FF0000B0BFB0BF3322293FBF2F3B9F906
:103BF80006205B445A434FF47A7392FBF3F3534421
:103C080000E0002333603368D7E90A0103FB08F8B2
:103C18004FF47A7398FBF3F810EB080041EBE87166
:103C28000023C7E90A014B4A0FF00CFC4A4B186005
:103C38004A4E3368DB0427D52F0622D5484B1B781C
:103C48009D071ED5474B187804281AD90022464BE1
:103C58000521D718951C4FF00A0E122AD154E9B243
:103C680087F801E004D0B0EB510F2A46EFD800E006
:103C780014215A18322002F8010CFF225A540F203E
:103C880000E00A2004F0CAF9384D2A68002A45D015
:103C9800374B384F18683968984681423ED8364BBA
:103CA800DFF8E09018785168B0B901221A70B9F8B5
:103CB8000030CB5CD3B1314B1A700FF06BF8B9F808
:103CC80000309BB92B681B78053B012B0ED804F0FC
:103CD800DFF92B4B186009E000221A70B9F80030A0
:103CE800CB5C1BB1254B1A700FF054F82B68B9F850
:103CF80000205B6823499B5CFE2B02D100230B80CC
:103D08000CE0FF2B02D104F077F907E0D8F80000A7
:103D18000A2505FB030301323B600A800B4D2B7813
:103D2800580733D5184B08225A616DE0440000202B
:103D3800141A002088100020CC300020B019002070
:103D4800BC1900201C2900202C290020E730002065
:103D58005E130020407E0500C0190020E8100020F6
:103D6800C8190020CE190020D42C0020C41A002025
:103D7800202D0020BC1A0020B81A0020B8300020DE
:103D8800182F0020C01A0020000C01403268D1070B
:103D98005CBF43F001032B70984B1B781F075EBF75
:103DA8002B7823F001032B70D60248BF2B78944A56
:103DB80044BF23F001032B70924B1B6813F0040FD0
:103DC80002D09149098851B99049098809B19807E1
:103DD80005D48F4B1B88003318BF012333B102234E
:103DE80013702B7823F001032B7004E02978C9079E
:103DF80058BF0223137004F04BF9864B1B68C01A96
:103E0800002801DB0EF0C6FF09F0DAFB824B1E78B2
:103E18009846002E00F0AB80804E3368002B00F0EF
:103E2800EC8630680CF058F9002800F0E6867B4BE9
:103E38007B4C18680CF04DF9092801D03F2850D167
:103E48004FF0000A5746D4F80090764DB9F1000FAC
:103E580005D0754829684A4612F096FE10B9AA4658
:103E680007B92F46714B10359D42EFD3C7B1D7F82C
:103E780000E0DAF800C023681EF803501CF80300BD
:103E8800A8420DD15A1C684938B92D2B05D8644D64
:103E98002A602025CD54885402E0CD542260EAE7F8
:103EA80023680BB1574511D061480DF087FB574582
:103EB80007D857F8100B0DF081FB09200DF076FBA1
:103EC800F5E75C480DF07AFB4FF000092368994547
:103ED800A7D2554B13F809000DF068FB09F1010949
:103EE800F4E72368002B40F06D86042840F0AB8689
:103EF8004D4804F0F9FA00F080BED9F80000DFF868
:103F080044A10CF0E9F840B3DAF800000CF0E1F84D
:103F1800DBF80030024693F84810002935D12428F0
:103F280040F09280012283F84820DBF80030DFF867
:103F380010A193F84820062ADFD193F8490001F030
:103F480085FE8146002800F0AA803B6898790DF02C
:103F580082FA3B68002283F84820374B93F83530C3
:103F6800002B40F01D864C36982E00F04686334BC9
:103F7800F21892F84A100129F5D1314FF3583A60F6
:103F8800304ABB4613609146B7E7012904D14D2852
:103F980014BF00220222C6E7022904D13C2814BF1C
:103FA80000220322BFE703290CD140284FF000016B
:103FB80002D983F84810B8E758711971D971987106
:103FC8000422B0E7042906D1997983F849004A40C8
:103FD8009A710522A7E70529A7D158791979884246
:103FE800987906D950409871481C18710B441A7278
:103FF8009BE790420CBF0622002294E7C8190020D4
:10400800B8300020C4190020DC300020B60F002092
:10401800DE300020BC300020E8300020C42C002016
:10402800101B002070990108E01A0020209B01084D
:104038004FB5010854B50108881000201828002041
:104048006C1A0020701A00202B78D84958073FF5C1
:104058006CAF232ADAF8003014D1012088F8000068
:10406800D34803910360D34802920363D2480DF00A
:10407800A5FAD2480DF0A2FA0399029A0B7843F0F8
:1040880002030B70CE4B1B681B78934201BFCD4ACD
:10409800CD4B1A60CD4A04BFCD4BDA6045E7DAF85C
:1040A800002092F849304C2B00F069845DD8332BFE
:1040B80000F0A08421D8292B00F02D8409D8252BC5
:1040C80000F00484272B00F00884232B40F0B785E8
:1040D8002FE22D2B00F0308407D82B2B40F0AF8532
:1040E8000DF09CF9607100F03EBD2F2B00F0EE84BE
:1040F800312B00F0008500F0A2BD3E2B00F0F280CD
:104108001DD8372B00F0AA8404D8352B00F04A823A
:1041180000F095BD392B00F0ED833C2B40F08F85E6
:10412800DFF8B092D9F800A00DF078F98AF800000D
:10413800D9F8003018780CF03FFA00F014BD432B82
:1041480000F0698406D8412B40F079854FF00009CA
:1041580000F055BC442B00F002854A2B40F06F85D7
:104168000DF066F9A08100F0FEBCD02B00F01083A2
:1041780055D8CA2B00F0C08009D8C82B00F085801C
:1041880000F23E834E2B00F0078400F058BDCD2B83
:1041980000F0098304D8CC2B00F02C8200F04FBD2E
:1041A800CE2B00F00983CF2B40F049850DF040F964
:1041B8006FF4AF6283189BB2C62B98BFA4F898011E
:1041C8000DF036F9A4F844010DF032F9A4F84601CF
:1041D8000DF02EF9A4F848010DF02AF9A4F8DA0137
:1041E8000DF01CF984F8EF010DF018F90DF016F92F
:1041F80084F8F0010DF012F984F887010DF00EF93A
:1042080084F894010DF00AF9724BD3F800900DF080
:104218000FF900EB80004000A9F856006AE3D62B9E
:1042280000F03B820AD8D22B19D0C0F01083D32BD0
:1042380025D0D42B00F03C8200F001BDEF2B41D0FB
:1042480005D8D82B40F0FB844FF0000904E1F22B8D
:1042580000F07682FA2B00F0B88200F0F0BC2B78E0
:10426800590700F180840DF0D9F8022884F8B007C6
:1042780040F29482584B002283F8B0278EE20DF06A
:10428800D7F8564B188000F06EBC92F805904FEAAC
:104298005909B9F1120F03D90AF026FF00F063BCDF
:1042A8004FF0000ACA4507D20DF0C2F84C4B23F86C
:1042B8001A000AF1010AF5E73E4B012283F834207F
:1042C80000F051BCDFF80C91D9F800A00DF0B0F85F
:1042D800AAF85A00D9F800900DF0AAF8A9F85800E1
:1042E80000F041BC0DF09AF884F8E2010DF096F860
:1042F80084F8E10100F037BC364B1A689A46127808
:10430800022A40F08E80DAF8003009F1080B029397
:104318000DF084F80EF032FE32490EF03BFF029B9E
:1043280043F82B00DAF800B00DF078F809F10A0329
:104338000BEB830B0EF022FE2B490EF02BFFDAF865
:104348000030CBF8040002930DF068F80EF016FE6A
:1043580026490EF01FFF09F10E0B029B09F1010916
:10436800B9F1030F43F82B00CDD1B9F1070FDAF8F3
:1043780000B03DD10DF052F80EF000FE19490EF0D4
:1043880009FFCBF84400DAF800B00DF047F80EF05A
:10439800F5FD14490EF0FEFECBF84800DAF800B03F
:1043A8000DF03CF88BF84C0035E000BFE7300020FA
:1043B800C42C00208810002084B5010854B50108D9
:1043C800BC280020EFBEADDEF04F00200400FA0547
:1043D80000ED00E024110020D4110020F80F002087
:1043E800382D0020000020410000C84200007A4417
:1043F8000DF014F8CB448BF80100DAF800B00DF09A
:104408000DF8CB448BF80B00DAF800B00DF006F885
:10441800CB448BF8150009F10109B9F10A0FA4D1B1
:10442800A1E3DAF800B00CF0F9FFCB448BF80100F7
:10443800DAF800B00CF0F2FFCB448BF80B00DAF896
:1044480000B00CF0EBFFCB4409F10109B9F10A0FF8
:104458008BF81500E5D186E3DFF890A309F1080B86
:10446800DAF8003002930CF0E3FF0EF087FDD9492B
:104478000EF090FE029B43F82B00DAF800B00CF027
:10448800D7FF09F10A030BEB830B0EF077FDD14937
:104498000EF080FEDAF80030CBF8040002930CF03E
:1044A800C7FF0EF06BFDCB490EF074FE09F10E0B41
:1044B800029B09F10109B9F1030F43F82B00CBD195
:1044C800B9F1070FDAF800B01AD10CF0B1FF0EF00D
:1044D80055FDC0490EF05EFECBF84400DAF800B096
:1044E8000CF0A6FF0EF04AFDBA490EF053FECBF8C9
:1044F8004800DAF800B00CF09BFF8BF84C0012E093
:104508000CF096FFCB448BF80100DAF800B00CF001
:104518008FFFCB448BF80B00DAF800B00CF088FF63
:10452800CB448BF8150009F10109B9F10A0FC7D17D
:1045380019E30CF073FF132883463FF6ADAEDFF89E
:10454800ACA2DAF800900CF069FF0023A2490C2213
:1045580002FB0312117A814220D1137809EB8B09EF
:1045680089F879300CF05AFF89F87A000CF056FF78
:1045780089F87B000CF052FF984A994B89F87C0027
:104588001A60DAF80000974B00211860793003F0C0
:10459800DFFC954B80F001001870E4E201331C2B1E
:1045A800D4D179E60CF03AFF0B2882463FF674AE78
:1045B8008E4BD3F800900CF031FF03283FF66CAE19
:1045C800062303FB0A9989F8CE000CF027FF89F827
:1045D800C9000CF023FF89F8CA000CF01FFF89F806
:1045E800CB000CF01BFF89F8CC000CF017FF89F802
:1045F800CD00B8E25379092B7FF64EAE019BD3F874
:1046080000900CF00BFF019B89F80000D3F8009094
:104618000CF004FF89F801000CF000FF019B6428EE
:104628001B68A8BF642018710CF0F8FE019B642871
:104638001B68A8BF642058710CF0F0FE019BFF288E
:104648001B68A8BFFF2098710CF0E8FE019B642846
:10465800D3F8009028BF642089F807000CF0DEFE2C
:10466800019B89F80200D3F800900CF0D7FE019B5B
:1046780089F80300D3F800900CF0DAFE3B68A9F83B
:104688000A005B790A2B40F26E82594BD3F80090EE
:104698000CF0C4FE89F8080065E20CF0C9FE554B21
:1046A80023F8190009F10109B9F1080FF5D15AE207
:1046B80053790F2B7FF4F0AD0CF0B0FE072881463C
:1046C8003FF6EAADDFF824A1DAF800B00CF0B0FE4E
:1046D8000E2303FB09F9CB44ABF81901DAF800B053
:1046E8000CF0A6FECB44ABF81B01DAF800B00CF0D6
:1046F8009FFECB44ABF81D01DAF800B00CF08EFE3B
:10470800CB448BF81F01DAF800B00CF087FECB44DD
:104718008BF82001DAF800B00CF080FECB448BF85F
:104728002101DAF800B00CF079FECB448BF82201B5
:10473800DAF800A00CF086FED144C9F8230112E291
:104748000CF06CFE0F2881463FF6A6AD0CF066FE15
:10475800C9EBC909A14489F8D4000CF05FFE89F8B7
:10476800D5000CF05BFE89F8D6000CF057FE89F8EE
:10477800D7000CF053FE89F8D8000CF04FFE89F8EA
:10478800D9000CF04BFE89F8DA000BF067FEEAE17D
:104798002B785B0700F1E7810DF060F905F032FE38
:1047A80005F0D6FEDFE12B78580700F1DC81124BCB
:1047B8004FF4C8721A80D6E12B78590700F1D381DB
:1047C8000E4A137843F004033FE02B785A07E5D5E7
:1047D80035E200BF00007A44349301081813002022
:1047E800F00F0020F40F00201800002024110020F2
:1047F8004C110020AA2C0020B60F0020C819002058
:104808000CF00CFEDA4B1A7810B142F0020201E00B
:1048180022F002021A700CF001FED64BDFF87893F2
:1048280018700CF00FFEC9F800000CF00BFEC9F868
:1048380004000CF0FDFDD04B18800CF0F9FDCF4BB7
:10484800CF4A1880137843F0020313708BE10CF001
:10485800E5FD02900CF0F6FD83460CF0F3FD824670
:104868000CF0F0FD81460CF0E3FD0CF0E1FD0CF0DE
:10487800D5FD029BA3B9C34B1020C3F800B0C3F801
:1048880004A005F06CFDBA4A137843F001031370D5
:10489800B9F1000F00F06781BB4BC3F8009062E1EB
:1048A800102B40F06081B94BC3F800B0C3F804A0E6
:1048B800B9F1000F02D0B44BC3F80090B348B44B21
:1048C8000222011D1A7006F0D1FB4CE1A0600CF029
:1048D800B9FDA3681843A06045E10CF0A9FDA4F850
:1048E8005C010CF0A5FDA4F85E010CF0A1FDA4F894
:1048F800600138E10CF092FD84F87C010CF08EFD2B
:1049080084F880010CF08AFD84F87F010CF086FDA4
:1049180084F8810127E10CF08BFDA4F882010CF0EA
:1049280087FDA4F884010CF079FD84F886010CF069
:104938007FFDA4F8880116E10CF070FD84F892015F
:104948000CF076FDA4F89C010CF072FDA4F8980117
:104958000CF06EFDA4F89A010CF060FDDAF8003056
:1049680084F893015B79082B40F2FD800CF060FD20
:10497800A4F89E010CF05CFDA4F8A001F3E00CF093
:104988004DFD84F8D8010CF049FD84F8D9010CF0EC
:104998004FFDA4F8DA01E6E092F805900323B9FB8D
:1049A800F3F9B9F1120F3FF677ACDFF8F0A14FF049
:1049B800000BCB4580F0D7800CF030FD8AF8A201BF
:1049C8000CF036FD40F2ED23984205DD40F6CA03AF
:1049D8009842A8BF184601E040F2EE20A0F2EE206F
:1049E800192390FBF3F00BF1010B8AF8A3010AF1EC
:1049F800020ADEE70CF012FD84F89401B3E00CF033
:104A08000DFD04EB090309F10109B9F1080F83F859
:104A18008A01F4D1A7E00CF001FDC4F80890607198
:104A28000CF010FDA3681843A0600CF0F7FC84F8A4
:104A380092010CF0FDFCA4F85C010CF0F9FCA4F860
:104A48005E010CF0F5FCA4F860010CF0F1FCA4F890
:104A580082010CF0EDFCA4F8840184E053794FF056
:104A6800070AB3FBFAF2C2EBC2029A1A12F0FF0F5E
:104A78007FF412ACB3FBFAFA0AF1FF3A5FFA8AFA4A
:104A8800BAF1FF0F6FD00CF0C9FC5FFA80FB4FFA48
:104A98008BF003F0F7F8814600283FF4FDAB80F86F
:104AA80000B00CF0C5FCA9F802000CF0B7FC89F8BE
:104AB80004000CF0B3FC89F805000CF0AFFC89F891
:104AC80007000CF0ABFC89F80600D5E7DFF8CC90BE
:104AD80009F1400A0CF0ACFCA9F8A8020CF09EFC05
:104AE80089F8AA020CF09AFC09F1040989F8A702CE
:104AF800D145EFD137E00CF091FC1F2881463FF6F5
:104B0800CBAB3B685B79082B7FF4C6AB0CF090FC11
:104B180009F18A0904EB890A00F03F00AAF80200AB
:104B28000CF086FCBAF80230800100F4FE501843FD
:104B3800AAF802000CF072FC000104F829000CF03D
:104B48006DFC14F8293000F00F00184304F8290010
:104B58000CF064FC8AF801000BF0C2FD03E00D4B79
:104B6800012283F8352000200CF0A4FCFFF7EDB9F2
:104B7800C8190020CE190020CC190020CA1900201D
:104B88005211002054110020641100205C110020F3
:104B9800FC0F002088100020D0190020D41100201C
:104BA8005B4B985903F044FB18B9322003F097FA8D
:104BB800F6E70BF013FC05F0FBFB564A564BDA60A0
:104BC800FFF7D1B90C2840D00A2847D1534D544893
:104BD8000CF0F4FC2846232111F0BFFF08B1401B5C
:104BE80020602368002B5CD14C48002130222360D0
:104BF80011F07DFF98F8003053BB4A4B1B689B06A9
:104C080014D5494B49491B688A6B9A1A002A0DDB4F
:104C1800474A1278042A09D903F5123303F5F873C1
:104C2800444A8B63D36883F01003D360424B9B687C
:104C3800002B69D0414805B0BDE8F04F18470AF08D
:104C480053FAFFF782B90C2804D13D480CF0B6FCA2
:104C58003C480DE07F2812D1FFF7E3B80D28B5D006
:104C68007F2809D12D4A013B002137482360D154C0
:104C78000CF0A4FCFFF7D5B82F2B3FF6D2A8A0F173
:104C88002002D2B25E2A3FF6CCA813B920283FF4FE
:104C9800C8A85A1C2260214AD0540CF087FCFFF7A0
:104CA800C0B85A1EA95C202901D113469AE71B4AAD
:104CB80000212360D154254B254DD3F800A0D5F809
:104CC80000B0DFF85890584611F055FF074659468E
:104CD8003A46484611F058FF1E4A28B919F80730D5
:104CE80053445B785B0703D010359542E7D306E061
:104CF800954204D2781CEB684844984702E016486D
:104D08000CF05CFC00236FE705B0BDE8F08F00BF36
:104D1800182800200400FA0500ED00E0E01A002041
:104D28003AC40108C4190020CC30002088100020A3
:104D3800CE190020000C014094270020C410002048
:104D480059B5010854B5010880B50108580000207C
:104D580070990108209B010864B501086B4B6C4AE7
:104D68002DE9F04F5E8914684FEA062AB4EB0A0A67
:104D78009C884FF000054FEA04481C894FF0000B4F
:104D8800A4FB0A6765EB0B0B04FB0B77F40944EAF9
:104D9800476418EB04065C884FF000094FEAE715F2
:104DA8004FEAC438DC8849EB050787B0CDE90467CA
:104DB800A4FB0A6704FB0B77340A44EA076418EB80
:104DC80004064FEA27259C894FF0000949EB05079F
:104DD800CDE90067AAFB046704FB0B77F40D44EAEE
:104DE800472414F5FA664FEAE75545F10007B6F58A
:104DF800FA6F77F10003CDE90267964666DADDE9D6
:104E08000489A4FB046704FB05F34FF0050C07EBCA
:104E18004307A6FB0C230CFB07335F104FEA32064F
:104E2800B8EB06084FEA920646EA837669EB07096B
:104E38009F10DDE90023921B63EB0703CDE90023F4
:104E4800DDE90267334A4FF0FF33964277EB0303FD
:104E5800CDE9048927DA40F6AC520023A4185D4155
:104E680004FB05F3A4FB04456FF0060205EB4305BC
:104E7800664202FB0566A4FB0223334418EB0206D4
:104E880049EB0307CDE904670B26A4FB062306FBC1
:104E98000533DDE900455B104FEA3202A41A65EBE1
:104EA8000305CDE90045DDE902450AFB0BF3AAFB42
:104EB8000AAB0BEB430B4FEADA7242EA4B02A41A35
:104EC8004FEAEB7365EB0305CDE90245DEF80440D4
:104ED800009B019DA4FB032304FB05334FEA5258B2
:104EE80048EAC3284FEA6359DDE90423B8EB020214
:104EF80069EB03039946D30B43EA494300B10360C6
:104F080009B1029B0B6007B0BDE8F08F4E0200208C
:104F1800C810002024FAFFFF2DE9F04FDFF858925F
:104F280085B00746D9F808000E460EF02BF88E4CCF
:104F3800804620880EF022F84FF05C510546404626
:104F48000EF074F84FF06451824628460EF06EF861
:104F5800014650460DF060FF4FF0625182464046D0
:104F68000EF064F84FF06A51804628460EF05EF85D
:104F7800014640460DF050FF0546B4F902000EF018
:104F880001F8014628460EF051F8514605465046AC
:104F98000EF04CF88046B4F904000DF0F3FF01461A
:104FA80040460EF043F8014628460DF037FF80468C
:104FB8000EF002FA6D490546A06140460EF0EAF887
:104FC800D9F80C308046284601930DF0DBFF4FF0EE
:104FD8007C510EF02BF866490DF01EFF0546E3895B
:104FE800B4F90A0002930DF0CDFF29460EF01EF821
:104FF80029460EF01BF84FF058510EF017F881466D
:10500800B4F90800B4F810B0B4F80CA00DF0BAFF69
:1050180029460EF00BF8014648460DF0FFFE4FF00A
:1050280058510EF003F84FF060510DF0FFFF4FF0AC
:105038007E510DF0F3FE8146E0880DF09FFF01469A
:1050480048460DF0F3FF002181460EF083F9002851
:105058007BD1294628460DF0E9FF03900FFA8BF023
:105068000DF090FF039B014618460DF0DFFF4FF04F
:1050780060510DF0DBFF8346BDF908000DF082FF9B
:10508800014628460DF0D2FF01460DF0C7FE014645
:1050980058460DF0C3FE4FF07A510DF0C7FF834616
:1050A80001980DF06FFF01464FF093400DF0B4FEEC
:1050B80005460FFA8AF00DF065FF4FF08F410DF0AD
:1050C800B5FF014658460DF0A9FE4FF066510DF0A8
:1050D800ADFF014628460DF09FFE26490DF0A6FFBC
:1050E80049460EF057F80546B4F916000DF04AFF88
:1050F80029460DF09BFF29460DF098FF4FF04051CF
:105108000DF094FF8146B4F914000DF03BFF014601
:1051180028460DF08BFF4FF060510DF087FF0146D8
:1051280048460DF07BFE8146B4F912000DF02AFFC7
:10513800014648460DF072FE4FF076510DF076FFAD
:10514800014628460DF06AFE00E0002017B10EF077
:1051580033F938602EB140460EF02EF964235843D7
:10516800306005B0BDE8F08F880200200000A0453F
:1051780000007A470050C345C810002070477047A8
:105188002DE9F041324C334D62892B8AB4F9048001
:105198009A1A2389B4F902E05A43B4F91230D613A3
:1051A800B4F91420DB02324493FBF2F232440A26AB
:1051B800E2615643A2F57A6202FB02F3B4F90EC02B
:1051C80002FB0EFE02FB08F2B4F90C801B130CFB69
:1051D80003FC03FB08F31B1403EB62320232E3887F
:1051E800921002F5004253434CF25032B4F9207049
:1051F8004FEAEE2EB4F900400EEBEC2C0CEB8404D5
:10520800BC406D690234A5EBA4043A4162434FEAFD
:10521800D3384EBFB2FBF8F35400B4FBF8F340F6B2
:10522800DE3448BF5B001A12524362430A4C083608
:105238005C43241404EB224202F6CF62361103EBDE
:10524800221300B1036001B10E60BDE8F08100BF18
:1052580060020020C810002043E3FFFF024B4FF418
:1052680080521A80704700BF1A0000207047064A13
:1052780008B5138801339BB21380044B187806F0E5
:10528800E9FA002008BD00BFE61000206C1D0020D0
:105298000F4B13B51A7E1C46C2B90E4B1B68ABB137
:1052A8001A681AB10C49886902438A619A88986811
:1052B800ADF8042002228DF8072004220DEB02012C
:1052C8008DF8062007F0BEFD0123237602B010BD3D
:1052D800C8100020440200200010024008B5FFF763
:1052E800D7FF074B1B7813B1012B03D008BD4FF430
:1052F800006201E04FF48052024B1A8008BD00BFE3
:105308004C0200201A000020F8B50F461646074C3C
:105318004FF48055656140F080000CF00DFF384671
:1053280031460CF02FFF2561F8BD00BF000C01408D
:1053380013B501220DF1070104463820FFF7E4FFF9
:10534800052002F0C1FE9DF8073003B10123237048
:1053580002B010BD13B50446694643200622FFF784
:10536800D3FF9DF800209DF80130012043EA022375
:1053780023809DF802209DF8033043EA02236380CE
:105388009DF804209DF8053043EA0223A38002B06B
:1053980010BD13B5044669463B200622FFF7B4FF4B
:1053A8009DF800209DF80130012043EA0223238064
:1053B8009DF802209DF8033043EA022363809DF89C
:1053C80004209DF8053043EA0223A38002B010BDF3
:1053D80070B50E46054C4FF4805565610CF0ACFE77
:1053E80030460CF0A9FE256170BD00BF000C0140DD
:1053F80008B580216B20FFF7EBFF642002F06FFEF9
:1054080000216B20FFF7E4FF642002F068FE6B20A8
:105418000121FFF7DDFF1B201821FFF7D9FF1C2012
:105428001021FFF7D5FF054B1A201978FFF7D0FF99
:10543800BDE8084019200021CAE700BF010000208C
:1054480010B54000204CC0B220702048204C01709C
:10545800204800210170012020701F4C23601F4C40
:1054680023601F4B1A701F4A1F4B107019701F4979
:10547800086811461A4630B383889C0515D40388FA
:10548800DB050DD447F230530488A40502D5013B4F
:10549800FAD112E08BB103889BB243F48073038086
:1054A80083889BB243F44073838047F23053087873
:1054B80010B1013BFBD100E013B9BDE81040D6E6BE
:1054C800107880F0010010BD721D0020701D0020B2
:1054D8006E1D0020781D0020741D00207C1D0020FA
:1054E800711D0020801D0020811D0020681D0020E6
:1054F80007B5002101AB03227720FFF7A1FF9DF834
:1055080005309DF804001B0243EA00439DF806009D
:10551800184303B05DF804FB08B5FFF7E9FF014B3A
:10552800586008BDC810002008B5FFF7E1FF014B1F
:10553800186008BDC810002007B5F7216B46062281
:105548007620FFF77DFF9DF800309DF801101B03C2
:1055580043EA01139DF80210094A43EA1113D36084
:105568009DF803309DF804101B0343EA01139DF8CE
:10557800051043EA1113936003B05DF804FB00BF04
:10558800C810002007B5F62101AB03227720FFF7EA
:1055980057FF9DF805309DF804201B0243EA02439B
:1055A8009DF806201343054AB2F92020C2F10802EB
:1055B800D340034A536103B05DF804FB6002002046
:1055C800C810002007B5F62101AB02227720FFF7AB
:1055D80037FF9DF804209DF8053043EA0223024A6C
:1055E800138203B05DF804FBC810002013B5012234
:1055F8000DF107033A2104466820FFF721FF052033
:1056080002F062FD9DF8073003B10123237002B058
:1056180010BD13B506220446432168206B46FFF7E8
:105628000FFFA8B19DF800209DF80130012043EA42
:10563800022323809DF802209DF8033043EA0223C9
:1056480063809DF804209DF8053043EA0223A38077
:1056580002B010BD13B5062204463B2168206B46F4
:10566800FFF7EEFEA8B19DF800209DF8013001205B
:1056780043EA022323809DF802209DF8033043EA81
:10568800022363809DF804209DF8053043EA022335
:10569800A38002B010BD13B50622044601211C20C8
:1056A8006B46FFF7CDFE08B39DF801309DF800204A
:1056B800042143EA022242F38D0292FBF1F29DF8A3
:1056C800023022809DF8032042EA032242F38D0231
:1056D80092FBF1F29DF8043062809DF8052042EAC1
:1056E800032343F38D0393FBF1F3A38002B010BDB2
:1056F80013B506220446A82168206B46FFF7A0FED2
:10570800A0B19DF800209DF8013043EA02232380D0
:105718009DF802209DF8033043EA022363809DF838
:1057280004209DF8053043EA0223A38002B010BD8F
:1057380013B506220446022118206B46FFF780FEA7
:10574800B8B19DF800309DF801209B0803EB0223B7
:1057580023809DF802309DF803209B0803EB022369
:1057680063809DF804309DF805209B0803EB022315
:10577800A38002B010BD314B2DE9F3411B780546DB
:10578800002B3BD0002426462746A0460134532050
:10579800322108226B46E4B2FFF752FE08B9002016
:1057A80049E09DF801209DF80030202C03EB0223EE
:1057B8001BB29DF8032098449DF8023003EB0223A6
:1057C8001BB21F449DF805209DF8043003EB02230B
:1057D8001BB21E449DF8073003F07F0301D0002B55
:1057E800D4D198FBF4F897FBF4F796FBF4F6144B36
:1057F800A5F800806F80AE805C761CE053203221D3
:1058080006226B46FFF71CFE0028C8D09DF8012031
:105818009DF8003003EB02232B809DF803209DF8B0
:10582800023003EB02236B809DF805209DF80430BD
:1058380003EB0223AB8002B0BDE8F0814B020020ED
:10584800C810002013B502AB03F8012D4000214A0F
:10585800C0B21070204A00201170204901220A703D
:105868001F4908701F490B601F490B601F4B2049D7
:105878001A700A701F4B204A187010681A4630B305
:1058880083889C0515D40388DB050DD447F2305373
:105898000488A40502D5013BFAD112E08BB1038834
:1058A8009BB243F48073038083889BB243F44073B4
:1058B800838047F23053087810B1013BFBD100E0F8
:1058C80013B9FFF7D4FC02E0107880F0010002B0B1
:1058D80010BD00BF721D0020701D0020781D002023
:1058E8006E1D00207C1D0020741D0020711D0020ED
:1058F800801D0020811D0020681D00207720482180
:1059080001229FE77720582101229BE77620F42186
:10591800312297E7044B772093F82020F421920155
:10592800343202F0FC028DE7600200207720F42177
:105938002E2287E708B5FFF7ABFC6B218022682091
:10594800FFF780FF642002F0CAFB6B210322682066
:10595800FFF778FF0F2002F0C2FB0F4B19211A78CE
:105968006820FFF76FFF0F2002F0B9FB0B4B1A21DD
:105978001A786820FFF766FF1B2118226820FFF7B6
:1059880061FF1C2110226820FFF75CFFBDE808407A
:1059980068203721002255E74A0200200000002035
:1059A80008B52A2100221C20FFF74CFF0E210222F5
:1059B8001C20FFF747FF0F2103221C20FFF742FF9F
:1059C8002B2112221C20FFF73DFF2C2102221C2034
:1059D800FFF738FF2D2101221C20FFF733FF2E216E
:1059E80000221C20FFF72EFF05221C202A21FFF78A
:1059F80029FF024B4FF480721A8008BD1A0000205C
:105A080008B5642002F06BFB68202321F022FFF721
:105A180019FF10B9022002F06CFB052002F05FFBB1
:105A2800044B68201A78202142F00F02BDE8084094
:105A380008E700BF4802002008B50F2108221820F7
:105A4800FFF700FF0E2218201021FFF7FBFE024B84
:105A58004FF480521A8008BD1A00002008B5134B75
:105A680053201B782D2108227BB1FFF7EBFE312153
:105A78000A225320FFF7E6FE2C210C225320FFF7C1
:105A8800E1FE53203821902209E0FFF7DBFE3121A7
:105A98000A225320FFF7D6FE53202C210A22FFF7B3
:105AA800D1FE40F20912024B1A8008BD4B020020B9
:105AB8001A00002005F0C6BF06F0EAB805F0C2BF1C
:105AC80006F0E6B873B51D4CA37E53BB1C4A1D4DAA
:105AD80093694FF4805643F00803936110238DF8BF
:105AE80006302846032301A98DF80730ADF8046075
:105AF80007F0A8F9144A2E61138823F040031B0409
:105B08001B0C1380138823F038031B041B0C43F071
:105B18000803138013889BB243F0400313800123CA
:105B2800A376752001A90122FFF7EEFB9DF804007A
:105B3800A0F170035842584102B070BDC81000204F
:105B480000100240000C014000380040F8B50F4634
:105B58001646074C4FF48055656140F080000CF004
:105B6800EBFA384631460CF00DFB2561F8BD00BF55
:105B7800000C014013B501220DF1070104463A203B
:105B8800FFF7E4FF052002F09FFA9DF8073003B104
:105B98000123237002B010BD184A13B513880446B8
:105BA80023F040031B041B0C13801388432023F0AD
:105BB80038031B041B0C1380138869469BB243F0FF
:105BC800400313800622FFF7C1FF9DF800209DF8CF
:105BD8000130012043EA022323809DF802209DF82A
:105BE800033043EA022363809DF804209DF80530C2
:105BF80043EA0223A38002B010BD00BF0038004072
:105C080070B50E46054C4FF4805565610CF094FA5A
:105C180030460CF091FA256170BD00BF000C0140C0
:105C280007B5232002F05BFA6820752101220DF1E7
:105C38000703FFF705FC28B19DF80700A0F16803EA
:105C48005842584103B05DF804FB00BF4D282DE9C8
:105C5800F047044600F0548600F2B980302800F07E
:105C6800B48651D8222800F0908423D8032800F065
:105C7800058214D8012800F0F581022840F0F48646
:105C880004200BF017FC43200BF0E5FB4C200BF035
:105C9800E2FB46200BF0DFFB4C2000F056BE042848
:105CA80000F0F581052840F0DF861A200BF002FC91
:105CB8000024FCE1282800F0E28515D8242800F00B
:105CC800C985262840F0D086DA4C06200BF0F2FB76
:105CD800B4F85C010BF0F1FBB4F85E010BF0EDFBDE
:105CE800B4F8600100F0B3BD2C2800F0DB852E2845
:105CF80000F055862A2840F0B78601200BF0DAFB21
:105D0800CC4B587900F021BE3D2800F0F8821ED80F
:105D1800362800F02B860BD8322800F0108634285D
:105D280040F0A28648200BF0C5FB002500F04FBCD0
:105D38003A2800F0B9823B2800F02084382840F047
:105D4800938604200BF0B6FBBA4C00F089BD4528B9
:105D580000F0768627D8402800F0FA85422840F0DF
:105D68008386B44C10200BF0A5FB60790BF073FB15
:105D7800A0680BF0ABFB94F892010BF06CFBB4F845
:105D88005C010BF09AFBB4F85E010BF096FBB4F8DB
:105D980060010BF092FBB4F882010BF08EFBB4F8B3
:105DA800840100F054BD492800F0B4824B2800F06B
:105DB8009885462840F058860D200BF07BFB002084
:105DC8000BF049FB00200BF081FB00F044BE70286B
:105DD80000F0F08200F2E180692800F0458200F2CC
:105DE800B280662800F0A08100F2A280642800F04A
:105DF8007781652840F038868F4C0B200BF05AFBD2
:105E080020880BF05AFB608880B20BF056FB8B4B56
:105E18001B68C3F3C000C3F38002800040EA42005D
:105E2800C3F340021043C3F3401240EAC20003F038
:105E3800100318430BF041FB814B1A88636802F08A
:105E4800080103F4475949EA010903F4804149EA82
:105E5800010903F4004149EA010903F4803149EAE0
:105E6800010903F4003149EA010903F4802149EAF0
:105E7800010903F4002149EA010903F4801149EA00
:105E8800010903F0007349EA0303DFF8D49112F023
:105E9800010F99F8009018BF4FF00208C9F3800964
:105EA80008BF4FF0000843EA090312F0020F43EA63
:105EB800080314BF4FF0040C4FF0000C12F0040F4D
:105EC80043EA0C0C14BF4FF0100E4FF0000E12F006
:105ED800400F14BF202700274CEA0E0E12F0100FB7
:105EE80014BF4FF4007600264EEA070712F0200F81
:105EF80014BF4FF4806500253E4312F4807F14BF21
:105F08004FF400600020354312F4007F14BF4FF4B3
:105F180000110021284312F4806F41EA000114BFE8
:105F28004FF08063002300201943247A0346E7E0FA
:105F3800672800F02181682840F0968510200BF032
:105F4800B9FA002488E16C2800F0A18117D86A28E2
:105F580000F003846B2840F0878505200BF0AAFA2F
:105F6800384B18880BF0A9FA374B18880BF0A5FAAC
:105F7800314B93F86E0000F0010000F0E6BC6E288B
:105F88002D4D00F0978100F2CB8106200BF092FA9C
:105F9800E86D0BF09BFA2D4B84E1782800F0F9802E
:105FA80018D8742800F034830AD8722800F0958332
:105FB800732840F0598508200BF07CFA0124C5E3CA
:105FC800762800F0EA8300F25C832F200BF072FA47
:105FD8001F4CCBE2A42800F0068414D87B2800F0DC
:105FE8006B82A02840F040850C200BF063FA194B17
:105FF80018680BF06BFA184B18680BF067FA174B18
:10600800186800F02CBDF12800F0FF80FE2800F091
:106018001184F02840F02885074C04200BF04AFA38
:10602800236CB3F85A000BF048FA236CB3F8580005
:1060380000F00DBCD4110020E4100020C419002089
:106048008C1A0020421A0020441A0020BC1100209B
:1060580003930108E8F7FF1FECF7FF1FF0F7FF1F96
:10606800E730002003200BF025FA00200BF0F3F9AD
:1060780020460BF0F0F90D2000F067BC0BF01AFA7F
:1060880001200BF0E8F90A200BF0E5F9A9E3062056
:106098000BF010FA45200BF0DEF955200BF0DBF978
:1060A80046200BF0D8F931200BF0D5F9CEE3B04BF0
:1060B800185D01340BF0CFF90B2CF8D10024AD4B4F
:1060C800185D01340BF0C7F9082CF8D10024AA4B4D
:1060D800185D01340BF0BFF9072CF8D100F0C1BCF2
:1060E80007200BF0E7F9E7200BF0B5F9A34B587937
:1060F8000BF0B1F900200BF0AEF9042000F0AFBCB2
:10610800A3420AD29E4A9D5C012202FA05F50D427D
:106118001CBF9A4010430133F2E70BF0D7F9974BB5
:1061280093F8B00700F011BC12200BF0C3F9954B9F
:1061380000241B88B3F5806F8CBF08250125924B7E
:1061480033F91400013490FBF5F080B20BF0B5F987
:10615800032CF4D18D4CA08C0BF0AFF9E08C0BF034
:10616800ACF9208D0BF0A9F9608D0BF0A6F9A08D84
:106178000BF0A3F9E08D6AE310200BF09BF90024E3
:10618800834B185D01340BF066F9102CF8D100F040
:1061980068BC70200BF08EF900260E2474437B4DEA
:1061A80001362B6C2344B3F819010BF086F92B6CDC
:1061B8002344B3F81B010BF080F92B6C2344B3F88C
:1061C8001D010BF07AF92B6C234493F81F010BF097
:1061D80042F92B6C234493F820010BF03CF92B6C0B
:1061E800234493F821010BF036F92B6C234493F8E0
:1061F80022010BF030F92B6C1C44D4F823010BF06E
:1062080065F9082EC9D100F02CBC70200BF052F9AA
:106218005A4C04F1700594F8D4000BF01CF994F86A
:10622800D5000BF018F994F8D6000BF014F994F88F
:10623800D7000BF010F994F8D8000BF00CF994F88B
:10624800D9000BF008F9073494F8D3000BF003F9E0
:10625800AC42E0D100F005BC4E4B185D01340BF0A8
:10626800FAF8102CF8D1FCE34B4D002428784000B4
:1062780000F0FE000BF01EF92B789C4280F0F183B1
:10628800464B33F814000BF018F90134F4E7444C8A
:1062980006200BF00FF920880BF00FF960880BF03F
:1062A8000CF9404B1888D2E204200BF003F9374B65
:1062B800186ED4E307200BF0FDF83B4B1888FF2835
:1062C800A8BFFF20C0B20BF0C6F8384B186880F39F
:1062D800100080B20BF0F1F8B5F864000BF0EDF89F
:1062E800264B93F88721324B186822B10A2358436A
:1062F80080F3100001E000F30F0080B2A7E21F4C0A
:1063080002200BF0D7F894F8E2010BF0A4F894F807
:10631800E1011AE302200BF0CDF8184B988996E2B8
:106328000B200BF0C7F8AB6E002618780BF093F82B
:10633800AB6E58780BF08FF8AB6E144C3344187969
:1063480001360BF088F8032EF6D1A36ED8790BF03E
:1063580082F8A36E98780BF07EF8A36ED8780BF0CD
:106368007AF8A36E58890BF0A8F8A36E187AECE2B5
:10637800BCB50108C8B50108D1B50108D411002081
:10638800ED1000201A000020B6110020E4100020B3
:106398001411002028110020B4280020382D0020D6
:1063A800F42C0020C4110020B4190020C0190020CA
:1063B800BC190020C04C1E200BF07CF8236C002573
:1063C8001B78022B65D1236C05F1080253F82200D3
:1063D800BA490CF02BFE10F097FD80F30800C0B20C
:1063E8000BF039F8236CB64903EB8503D86A0CF037
:1063F8001DFE10F089FD80F30800C0B20BF02BF8E9
:10640800236C05F10E0253F82200AE490CF00EFE83
:1064180010F07AFD80F30800C0B201350BF01BF8CC
:10642800032DD0D1072D236C21D1586CA3490CF032
:10643800FDFD10F069FD80F30800C0B20BF00BF809
:10644800236C9E49986C0CF0F1FD10F05DFD80F313
:106458000800C0B20AF0FFFF236C93F84C000CF060
:106468008DFD10F051FD80F30800C0B20BE02B4405
:1064780058780AF0F0FF236C2B44D87A0AF0EBFF27
:10648800236C2B44587D01350AF0E5FF0A2DC9D14C
:10649800E7E2236C2B4458780AF0DDFF236C2B4489
:1064A800D87A0AF0D8FF236C2B44587D01350AF0BE
:1064B800D2FF0A2DEDD1D4E23C200AF0FBFF0024E4
:1064C8007D4D04F108022B6C7E4953F822000CF034
:1064D800ADFD10F019FD80B20AF0EFFF2B6C794981
:1064E80003EB8403D86A0CF0A1FD10F00DFD80B217
:1064F8000AF0E3FF2B6C04F10E0253F822007149F5
:106508000CF094FD10F000FD013480B20AF0D5FFC4
:10651800032CD5D1072C2B6C16D1586C69490CF07B
:1065280085FD10F0F1FC80B20AF0C7FF2B6C6549BD
:10653800986C0CF07BFD10F0E7FC80B20AF0BDFF10
:106548002B6C93F84C000BE0234458780AF0B5FF05
:106558002B6C2344D87A0AF0B0FF2B6C2344587D67
:1065680001340AF0AAFF0A2CD4D17AE214F8010FF8
:10657800002800F076820AF06EFFF7E701200AF0A3
:1065880099FF4D4B1B6C1878DFE150200AF092FF01
:106598000025494B0C211C6C4B4B04EB850494F8EB
:1065A8007920013501FB023393F838000AF053FFD4
:1065B80094F87A000AF04FFF94F87B000AF04BFF3A
:1065C80094F87C000AF047FF142DE2D149E23A4BD7
:1065D8001C6C062303FB054494F8CE000AF03BFF2D
:1065E80094F8C9000AF037FF94F8CA000AF033FF9C
:1065F80094F8CB000AF02FFF94F8CC000AF02BFF98
:10660800013594F8CD000AF026FF0C2DDFD128E2E1
:106618004FF0000801260027274B1A7A974227DAFD
:106628000933FA5C00240C236343274D05F130013C
:10663800595C914207D12B44586B10F09CFA824662
:106648002EB9B14605E001341C2CECD10EE0804493
:106658000CE0D1450ADA0C2303FB04535B6B13F8F7
:1066680009000AF0F8FE09F10109F2E70137D3E75A
:10667800002E00F0F6815FFA88F00AF01BFF002672
:10668800C9E70D4D0024287A0AF014FF2B7A9C42A2
:1066980080F0E7810D4B0021E65C0C2202FB01F340
:1066A800094800F13007DA5DB24211D1034493F88A
:1066B80038000AF0D0FE0EE0E4100020000020416F
:1066C8000000C84200007A4404930108ED1000203D
:1066D80001311C29E1D10134D8E7CE4C16200AF04B
:1066E800E9FEB4F898010AF0E8FEB4F844010AF0AB
:1066F800E4FEB4F846010AF0E0FEB4F848010AF0F6
:10670800DCFEB4F8DA010AF0D8FE94F8EF010AF0DA
:10671800A2FE00200AF09FFE94F8F0010AF09BFE0A
:1067280094F887010AF097FE94F894010AF093FE12
:1067380000200AF090FEB84B0A201B6CB3F95630C3
:1067480093FBF0F080B20AF0B8FE89E0E0B20134C1
:106758000AF081FE092CF9D183E110200AF0AAFE83
:10676800AE4BAF4C187800F002000AF074FEAD4B47
:1067780018780AF070FE20680AF0A8FE60680AF02F
:10678800A5FEA94B18880AF098FEA84B18880AF0AD
:1067980094FEA14BB3F86C0059E00AF03FFE07469F
:1067A80012200AF087FE9C4C17B9266F656F05E02A
:1067B800102F19BF00252E46A66FE56F38460AF040
:1067C8004AFE30460AF082FE28460AF07FFED4F8D8
:1067D80080000AF07BFE00200AF06FFE00200AF01D
:1067E8006CFE0020B1E08C4D002495F884002E4604
:1067F80080000130C0B20AF05DFE95F884000AF00E
:106808002AFE96F884309C4280F02B81884D285DC2
:106818000AF021FE05F11003185D0AF01CFE05F1CF
:106828002003185D30350AF016FE285D0AF013FEC5
:106838000134E6E708200AF03DFE00200AF03DFE9C
:1068480000200AF03AFE00200AF037FE00200AF085
:1068580034FE06E104200AF02DFE6E4B9868FEE037
:1068680094F87C010AF0F7FD94F880010AF0F3FD32
:1068780094F87F010AF0EFFD94F8810165E0654C1A
:1068880007200AF017FEB4F882010AF016FEB4F8E1
:1068980084010AF012FE94F886010AF0DCFDB4F8CF
:1068A8008801D4E75B4C0C200AF004FE94F89201AE
:1068B8000AF0D1FDB4F89C010AF0FFFDB4F8980184
:1068C8000AF0FBFDB4F89A010AF0F7FD94F8930179
:1068D8000AF0C1FDB4F89E010AF0EFFDB4F8A0017A
:1068E800B5E74C4C04200AF0E5FD94F8D8010AF00D
:1068F800B2FD94F8D9010AF0AEFDB4F8DA01A6E7C2
:106908004C4C4D4D2078002600EB4000C0B20AF0F8
:10691800D1FD237802359E4280F0A38015F8020C41
:106928000AF099FD15F8010C013600EB800000EB28
:10693800800000F2EE2080B20AF0BFFDE9E70120F6
:106948000AF0B8FD334B93F894010AF084FD88E00F
:1069580008200AF0AFFD00242E4B234493F88A0147
:1069680001340AF078FD082CF6D17AE02A4B294C3C
:1069780093F8C50004F12005C0EBC000C0B20AF0CE
:1069880099FD94F8F60100232C4AD25C90426ED00F
:106998000C33302BF8D10834AC42F2D161E04020FE
:1069A8000AF088FD1B4C04F14005B4F8A8020AF06F
:1069B80084FD94F8AA020AF04EFD043494F8A70264
:1069C8000AF049FDAC42F0D14BE0E0200AF072FD3C
:1069D800104C04F18005B4F82A02043400F03F009A
:1069E8000AF06BFDB4F82602C0F386100AF065FDC4
:1069F80094F8240200090AF02EFD94F8240200F00D
:106A08000F000AF028FD94F825020AF024FDAC4294
:106A1800E1D126E0D4110020E4100020C81900209C
:106A2800D0190020CE190020CC190020CA19002046
:106A380069110020B428002076130020C028002007
:106A480013200AF037FD0024144B185D01340AF0B6
:106A580002FD0B2CF8D100200AF038FD00200AF0C6
:106A680035FD0120BDE8F0870020BDE8F0870AF079
:106A7800F2FCB4F8F8010AF020FD94F8FA010AF0E3
:106A8800EAFC94F8FB010AF0E6FC94F8FD010AF030
:106A9800E2FC94F8FC010AF0DEFC7CE7BCB50108D6
:106AA8002DE9FF47CB4C07462378CB4E002B00F04F
:106AB800E78132686368D31A7C2B40F2E181237A3C
:106AC8006260013323724FF0000808F12400C14DC1
:106AD800C0B206F029FD05F10A0333F918000CF0DD
:106AE80051FABE4B814618880CF04CFA01464846CC
:106AF8000CF050FBBA490CF099FA0CF05DFC08F167
:106B0800010800B206F0FEFCB8F1030FDDD1302019
:106B180006F00AFDB5F9100006F0F4FC06F0FCFCDE
:106B28002B7A9A072CD141F288336A689A4218D98D
:106B3800102006F0F9FC68694FF0640890FBF8F043
:106B480000B206F0DFFC212006F0EEFC686990FB3D
:106B5800F8F308FB13000028B8BF404200B206F063
:106B6800D1FC142006F0E0FCB4F9180006F0CAFCC9
:106B78001C2006F0D9FC002006F0C4FC06F0CCFC72
:106B8800237ADFF850825B0740F05781022006F035
:106B9800CBFCD8F81C006423323090FBF3F000B231
:106BA80006F0B0FCB8F926504FF0050A95FBFAF547
:106BB800032006F0B9FC8B4BADB21B78DFF8389296
:106BC80013F0040F0DD008F5D970394601F0D1F94A
:106BD80028B9D9F8003013F0100F18BF002528B2D3
:106BE80005E0D8F804389889B0FBFAF000B206F04E
:106BF80089FCD9F800309F076ED5DFF80092B4F809
:106C0800082899F800304FF0640808FB02325B004E
:106C1800B2FBF3F3B4F80A7806203F01BFB247EAA3
:106C28000327BFB2C3F303231F4306F07DFC38B22A
:106C380006F068FCB4F80A3899F8001001339BB2E2
:106C480093FBF1F201FB1233A4F80A38D4F80C389C
:106C5800604D9B7B012B05D1392006F065FCB5F909
:106C680008081AE0B5F808586E235D43152795FB08
:106C7800F7F53A20AFB206F057FCB7FBF8F528B2A3
:106C880008FB157506F03EFC3B2006F04DFCA8B24B
:106C9800451D0A2095FBF0F000B206F033FC2820D1
:106CA80006F042FCD4F810380A2093FBF0F000B24A
:106CB80006F028FC042006F037FCD4F804389B8939
:106CC80013B108F083FD04E0424BD3F8140880F3B5
:106CD800100000B206F016FCD4F818383D4F9D0697
:106CE80040F1A08097F81C3898071DD5112006F0B0
:106CF8001BFCB7F81E084FF4F36568433A4B90FB4A
:106D0800F3F000B206F0FEFB192006F00DFCB7F810
:106D18001E084543642095FBF0F595FBF0F300FB56
:106D2800135000B206F0EEFB94F81C38B4F8205863
:106D380013F0020F08BF0025012006F0F5FB28B26A
:106D480006F0E0FB092006F0EFFB002006F0DAFB76
:106D5800264B94F822581A88B2F5967F0AD91D4B0B
:106D68001B7A03F00F03072B04D842F20F759542E4
:106D780028BF1546052006F0D7FBD4F80C385B7BF6
:106D88000BB928B216E0A5F120000CF0FBF8184961
:106D98000CF000FA002105460CF0E6FA10B94FF0A5
:106DA8007C5101E04FF03F4128460CF037F80CF0D9
:106DB80003FB00B206F0A6FB94F81C28054B9107CC
:106DC80003D493F82328012A1AD1012384F82338FD
:106DD80008482EE0AC110020202D00201A000020C9
:106DE80000007A44E7300020A08601004600002019
:106DF8006666E63FD0190020FC2C002044000020E5
:106E0800D3F80C58C04968680CF010F90CF0D4FAA3
:106E1800BD490290A8680CF009F90CF0CDFA03906E
:106E280002A806E0B94A02AB92E8030083E803002F
:106E3800184606F089FB06F06FFB237A282B1FD132
:106E4800B34B00221A7233684FF47A70B3FBF0F830
:106E58003C27172006F068FBB8FBF7F5B5FBF7F001
:106E680007FB1050000200B206F04CFB182006F099
:106E78005BFB07FB158000B206F044FB06F04CFBF9
:106E880094F82C38A24D002B00F0618101F000F934
:106E9800D5F830389F4AC31A9342074640F2C78054
:106EA800002385F8363885F83838B5F80838DAB266
:106EB8001B0A85F8522885F8533885F8482885F83C
:106EC8004938D5F8602833689A1AD5F86438D97BD8
:106ED8004FF47A734B439A420ED38F4B1B68C5F815
:106EE800603895F86838013B012B9FBF102385F85F
:106EF8003638022385F83838D4F810280A20D4F810
:106F0800143892FBF0F293FBF0F384F85028121235
:106F180084F8512884F8543894F81C281B1284F8F3
:106F2800553894F822389207794984F8833803D47D
:106F38002D2381F8843878E0D4F824987748DFF84E
:106F4800E8C199FBF0FA0CFB0A924FF0060E042BED
:106F58000EFB02F28CBF3323322381F88438704B46
:106F6800D4F8286892FBF3F196FBF0F003FB1122AA
:106F7800642592FBF5F20CFB006C0EFB0CFE84F80A
:106F88007528121284F876289EFBF3F203FB12E3AD
:106F980093FBF5F30AEB8A0A4FFA81F80AEB8A0A9F
:106FA80008EB8A0189B284F8731800EB8000090A9B
:106FB80084F8741800EB800051B201EB800292B2A1
:106FC80084F87828120A84F8792884F87A38B4F88A
:106FD8001E281B1284F87B382423534393FBF5F5B2
:106FE800B4F896380A2284F87C381B0A84F87D386D
:106FF800B4F820384FEAD979B3FBF2F303F5FA7302
:107008009BB284F87E381B0A84F87F38B4F8983825
:10701800F60F84F87058C5F3072584F8729884F839
:10702800776884F8715884F88538C4F8307894F80B
:107038009A88374DB8F1000F0DD1D5F8A00809F09E
:107048004BF8012807D90228364E00F05E8202F07C
:1070580041FD0123B370D4F8A4282D4D002A76D021
:1070680095F89A683EB140F6B731D5F8AC38FB1AB6
:107078008B4219D86BE00123D5F8A00885F89A3817
:1070880000F0ECFDD5F8B038082193F90000022390
:107098008DE8480032464FF4964301F080F885F8B1
:1070A800B468C5F8A00850E095F8A868CEB9D5F836
:1070B800A008C5F8A46885F89A6800F0CFFDD5F84F
:1070C800B038082193F9000001238DE848003246C2
:1070D8004FF4964301F063F8C5F8A00802F0FAFCF3
:1070E80033E0013EF6B285F8A86895F8B41895F82B
:1070F800B538DEB94A1C013385F8B42885F8B538A7
:10710800D5F8A0081FE000BF8096184B909401089E
:10711800AC1100203F0D0300202D00208096980020
:1071280040420F001A000020806967FF12F8016BC7
:1071380001337018314685F8B408D5F8A008C5F8A9
:10714800A42885F8B53808F0CAFFC4F8AC7894F8D4
:10715800B638A14DF3B1D5F8B838DBB1D5F8BC389D
:10716800C3B1C5F8C0381B689C4AC5F8C438D5F8FF
:10717800C8381344187AFEF769FDD5F8C0389879ED
:107188000AF069F9D5F8C8380133092B88BF0023FC
:10719800C5F8C838924D94F8CC282E688E4B002A32
:1071A80000F0EE81D3F8D028002A00F0E98193F8A6
:1071B800D438013B012B00F2E381D4F8D008864F84
:1071C80008F08AFFE0B1D7F8D00808F082FF97F8F6
:1071D800D53880467E2BD5F800900ED102231B2887
:1071E80087F8D43809D1D7F8D00808F075FF20B946
:1071F8000123C7F8D89887F8DC3884F8D588DCE705
:10720800D7F8D8282B689B1A41F6583293421ED9D2
:10721800032387F8D438B3E1724A32F8130010B95F
:1072280003464FF403600133B0F5C06FDBB279D089
:107238001ED9B0F5006F7FD032D9B0F5036F3FD1BA
:1072480084F8DD38D4F81838634F99063FD494F899
:10725800DC1894F8DD38002900F054812A68921B64
:10726800012AD9D984F8DD38002384F8DC3887E18D
:10727800B0F5007F43D007D8B0F5807F49D0B0F58E
:10728800887F00F08B80E6E7B0F5806F00F0AE8075
:10729800B0F5826F00F0F380B0F5047FDBD123E016
:1072A800B0F5E26F00F08B80B0F5E46F00F08C80F1
:1072B800B0F5E06FCFD184F8DD38B4F90A1087E073
:1072C800B0F5046F74D0B0F5026FC4D103E197F83C
:1072D8001C389A07BBD5B7F81E1824234B436421E2
:1072E800123393FBF1F107E184F8DD383E4B3A4F56
:1072F8001B689B07ABD5B7F808380A21FBE084F870
:10730800DD38394B344F1B681905A0D5D7F810184C
:10731800F2E084F8DD38D4F818382F4F5A0796D59C
:107328007969E9E084F8DD382F4B2B4F1B681B0582
:107338008DD5D7F81418DFE0D4F81818264A8F0628
:1073480084F8DD3883D592F81C1888077FF57FAF5D
:10735800D90711D5D2F82838192283EAE371A1EBAD
:10736800E37101EB5101B1FBF2F1002BACBF41F02D
:10737800004141F040410EE0D2F82438192283EA56
:10738800E371A1EBE37101EB5101B1FBF2F1002BC9
:10739800B8BF41F080414FF400608BE084F8DD38DD
:1073A800D4F818380C4F5B077FF551AF3969A3E063
:1073B80084F8DD38B4F91830642159437AE084F848
:1073C800DD38B4F90C1003E0B4F90E1084F8DD3898
:1073D8002C2391FBF3F16DE0AC110020909401088F
:1073E800202D0020BEB60108FC2C002084F8DD38D2
:1073F80094F8DE38644A0133DBB2032B88BF0123DB
:1074080082F8DE3842F2107394F8DE1859435F4B65
:107418001B78D80748BF01319A0748BF02315F0778
:10742800B4F8E03848BF0431D80748BF0A319A0792
:1074380048BF14311F0648BF2831D80548BF283136
:107448005A0748BF64311F0748BFC831980548BF6D
:1074580001F5C8719A0648BF01F57A71DF0648BF81
:1074680001F5FA61580648BF01F57A614FF480606A
:1074780002F0FCFA444B002283F8DC28E7E6D4F853
:107488001818DFF8048111F0200784F8DD3817D0C8
:1074980098F81C2812F0020F14BF4FF47A710021DB
:1074A80012F0010F14BF4FF4FA6300230B4494F851
:1074B8002218194402F0DAFA002384F8DC38C6E608
:1074C800334B1B6819067FF5C2AE394602F0CEFA77
:1074D80088F8DC78BBE684F8DD38D4F818382A4F09
:1074E8009A067FF5B4AE97F81C389B077FF5AFAEC8
:1074F800B7F820386421594302F0B8FA002387F816
:10750800DC38A4E684F8DD383AE0B37823B1C5F86E
:107518009C7886F802809EE5D5F89C38FB1AB3F56E
:107528007A6FFFF498AD0123D5F8A008B37008F07E
:10753800D0FD0646D5F8A00808F0CBFD76067FF406
:107548008AAD8A2802D08E280DD084E5D5F818385F
:1075580098067FF580AD95F89A38002B7FF47BADBF
:1075680005F6690306E095F89A38002B7FF473ADA9
:1075780005F63403C5F8A4382D2385F8A8386AE53C
:1075880004B0BDE8F08700BFAC110020E730002050
:10759800FC2C0020F8B504460E4617460025204668
:1075A80020210FF0DAFA0446D0B1013420460FF05A
:1075B80037FBB0F5617F05DB40F634039842A8BF7E
:1075C800184601E04FF46170A0F56170192390FB33
:1075D800F3F00DB9307000E070703B7801333B7008
:1075E8000DB90125DBE72046F8BD30B505460C4648
:1075F800134629462246BDE83040014802F03CBD0A
:10760800B0B701087FB504780646E4B9354B1921AF
:10761800186800EB840090F87B5090F879204D436F
:1076280005F5617590F87A30009590F87C00414333
:1076380001F5617101912C482146013402F01CFDCD
:10764800142CE3D14BE00FF0EBFA1328054641DC8C
:10765800244B701C1C68202100238DF80F300FF07C
:107668007CFA1E35064670B1013630460FF0D8FA5E
:107678001A289FBF04EB850358709DF80F3001331B
:1076880098BF8DF80F30304620210FF066FA064675
:1076980070B1013630460FF0C3FA0D289FBF04EBD6
:1076A800850398709DF80F30013398BF8DF80F301F
:1076B80004EB85043046E11C0DF10F02FFF76AFF69
:1076C8009DF80F30042B0AD0601C002104220FF013
:1076D8000EFA04E0054800211322FFF786FF04B0E4
:1076E80070BD00BF24110020CFB70108E4B701081E
:1076F800014809F063BF00BFEAB70108F8B504788C
:10770800064674B9304D2146B5F8C621B5F8C831DA
:107718002E48013402F0B0FC042C05F10405F2D126
:10772800F8BD2B490FF0ECF9A8B9274B4FF47A7143
:107738004FF4FA62A3F8C611A3F8C821A3F8CA1136
:10774800A3F8CC21A3F8CE11A3F8D021A3F8D21125
:10775800A3F8D421F8BD30460FF062FA0328054695
:107768002BD8304620210FF0F8F9044630B1013407
:1077780020460FF055FA0126074600E00646204647
:1077880020210FF0EAF910B9BDE8F840B0E7013060
:107798000FF046FA012EF7D140F2DC53A7F2EE22A1
:1077A8009A42F1D8A0F2EE229A42EDD8064B7035F3
:1077B80003EB8503DF801881F8BD0648002103220A
:1077C800BDE8F84011E700BFD4110020F8B7010860
:1077D8000BB8010862C601082DE9FF410478054687
:1077E800002C34D16D4809F0E9FE6D4D686900211F
:1077F8000BF0B0FD002840F0CE802146694802F029
:107808003BFC6869694602F0BDFA0146664802F029
:1078180033FCA869694602F0B5FA0146624802F0ED
:107828002BFCE869694602F0ADFA01465E4802F0B1
:1078380023FC286A694602F0A5FA013401465B4830
:1078480002F01AFC0C2C05F11005CFD1A3E0584921
:1078580005220FF099F938B9514B00220344103032
:10786800C0285A61F8D196E02846524904220FF000
:107878008BF904462846002C3FD120210FF06DF9E2
:10788800002800F08880451C28460FF074F9074648
:10789800494B53F824601EB9484809F08FFE7AE036
:1078A80028463146FAB20FF06FF901340028EFD1BB
:1078B8003B4B0021C2181030C02851619E46F7D1B9
:1078C8003F4B03EBC402D2F804C09846BCF1000F4A
:1078D80004D131463B4802F0CFFB53E0002718F8AB
:1078E80034309F42F5DA3B010EEB0305143563444F
:1078F8000FCB013785E80F00F1E70FF091F90B285E
:10790800064643DC284620210FF027F9054648B1F2
:107918000135284602F0A0F9214B012403EB061398
:10792800586100E00446284620210FF016F9054664
:1079380040B10135284602F08FF9194B013403EBA9
:1079480006139861284620210FF007F9054640B133
:107958000135284602F080F9114B013403EB061378
:10796800D861284620210FF0F8F810B9FFF7C0FEBB
:1079780011E0013002F070F9094B032C03EB0616F5
:107988003062F3D11048FFF727FF04E00F480121C8
:107998000C22FFF72AFE04B0BDE8F08111B80108F7
:1079A800D41100202CB8010832B801087CC30108A2
:1079B8000BB8010836B80108D0B101083BB8010876
:1079C800E0B601084AB8010883B50108E4B7010820
:1079D800F0B5047887B0064614BB514B19201968D6
:1079E800062303FB041191F8CA5091F8CE204543B1
:1079F80005F5617591F8C930009591F8CB50C831FB
:107A0800684300F56170019008790290497945480A
:107A180003912146013402F02FFB0C2CDDD17CE0D0
:107A28000FF0FEF80B28044672DC3D4B701C1D68F5
:107A3800202100238DF817300FF08FF8064680B10B
:107A4800013630460FF0ECF803289FBF062303FBEE
:107A5800045383F8CE009DF817309CBF01338DF88E
:107A68001730304620210FF078F8074680B10137EB
:107A780038460FF0D5F80D289FBF062303FB0453A3
:107A880083F8C9009DF817309CBF01338DF8173073
:107A980006266643A9193846CA310DF11702FFF7C1
:107AA80079FD20210FF059F8074670B101373846A3
:107AB8000FF0B6F814289FBF9DF8173076190133D8
:107AC80086F8CC0098BF8DF81730384620210FF083
:107AD80044F878B101300FF0A3F80D289FBF0623B2
:107AE80003FB045383F8CD009DF817309CBF013386
:107AF8008DF817309DF81730062B0ED0062202FBA2
:107B080004500021C9300EF0F2FFFFF7F1FD04E048
:107B1800054800210B22FFF768FD07B0F0BD00BF44
:107B28002411002056B80108E4B701082DE9F347ED
:107B3800047806464CB9204601A90AF071FD0134C3
:107B4800FFF7F4FF122CF6D17AE00FF069F8C5B20E
:107B5800112D70D83C4C05F1D00704EB4703701C7D
:107B6800202193F802800EF0F8FF384E034630B912
:107B7800A8F10202D2F1000848EB020845E000F142
:107B8800010A597830460EF0E8FF60B1032D8CBF2A
:107B980003230023801BC0B23344184490F8049098
:107BA800B9F1030F02D1FFF7A3FD49E0A9F10203E0
:107BB800D3F1000850464FF0200148EB03080EF0BF
:107BC800CCFFD8B1B8F1000FEDD001300FF028F894
:107BD80040F2ED2380B2984205DD40F6CA03984290
:107BE800A8BF184601E040F2EE20A0F2EE201922CC
:107BF80090FBF2F004EB4703D87002E0B8F1000FF5
:107C0800D1D104EB470383F8029004EB4704A3782F
:107C1800F25CB8F1000F09D0E17819234B430C4806
:107C2800294603F2EE2302F027FA09E0294609481B
:107C380002F022FA04E0084800211122FFF7D5FCDF
:107C480002B0BDE8F08700BFD4110020A494010859
:107C580076B8010888B8010862C6010800220849F8
:107C68000C2303FB02135968814204D10022C2622B
:107C78001A725A6070470132042AF0D1704700BF67
:107C8800C028002010B5084B0022196801EBC20378
:107C980093F90240844201D1981C10BD0132042A94
:107CA800F4D1002010BD00BFBC280020F0B5027838
:107CB80087B08AB94A4C04F1200694F8F6210023CB
:107CC800484950B2595681426DD00C33302BF7D108
:107CD8000834B442F1D180E0002204920592451C98
:107CE8000EF09EFFC4B260B2FFF7CCFF074618B192
:107CF8008DF81040012400E00446284620210EF0AB
:107D08002CFF054638B1013528460EF089FF0134AD
:107D1800ADF81200E4B20026284620210EF01DFF1F
:107D2800B0B3451C28460EF07BFF00222E495FFAAF
:107D380082FE51F82230834204D00132082AF5D15C
:107D4800002300E0734651F82320824220D1022EFE
:107D58000FD0032E12D05A1E012ED2B204D0042AFC
:107D680013D88DF814300EE0042A0ED88DF815308B
:107D780009E0052B09D88DF8173004E09A1E052A6A
:107D880003D88DF816300134E4B20136042EC3D17D
:107D9800052C03D807B0BDE8F040A9E404AB03CB39
:107DA8003860796019E094F8FB010F4B94F8FA51A8
:107DB80053F82000B4F8F821009094F8FD0153F826
:107DC8002000019094F8FC0153F8200053F8253066
:107DD8000290064802F050F97AE707B0F0BD00BFFC
:107DE800D4110020C028002088A0010897B80108F5
:107DF80038B1438811EA030003D08B420CBF01203D
:107E08000220704730B50A4B0A491C680A78032AD1
:107E18000AD81346551C04EBC303EAB29D882842CE
:107E2800F5D00A70981C30BD0A70002030BD00BF24
:107E3800BC280020901A0020014B00221A70E1E7AC
:107E4800901A00202DE9F047877890F803C0BBB25C
:107E5800C7F1640E03EB83065C42C3F178001C4D46
:107E68005FFA8EFE7600CCF16408A4B280B2A3B2A9
:107E78000FFA83F9B9F1000F04DC002B14BF3B465D
:107E8800012300E0734609FB09F25B4302FB0CF295
:107E980092FBF3F3434403FB09F30A2293FBF2F347
:107EA80033449BB225F8023FB1F800904A880A345F
:107EB800C9EB020A1AB202FB0AF24FF47A7392FB78
:107EC800F3F3A4B24B4484422B80D0D1BDE8F087B1
:107ED800901A002010B544780078002240F6C411AA
:107EE80002FB02F3193B634303F6C41353434343B2
:107EF80093FBF1F3034921F812300132072AEDD13F
:107F080010BD00BFAA1A0020104B043033F910002E
:107F1800B0F5617F05DB40F633039842A8BF1846E9
:107F280001E04FF461700A7819235A4302F2833250
:107F3800824208DA4A78534303F283338342B4BF58
:107F48000020012070470020704700BF382D002016
:107F580010B500F1500302788A4203D18478C278C0
:107F6800944204D304309842F5D1002010BD01207A
:107F780010BD0B4B1B6813F4805F0A4BB3F9063036
:107F880005D0C089421A934207DD084400E0008A00
:107F98008342B4BF0020012070470120704700BF12
:107FA800FC2C0020382D00201FB5084B1B681B0334
:107FB80009D58DF80400039101230D2001A98DF83E
:107FC800053001F0AFF905B05DF804FBFC2C00208A
:107FD8001FB5084B1B681B0309D58DF804000291D7
:107FE80000230D2001A98DF8053001F09BF905B09B
:107FF8005DF804FBFC2C002010B5064B00241C7017
:108008000AF0C8FE044B83F82840DC621C865C63D7
:1080180010BD00BFB8300020901A002010B510B96C
:10802800BDE81040E8E700230C225A430A4C111916
:10803800125D824203D00133102BF5D110BD074BDE
:10804800586B18B14A784078824203D200225963AB
:108058001A86DA6210BD00BF74A30108901A0020C6
:1080680010B540001428A8BF14200023074A022195
:1080780099540B4499181424834201F8014CF5DBF8
:10808800FF21D1540F20BDE81040C7E7D42C0020B1
:1080980010B50A4A0A4B11689B6800BF12689142E2
:1080A800F7D1084A4FF47A70946B00FB04F2D31AA4
:1080B800B3FBF4F300FB013010BD00BF202D0020FE
:1080C80010E000E0901A002038B50446FFF7E0FF02
:1080D8000546FFF7DDFF401BA042FAD338BD10B5B7
:1080E80004462CB14FF47A70FFF7EEFF013CF8E735
:1080F80010BD2DE9F84381460B26013E31D01B4BBC
:1081080010225A6108221A6109F101074FF032085A
:108118000525164C4046E36883F01003E360E368E6
:1081280083F00803E360FFF7DAFFE368404683F073
:108138001003E360E36883F00803E360FFF7CFFF11
:1081480045B1013DE5D14FF4FA70FFF7C8FF4FF094
:10815800FA08DEE7013FDCD14FF47A70FFF7BFFF82
:10816800CBE7034A034BDA60BDE8F883000C014013
:108178000400FA0500ED00E0024A136801331360B9
:10818800704700BF202D0020024BDB6B03B118475E
:10819800704700BF901A002003685B6918472DE9F3
:1081A800F743064689469DF8288011461A469DF8E9
:1081B8002C3000250C2068431A4FC419C057B04210
:1081C80002D1207A20B126E00135042DF2D122E037
:1081D800012E0AD003DCF6B90093134807E01E2EDF
:1081E8000AD01F2E17D1012006E0104800934346FD
:1081F80004F0B9FA044605E004F056FE4146044688
:10820800FFF7CAFF4CB10C2303FB0575267185F8EF
:1082180008906C6001E0002000E0204603B0BDE853
:10822800F08300BFC028002000380140004400400F
:1082380003681B69184710B504462046FFF7F8FF86
:1082480018B90A20FFF74BFFF7E710BD38B500242F
:108258000B4D6059254409F0B1F9696811B1094815
:1082680001F00AFFA96811B1074801F005FF0748A6
:10827800103409F0A3F9B4F5D87FE9D138BD00BFAF
:1082880070990108B6B80108BCB801083AC40108D9
:10829800F0B585B004460EF06EFC082826D1621EA3
:1082A800E01D1F4912F8013F09681944497801F097
:1082B8000301022908BF203B82421370F1D12546F1
:1082C80004F1080715F8016B164831460EF045FC15
:1082D80020B1284631460EF040FC10B1FFF708FAED
:1082E8001CE0BD42EED1204606F09CFE0E4809F087
:1082F80065F900230D4A04A91A4492F88A210A4410
:108308000849595C0133082B02F80C1CF2D10023F0
:10831800074801A98DF80C3001F0AEFE05B0F0BD9C
:10832800580000208ECF0108C2B80108D4110020DF
:108338007CC301082A4B2B4C1E6880B52068FFF7C8
:108348007AFF3046FFF777FF206841798D0703D41D
:1083580041F00201FFF720FF234B08221A61234D49
:1083680010221A612B689A0341BF06236371E379CF
:1083780023F0010344BF43F00203E371206807F0D0
:10838800ABFE90B1184F08237B61164B186807F0B5
:10839800A0FE804602F032FB08B108F0FBF9304637
:1083A800414607F09CFE08233B61304607F094FEE7
:1083B80078B10D4F4FF01008C7F814803046D4F844
:1083C800009007F086FE0146484607F088FEC7F889
:1083D80010802B689B03D1D505F01BFACEE700BFB0
:1083E800C42C0020D01A0020000C0140FC2C0020D6
:1083F8002DE9F04705460EF0BEFB2F4E0446D6F891
:10840800088090B92D4809F0D9F82D4B53F824105D
:1084180049B10123A34013EA080F02D0294801F00B
:108428002BFE0134F1E7284822E028462749224656
:108438000EF0AAFB58B9264809F0C0F8254C54F8A4
:10844800041F0029EFD01F4801F016FEF7E72B782C
:108458004FF000092D2B03BF013504F1FF344FF015
:10846800010A4FF0000A164B53F8297027B91A4829
:10847800BDE8F04709F0A2B82846394622460EF072
:1084880083FBA8B9012000FA09F0BAF1000F03D064
:1084980001F086FF114803E040EA0800B060104888
:1084A80009F08CF83946BDE8F0470E4801F0E4BD04
:1084B80009F10109D7E700BFD4110020C8B80108A5
:1084C800209B0108D2B801083AC40108D6B80108AF
:1084D800DBB801081C9B01083BB80108E7B8010894
:1084E800F0B801087BC3010810B5084809F066F820
:1084F800074B00241C741C64064B1C7007F092FF89
:1085080009F034FA044B1C6010BD00BFF8B801082C
:10851800D01A0020E8300020C42C002070B5064690
:1085280000240B4BE518AA8816420AD0E1580948DE
:1085380001F0A2FD2846002108F0D1FF064809F005
:108548003DF840F6BC4314349C42EAD170BD00BFEC
:1085580014A5010824B901083AC40108F0B5047843
:108568008BB005460CB1002436E04B4B19680E233E
:1085780003FB0411B1F91D51B1F91921B1F91B31EE
:10858800009591F8205101F58C70019591F82151D1
:1085980001F59071029590F90700039091F9021086
:1085A8003E4804912146013401F066FD082CDCD1D7
:1085B80070E02D2B14D1072C1BDC28460EF030FB65
:1085C8000AAB661C03EB440424F8100C15F8013FB1
:1085D800303B092BFAD934462B78002BE9D104E03B
:1085E800A3F13002092A09D8E5E7082CBDF81820BC
:1085F80009D00BB0BDE8F040FFF77AB8202BF8D1CE
:1086080001352646E7E7072AF3D840F2DC55BDF8DE
:108618001A00214BA0F2EE2189B2A9421B68E8D8C2
:10862800BDF81C10A1F2EE24A4B2AC42E1D8BDF80A
:108638001E6004B237B2A742DBDB0DB2AF42D8DC12
:10864800A542D6DBBDF8247007F16404A4B2C82C97
:10865800CFD8BDF826E00FFA8EF4112CC9DCBDF88E
:108668002050B42DC5D8BDF82240B42CC1D812B2C0
:108678004FF00E0C0CFB0233A3F81901A3F81B11E1
:10868800A3F81D6183F8205183F8214183F81F71F5
:1086980083F822E10BB0F0BD241100202EB90108A7
:1086A800F0B504468FB020460EF065FAC5B21DBB82
:1086B800AB4808F083FFAB4C94F8D61009B9AA4828
:1086C80053E049B294F8D42094F8D530009194F846
:1086D800D710A648019194F9D8100734029194F95B
:1086E800D210039194F8D31004912946013501F072
:1086F800C3FC102DE0D1E2E720469D4905220EF08B
:1087080043FA0546B8B929469A4870220EF0EFF99F
:108718002846994B19680E2303FB001301300022E9
:10872800082883F8232183F8242183F8252183F856
:108738002621F0D112E12046904904220EF024FAB5
:1087480005462046002D4AD120210EF006FA0028C1
:1087580000F00481461C30460EF00DFA2C46074600
:10876800874B53F824502DB986480FB0BDE8F04028
:1087780001F082BC30462946FAB20EF005FA0134FF
:108788000028EDD1774A164602F17001002382F8DD
:10879800DA3082F8D63082F8D53082F8D430073211
:1087A8008A42F3D1784901EBC40191F80822934237
:1087B80010DAD1F80C72C3EBC302B0183A44176848
:1087C80000F1D401C0F8D470908801338880927980
:1087D8008A71E7E729466D4801F04EFC8FE06C4945
:1087E80007220EF0D1F905462046002D49D1202157
:1087F8000EF0B3F906460EF0BEF9C4B26CBB65487C
:1088080001F03AFC21466448013401F035FC0E2C95
:10881800F8D1554801F030FC00246048214601F0A9
:108828002BFC0025544A012311680E2202FB041276
:10883800D2F82321AB401342594B5A495A4808BF32
:108848001946013501F018FC0E2DEBD146480134CC
:1088580001F012FC082CE0D180E0304653490EF0BC
:10886800E3F92C4600284CD0022C4FD00EF0D8F952
:1088780006AB43F824004D4900200EF0D5F9013429
:10888800F0E74A490EF0D0F9002460B1082C38D03E
:108898000EF0C6F906AB43F82400444900200EF058
:1088A800C3F90134F1E7082C2BD1069B0F2B28D8EC
:1088B800DDF81CE0BEF1070F23D8089F0D2F20D844
:1088C800099E06F16402C82A1BD80A9DFF2D18D8F4
:1088D8000B98642815D80C99642912D8884210DAA4
:1088E8000D9C032C0DD8324AC3EBC303134483F801
:1088F80004E05F719E71DD71187259729C722D4C83
:10890800D1E60FB0BDE8F040FEF7F2BE069B072B9C
:1089180020D807990D291DD80278722A0DD06E2A01
:1089280018D1154A0E20126800FB032301228A4041
:10893800D3F8231121EA020209E00F4A0E20126837
:1089480000FB032301228A40D3F823110A43C3F80A
:10895800232101E0FEF7CCFE0D4CA4E60FB0F0BDDC
:1089680056B90108D41100203AC4010881B9010898
:108978000BB80108A81200202411002036B80108FD
:10898800D0B101083BB80108709901084AB801083C
:108998004EB90108C0B801089DB90108ADC0010869
:1089A8004FC8010895C70108A2B90108A6B901086E
:1089B800A412002083B501082DE9F7430478054681
:1089C8008CB9324D95F8AB12B5F8A82295F8AA32B1
:1089D8002F4800912146013401F04EFB102C05F17F
:1089E8000405EFD14EE00EF01BF90F28044636DCE3
:1089F800284620210EF0B1F8264EE4B2D6F844807D
:108A0800451CA400002728460EF00AF95FFA87F9EA
:108A1800B9F1010F83B208D0B9F1020F0BD0B3F549
:108A2800B47F24D2726C13530AE0FF2B1FD8736CE7
:108A38002344987004E0FF2B19D8736C2344D87032
:108A480028462C210EF089F8054608B1013502E0C8
:108A5800B9F1020F0BD10137032FD4D112E00E4820
:108A680000210F2203B0BDE8F043FEF7BEBD08EBBE
:108A78000400002104220EF03AF803B0BDE8F043E8
:108A8800FEF736BE03B0BDE8F08300BFD411002066
:108A9800A8B90108D01A0020E4B701082DE9F0436D
:108AA80004788FB00546002C59D17C4B0021142244
:108AB80009A807AED3F848800EF019F80722304607
:108AC80000210EF014F800231A46A70005A8059304
:108AD80008EB070583807249B5F802E031F813C046
:108AE8001CEA0E0F0AD00E310DF1380C595C02F158
:108AF800010E624402F81C1C5FFA8EF20133072B48
:108B0800E9D100210B46674AB5F802E011F802C026
:108B18001CEA0E0F0AD006320DF1380C8A5C03F1FC
:108B2800010E634403F8242C5FFA8EF30131062901
:108B3800E9D118F807308DE841006A785A4902925D
:108B480009A81A0903F00F0301F081FA21465748D2
:108B580009AA013401F090FA202CA6D19BE00EF06E
:108B68005FF81F28044600F3898028462021E4B2D4
:108B78000DF0F3FF1F2C02D9FEF7BAFD8BE0474B2F
:108B8800451C9B6C002103EB8404204604220DF055
:108B9800AEFF0027464B09AE304600210A2217F8DF
:108BA80003905FFA87F80DF0A2FF002315F8012B58
:108BB80032B10A2B04D04A4502D0F2540133F5E70A
:108BC8004A4561D108F1FF33032B09D8DFE803F0E8
:108BD800100502420DF1230037E00DF123011FE0DB
:108BE80030460EF01DF82378C0B243EA001006E0C4
:108BF80030460EF015F8237800F00F001843207067
:108C080034E00133062B0BD02A4800F2F3269E5D90
:108C18009642F6D1034493F8ED22638813436380A8
:108C280011F8012F12B30023EEE70133072B0CD004
:108C3800204A02F2E6269E5D8E42F6D102EB4303FD
:108C4800B3F8D82263881343638010F8011F69B111
:108C58000023EDE730460DF0E3FF0F2804DC304633
:108C68000DF0DEFF607001E0002363700137052F0F
:108C780090D1012407F034FD6CB97DE70E4800213E
:108C88001F22FEF7B2FC06E02046002104220DF068
:108C98002EFF0024EEE70FB0BDE8F083D01A0020C5
:108CA800489C01085D9C0108BCB90108CBB90108C2
:108CB800699C010870990108E4B701082DE9F04F93
:108CC800AB498BB004460DF01BFFAA49002820468B
:108CD8000CBF012507250DF013FFA74900282046E2
:108CE80008BF02250DF00CFF002808BF0425E9077E
:108CF80040F1E680A14808F061FC002008F06EFA17
:108D08009F4CA04808F05AFC9F4808F057FC63792C
:108D18009E4A013B52F823109D4801F0ADF99D4849
:108D280001F0AAF926460027D6F81480002140460B
:108D38000AF010FB20B1984801F09EF9002669E07E
:108D480039469648D6F818B0D6F81CA0D6F8209020
:108D580001F092F9404600210AF006FB10B12020EC
:108D680008F024FC06A9404601F00CF801468C489E
:108D780001F082F9584600210AF0F6FA10B12020D5
:108D880008F014FC06A9584600F0FCFF0146844888
:108D980001F072F9504600210AF0E6FA10B12020DD
:108DA80008F004FC06A9504600F0ECFF01467C4898
:108DB80001F062F9484600210AF0D6FA10B12020E5
:108DC80008F0F4FB06A9484600F0DCFF013701462D
:108DD800744801F051F90C2F06F11006A4D1AAE746
:108DE80049B294F8D42094F8D530009194F8D7106B
:108DF8006D48019194F9D8100734029194F9D21072
:108E0800039194F8D31004913146013601F034F9F6
:108E1800102E03D094F8D6100029E1D1634808F049
:108E2800CDFB574B624C9F6854F8041F19B1614839
:108E380001F022F9F8E70E465F4B53F826404CB193
:108E48000123B3403B4203D05C48214601F014F9AA
:108E58000136F1E75A4808F0B1FB2146484B0AAA07
:108E68000B4493F88A311344564A8A5C0131082925
:108E780003F8102CF2D1002306A953488DF82030AE
:108E880001F0FAF8514808F099FB5148FEF70EFF37
:108E9800504808F093FB4E48FFF700FE4E4808F094
:108EA8008DFB4B48FFF788FD4C4801F0E5F8402062
:108EB800FFF734FB4A4808F081FB4548FEF736FEC9
:108EC800AA0739D5474808F079FB474808F076FBE8
:108ED8003F4808F0C3F9454808F070FB3C48FEF7E6
:108EE80091FB434808F06AFB3948FEF771FD414899
:108EF80001F0C2F83648FEF701FC3F4808F05EFB77
:108F08003348FFF72BFB00260E27774300243B4A04
:108F18000123D26CA3403A44D2F80A2013421ED14E
:108F280001340E2CF3D10136082EEDD12B4801F077
:108F3800A3F88020FFF7F2FA6B0716D5304808F03F
:108F48003DFB304808F03AFB214808F061F9234816
:108F580001F092F84FF48070FFF7E0FA05E031462F
:108F68002246294801F088F8DAE70BB0BDE8F08F0F
:108F7800D7B90108E7BD0108DEB90108E4B901085D
:108F8800D4110020F2B9010804BA0108D0B10108CF
:108F980010BA01081BBA010828BA010835BA010835
:108FA800BFB801087CC301084DBA01083DBA0108E1
:108FB8001C9B01086CBA0108209B01087ABA0108B9
:108FC80087BA01088ECF010893BA01089CBA010834
:108FD80083B50108ABBA0108B7BA01083AC4010859
:108FE800C5BA0108D2BA0108E5BA0108F3BA0108FE
:108FF800FDBA01080CBB01081ABB0108D01A0020F1
:1090080026BB010837BB010849BB0108344B354A68
:109018001B68126810B51A60334A116859605168A4
:1090280092689960DA60314A1168196151689268EA
:1090380059619A612E4A1168D9615168926819621A
:109048005A622C4A11881985518859859188D28885
:109058009985DA85284A118819865188598692880F
:109068009A86264A1188D98651889288198719467E
:1090780021F83A2F224A10780022824206DA214C3F
:1090880034F81240013221F8024FF6E71E4A1288DE
:10909800A3F864201D4A1288A3F866201C4A118888
:1090A800A3F86C1051889288A3F86E10A3F870206A
:1090B800184A3B2112689A66174A126892FBF1F225
:1090C800B2F5967FC8BF4FF0FF325A67134A12882D
:1090D800A3F87820124A5289A3F85E2010BD00BF79
:1090E800802D0020CC300020302A00203C2A00208F
:1090F800482A0020CC11002008110020B6110020B9
:109108007F2A00202811002034290020AC100020DC
:109118000E110020C011002004000020481100207A
:10912800141100202DE9F84305460E460D4B002486
:1091380093E88003B44213DA7B1933F9140008EB7F
:10914800050333F9142009EB050333F9143001340E
:109158001344022293FBF2F3C01A08F0C9FFE9E7AF
:10916800BDE8F883802D002070B5472008F010FF77
:10917800174B1B681B0307D5164B174A5B6810680B
:109188001B68C01A08F0A5FF144E154C154D307811
:1091980008F09FFF23682868C01A08F0A9FF6368D1
:1091A8006868C01A08F0A4FF0F4B188808F091FFF0
:1091B8000E4B188808F08DFF0D4B188808F089FFB2
:1091C800337823742B68A3606B68E36070BD00BFBD
:1091D800042F0020802D0020CC300020CE19002044
:1091E8006C2D0020D0190020CC190020CA190020AD
:1091F800501100207FB5264C264E274D2749284A76
:10920800284B20B128480088B0F5805F31D23088DB
:1092180091F820101278ADF8040028781C4D1B78BE
:109228008DF806008DF807108DF8082001A829464A
:1092380006228DF809300DF03FFC30B30198BDF8D7
:1092480008302860AB80532008F0A2FE208808F080
:1092580040FFA07808F03DFFE37801A80193237947
:1092680002936379039308F09BFE0F4B00221A8048
:109278000BE0308891F820102080127828781B782D
:10928800A070E17022716371DDE704B070BD00BFAA
:10929800201B00208C1A0020C819002094300020C0
:1092A800230F0020880F0020242F0020A0F17D0329
:1092B800012B70B504460D460A4E05D830687D214D
:1092C80006F00DFF84F020043068214606F007FF01
:1092D80035B12B881C4404EB142404F0FF042C80C3
:1092E80070BD00BF7C1A00200A4A1388013313801E
:1092F800094A136801331360084A138801339BB283
:10930800202B01BF00231380054A138808BF0133AF
:1093180013807047242F00200C2F0020102F0020CE
:10932800122F002038B53A4B05461B780C46083BEF
:10933800012B6BD8452008F02BFE284608F028FEA4
:109348000C2D23D004D80A2D0AD014D835B138BD35
:109358000E2D4BD02ED3FF2D50D038BD206849E0BC
:10936800207808F015FE62796378002A14BF8020FF
:109378000020184300E0207808F00AFEA07808F0E2
:1093880007FEE07808F004FE20793BE0B4F900001D
:1093980008F095FEA07808F0FBFDE07808F0F8FDED
:1093A800B4F9040008F08BFEB4F90600BDE83840B3
:1093B80008F085BE637820788BB180F0800008F0D3
:1093C800E7FDA468E0B208F0E3FDC4F3072008F065
:1093D800DFFDC4F3074008F0DBFD200E12E008F0C3
:1093E800D7FD6068BDE8384008F082BE206808F004
:1093F80070FE6068BDE8384008F06BBE054808F0AC
:10940800A5FD0020BDE8384008F0C2BD38BD00BF4A
:109418005C2D002058BF01082DE9F04FBE4B8BB0E2
:109428001A880193BD4F002A40F0A98042F2010337
:10943800B7F8D607BA4EC21A50425041FFF7DAFEC3
:10944800FFF7E4FD34684920254608F0A1FDB54B37
:1094580004F11C09186808F03CFE55F8040B08F0E4
:1094680038FE284605F066FD04F1100005F062FD9F
:109478004FF01008AC4D01232A6803FA08F3134291
:1094880003D0D9F8000008F033FE08F10108B8F15C
:10949800130F09F10409EDD104F1280005F03AFD94
:1094A800B7F84431B4F92E00C01A08F012FE2B6840
:1094B800DB0408D59D4BB4F864001B88181AC0F368
:1094C8000D0008F006FE2B68980403D5B4F8660072
:1094D80008F0FFFD2B68590503D504F16C0005F071
:1094E80019FD2B681A0502D5A06E08F001FE2B683D
:1094F8005B0402D5606F08F0FBFD2B68180403D5E8
:10950800B4F8780008F0E5FDA04604F1300005F055
:1095180001FD04F1360005F0FDFCB7F8443138F9D7
:109528003C0F0127C01A08F0D4FD814B1B789F42DD
:1095380008DA38F9020FB4F93C300137C01A08F0DC
:10954800D7FDF2E72B68990505D5B4F95E00A0F2BE
:10955800DC5008F0CDFD326876487260B260121AAD
:109568009110754A4A43531C032293FBF2F202EB13
:1095780042029A1A7C2303FB02033360D6E16F4B45
:109588006F4A1B6811688B4206D00AA941F8203D32
:1095980000201360FFF7C6FE019B97F8D6171B88BB
:1095A80097F8D7070B44013BB3FBF0F200FB1233EB
:1095B8008B4280F086815A4F0120FFF71BFEFFF790
:1095C80025FD50203E687D6808F0E2FCBA683B68DB
:1095D80010681B687A680344106806F11C0BA3EB3B
:1095E800400008F085FD6A68736802A89B1A029318
:1095F800AA68B36805F11C089B1A0393EA68F36824
:1096080010249B1A049305F095FC2A69336902A873
:109618009B1A02936A6973699B1A0393B369AA69CF
:109628009B1A049308F0BCFC3F4901220B68A24036
:109638001A428A4606D0DBF80000D8F80030C01A73
:1096480008F056FD0134132C0BF1040B08F1040843
:10965800EAD106F1260005F12601002331F9024F6F
:1096680030F9022F121B02AC44F823200133042BDB
:10967800F4D103214FF000094FEA89035FFA83F917
:1096880002AB53F821206AB102F108000F2802D872
:1096980049F0010906E08032FF2A94BF49F0020927
:1096A80049F0030911F1FF31E6D24846002408F0D9
:1096B8006FFCA0460DF1080B09F00302022A16D030
:1096C800032A1DD0012A4ED1B8F1000F05D1DBF8CD
:1096D800004090462401E4B245E0DBF800004FF07A
:1096E800000800F00F00204308F052FC3BE0B8F1FE
:1096F800000F0CD0DBF80000C0F3031020432CE06F
:10970800B8F1000F1ED19BF8010008F041FC9BF84E
:10971800000008F03DFC26E0102F0020D4110020A6
:10972800802D00200C2F0020042F0020002F002067
:109738007F2A00208C2D0020DF7BEFBD182F002012
:10974800142F0020DBF80000C0F30330204308F09A
:109758001FFCDBF80000C0F3071008F019FCDBF869
:1097680000402401E4B20BF1040B06AB9B454FEA21
:109778009909A1D1B8F1010F02D1204608F008FCDF
:10978800DAF8003013F480541FBFB6F86420B5F837
:1097980064100124521A18BF02929A040AD50AAA20
:1097A80002EB8401B5F86600B6F866200134121A97
:1097B80041F8202C580513D502AA02EB840C06F1B7
:1097C8006A0E05F16A0000223EF9021F30F9028F85
:1097D800C8EB01014CF822100132032AF4D10334FA
:1097E800190508D50AAA02EB8400A96EB26E0134E5
:1097F800521A40F8202C5A0408D50AAA02EB840011
:10980800696F726F0134521A40F8202C18040BD576
:109818000AAB03EB8402B5F87810B6F87830013457
:109828005B1A42F8203C00E0FCB1012C03D10298FD
:1098380008F05EFC19E0631E002002AA52F82320FB
:109848004000C0B20AB140F00100013BF5D508F074
:109858009FFB4FF0000802AB53F8280008B108F04E
:1098680047FC08F10108A045F5DB30200321FFF78C
:1098780059FC36200321FFF755FC2F4B3C20197863
:10988800FFF750FCDAF80030990506D5B6F95E0006
:10989800B5F95E30C01A08F02BFC3A6827487B6897
:1098A8007A60121A9110264ABB604A43531C03225D
:1098B80093FBF2F202EB42029A1A7C2303FB0203A7
:1098C8003B60204B1B681A0630D51F4C1F4D226881
:1098D8002B689A420BD162686B689A4207D1019B48
:1098E8001B88102B11D11A4B1B885B060DD1482001
:1098F80008F04EFB206808F0FBFB606808F0F8FBF6
:1099080023682B6063686B600EE0124A0F4B117876
:109918002A7C914208D1104A99681068884203D17C
:109928005268DB689A4201D0FFF71EFC08F000FB82
:109938000BB0BDE8F08F00BF7F2A00208C2D0020DF
:10994800DF7BEFBDFC2C0020541100206C2D002083
:10995800122F0020CE190020D01900202DE9F84F31
:109968000C9EC2EB030B394C0B9B002914BF4FF024
:10997800060A4FF0040AF61A636805460133904652
:1099880013D1236853455ED2314A032B98BF294629
:1099980052F823202F4808F0E9FA636800220133BF
:1099A80063602D4B05469A7113E0002511E02B4AA0
:1099B8001278954240DA0B9BE3B109FB06F2995CF9
:1099C80001228A40264909680A4213D16368013393
:1099D8006360D4F804900A9B1C4F9945E7DB2BD1B0
:1099E8000A2008F0D5FA3B6801333B604FF0FF339B
:1099F8007B6021E0184A917921B12C2008F0C8FA3F
:109A0800013501E00121917109FB0BF3226808EB94
:109A1800030752B958F8030008F098FA97F90410A8
:109A280005444B1CD2D00F4802E03A440E48117945
:109A380008F09CFA0544C9E7206850452CBF00206F
:109A48000120BDE8F88F0020BDE8F88F1C2F00200A
:109A58002C9D010863BF0108201B00205400002032
:109A6800042F002072BF0108ADC0010830B585B0D1
:109A780004AC002524F8025D0091ADF806002146EB
:109A88001020FFF713FC9DF806002146FFF70EFC97
:109A98009DF807002146FFF709FC9DF800002146C4
:109AA800FFF704FC9DF801002146FFF7FFFB9DF836
:109AB80002002146FFF7FAFB9DF803002146FFF755
:109AC800F5FB9DF80E002946C043C0B2FFF7EEFB38
:109AD80005B030BD10B5054C206806F0FDFA18B188
:109AE800206806F0F6FAF6E710BD00BF4C1A002011
:109AF800F0B50124B0FBF4F58D4201D34C43F9E7EE
:109B08000026D4B1B0FBF4F504FB1500B4FBF1F466
:109B18001EB9002D01DC002CF3D1092D03F1010E33
:109B2800EFB204DD002A14BF3725572500E03025A1
:109B38003D441D7001367346E3E71C70F0BDF0B577
:109B48000124B0FBF4F58D4201D34C43F9E700261C
:109B5800D4B1B0FBF4F504FB1500B4FBF1F41EB965
:109B6800002D01DC002CF3D1092D03F1010EEFB219
:109B780004DD002A14BF3725572500E030253D4471
:109B88001D7001367346E3E71C70F0BD03685A1C6C
:109B98000260197070472DE9F843089E002B0746AC
:109BA80088461446334614BF4FF030094FF0200959
:109BB80013F8012B0AB9254603E0002CFBDD013C14
:109BC800F6E7002D04DD38464946C047013DF8E771
:109BD800354624EAE474A01B284415F8011B11B18A
:109BE8003846C047F7E7BDE8F883024B186806F027
:109BF80076BA00BFB8100020F8B507460C4648688A
:109C0800002115461E4609F0A5FB58B1284609F063
:109C1800B9F9104909F00AFA01464FF07E5009F0E7
:109C2800B9FA60606168304609F0F8F801463046D4
:109C380009F0B0FA256806462946384609F0ECF8D6
:109C48000146304609F0F2F90146284609F0E6F8DF
:109C58002060F8BDDB0FC9402DE9F04102780346CA
:109C6800202A00F10100F9D0092AF7D02D2A02D1C3
:109C78000346414D04E02B2A08BF03464FF07E55AA
:109C88001C460026234614F8012BA2F13007F9B22E
:109C980009290DD83949304609F0C8F90646384629
:109CA80009F070F90146304609F0B8F80646E9E7C8
:109CB8002E2A17D1314F234614F8010B3038C2B27F
:109CC800092A0FD809F05EF9394609F063FA014606
:109CD800304609F0A3F829490646384609F0A6F99E
:109CE8000746E8E71A7802F0DF02452A39D15A78A0
:109CF8002D2A02D10233012704E02B2A14BF013395
:109D080002330027013B002413F8012F303AD1B267
:109D1800092903D80A2101FB0424F5E7B4F59A7F41
:109D280028BF4FF49A74A0464FF07E53B8F1070F3E
:109D380007D91846124909F079F9A8F10808034625
:109D4800F4E704F0070434B118460C4909F06EF939
:109D5800013C0346F7E719462FB1304609F01AFAD5
:109D680004E04FF07E51304609F060F9014628467C
:109D780009F05CF9BDE8F081000080BF00002041D7
:109D880020BCBE4C30B5054687B00C4603A8002160
:109D98000C220CF0ACFE2846002109F003FB20B190
:109DA8002846284909F03AF803E02846254909F0E9
:109DB80033F8254909F03AF909F0FEFA054680EA30
:109DC800E0706946A0EBE57008F02AFC002DACBFF6
:109DD80020232D2368468DF80C300CF0CCFE01288A
:109DE80007D130238DF80D308DF80E308DF80F30F7
:109DF8000CE0022805D130238DF80D308DF80E3097
:109E080004E0032804BF30238DF80D30694603A809
:109E18000CF094FE03A80CF0AEFE0338C5B22A4637
:109E280003A920460CF0D2FE0023635520460749BB
:109E38000CF084FE03AB204659190CF07FFE204637
:109E480007B030BD6F12033A00007A4496BF01088C
:109E580070B50646B6FBF2F40846154614B120461E
:109E6800FFF7F6FF05FB1464024B1B5D00F8013B8E
:109E780070BD00BF98BF01082DE9F04F81468A46A2
:109E880016461C4689B000253178002900F0DB8091
:109E9800252902D00136484674E072784FF0000850
:109EA800302A0CBFB278B71CA2F1300312BF4FF0B2
:109EB800000BF71C4FF0010B092B19D8A2F1300346
:109EC800D9B2092905D80A2202FB083817F8012B4C
:109ED800F4E7A2F16103052B02D8A2F1570305E0CC
:109EE800A2F14103052B03D8A2F137030A2BEADDBF
:109EF8006C2A30D13A787E1C642A00F083800BD813
:109F0800252A3DD003D8002A00F09D80BCE7582AB6
:109F18000CD0632A19D0B7E7732A22D002D86E2A48
:109F280037D0B1E7752A5CD0782AADD1271D2068D3
:109F3800A2F1580462424FF01001624155E02CD959
:109F4800582A32D0632A2AD13E4648462178271D0E
:109F5800D04701350FE0642A63D00ED9732A14D193
:109F68003E46236848460093514642460023FFF781
:109F780012FE271D05443C4686E7252ADFD13E46CA
:109F880048462521D04701357EE70AD86E2A06D1F2
:109F98003E46236804341D6076E7002A53D03E46C7
:109FA80072E7752A26D0782AF9D1A2F1580304F16C
:109FB800040C5A422068CDF80CC04FF010015A41E9
:109FC80005ABFFF795FDDDF80CC03E46644605ABD2
:109FD80000934846514642465B46FFF7DCFD054480
:109FE80052E72068271D0A21002205ABFFF7A7FDCD
:109FF8003C46ECE704F1040CCDF80CC020680A21BB
:10A008000022DDE72068271D002808DA2D238DF8B7
:10A01800143040420DF115030A210022E6E705AB92
:10A02800FAE7206804F1040C00280ADA2D238DF8D9
:10A03800143040420DF11503CDF80CC00A2100225E
:10A04800BFE705ABF8E7284609B0BDE8F08F0EB4C6
:10A058000FB505AB53F8042B0190064901A80393EB
:10A06800FFF70AFF019B00221A7004B05DF804EBA9
:10A0780003B07047959B00080FB413B50B4904ABA8
:10A0880008680B4953F8042B09680193FFF7F4FE9D
:10A098000446084B1868FEF7CBF80028F9D020468C
:10A0A80002B0BDE8104004B0704700BFCC000020EB
:10A0B800C8000020B810002080EAE073A3EBE0732A
:10A0C8008B4206DB002801DD401A704702D00844A5
:10A0D80070470020704770B5044609F06DF92030CC
:10A0E800402857D820462C4909F05CF928B1204669
:10A0F8002A4908F091FE0446F4E72046284909F069
:10A1080033F928B12046254908F088FE0446F4E7CB
:10A118002046244909F046F930B12249204608F082
:10A128007BFE01461F480AE020461F4909F01CF93A
:10A1380040B11C49204608F071FE01461A4808F053
:10A148006BFE04462146204608F070FF054620466F
:10A15800294608F06BFF15490646284608F066FFB1
:10A16800134908F059FE0146284608F05FFF1149D7
:10A1780008F054FE0146284608F058FF0E4908F03A
:10A188004BFE0146304608F051FF0146204608F0D4
:10A1980045FE70BD002070BDDB0F4940DB0FC94094
:10A1A800DB0F49C0DB0FC93FDB0FC9BF9A7C2E36D6
:10A1B800FAAF4F393587083CA4AA2A3E08B50349A7
:10A1C80008F02CFEBDE8084085E700BFDB0FC93F5B
:10A1D8002DE9F04F056885B0814628460C46FFF703
:10A1E800EDFF80462846FFF776FFD9F8045006466B
:10A1F8002846FFF7E3FF07462846FFF76CFFD9F824
:10A20800089005464846FFF7D9FF82464846FFF7BB
:10A2180062FF41468146504608F008FF41468346A2
:10A22800484608F003FF51460190304608F0FEFE0C
:10A2380049460290304608F0F9FE394603905046E8
:10A2480008F0F4FE4946206007F1004008F0EEFEF1
:10A2580029466060A560029808F0E8FE014601986A
:10A2680008F0DCFD2946E060039808F0DFFE0146AF
:10A27800584608F0D1FD3946206106F1004008F043
:10A28800D5FE29466061584608F0D0FE014603987D
:10A2980008F0C2FD2946A061019808F0C7FE0146F2
:10A2A800029808F0BBFD4146E061384608F0BEFE62
:10A2B800206205B0BDE8F08F2DE9F04107688AB04B
:10A2C800466885680446084601A9FFF781FF019999
:10A2D800384608F0ABFE04998046304608F0A6FEE2
:10A2E8000146404608F09AFD07998046284608F03E
:10A2F8009DFE0146404608F091FD029920603846CF
:10A3080008F094FE05998046304608F08FFE014615
:10A31800404608F083FD08998046284608F086FEE6
:10A328000146404608F07AFD03996060384608F017
:10A338007DFE06990746304608F078FE0146384605
:10A3480008F06CFD09990646284608F06FFE01469C
:10A35800304608F063FDA0600AB0BDE8F081074B05
:10A3680010B51A881C4622EA00009042188002D0D4
:10A378000120FDF775FE208810BD00BF8C1A002053
:10A38800064B10B51A881C4610439042188002D01C
:10A398000120FDF765FE208810BD00BF8C1A002043
:10A3A800024A936823EA000090607047D4110020A5
:10A3B80008B5104B1A780023D9B2914207D20E493A
:10A3C800002051F82310013309680880F4E732208F
:10A3D800FDF785FE094B1B685A0309D5084B9B6896
:10A3E8005B0305D4BDE8084040F2DC50FDF777BEBA
:10A3F80008BD00BF7F2A0020802A0020FC2C0020F6
:10A40800D41100202DE9F34108F0A2FC4B4A69233E
:10A41800137040F2DC735380BE231371EF2382F86C
:10A42800D93700231946164682F8DA37F25C013329
:10A43800514040F2DC729342F8D1404B404A83F8D5
:10A44800DA17404B04275A6002F188325A6000201C
:10A45800013F17F0FF075FD03A4B3422DA6000243F
:10A4680054B100234FF4005056F80480019304F0CF
:10A4780057FF0428ECD11DE04FF4302004F050FFC2
:10A488000428E5D12F4D4FF430202B6943F0020307
:10A498002B612D4B6B612B6943F040032B6104F05A
:10A4A8003FFF41F6FD732A69042803EA02032B6182
:10A4B800D7D0CDE7234D1FFA88F22B694FF400500F
:10A4C80043F001032B6104F1006303F57E331A8026
:10A4D80004F026FF042814D11C4B4FEA18482344E3
:10A4E8000193019B4FF40050A3F8008004F018FF7B
:10A4F80041F6FE732A69042803EA02032B6106D099
:10A50800A6E741F6FE732A6913402B61A0E740F2E3
:10A51800DC7304349C42A3D10A4A0428136943F02B
:10A528008003136102D107F077FA10B90520FDF70F
:10A53800E0FD08F0F7FB02B0BDE8F081D41100207F
:10A54800230167450020024000F8030802F80308C9
:10A558002DE9F04107F060FA10B90420FDF7C9FDB4
:10A56800B84C08F0F5FBB84940F2DC7220460CF014
:10A57800B3FA94F8B0374FF4CC71022B84BF0023A0
:10A5880084F8B03794F8B027B04D01FB02F303F517
:10A598003A7020442344286093F83C0301FB0242AC
:10A5A800022803F54E7384BF0020187192F83C33DB
:10A5B800A74A13700C2202FB0343A64A03F2B273A4
:10A5C800136046F20902A3681A401AB99D4A43F477
:10A5D80000539360A368DE0703D54FF40050FFF7DC
:10A5E800DFFEA368580409D50820FFF7D9FE4FF409
:10A5F8000050FFF7D5FE0120FFF7D2FEA368190728
:10A6080006D54FF40050FFF7CBFE0120FFF7C8FE38
:10A61800A3689A0413D54FF40040FFF7C1FE894B95
:10A6280093F88631012B03D14FF40060FFF7B8FE91
:10A638004FF48030FFF7B4FE4020FFF7B1FEA36867
:10A648005B0603D54FF48030FFF7AAFE94F8E021AB
:10A658007C4B2AB193F8E42112B1002283F8E4215B
:10A668004FF0000C67467C4E7C4B1E6004EB0C03DD
:10A67800B3F8F8E14FEA5E0101F077314FEA9E0343
:10A6880003F03333C1EB0E00C11A4FEADE0303F0C7
:10A698001133CB1A03EB231303F00F32FF2392FB82
:10A6A800F3F31EF00108C3EB032318BF0137A2EB35
:10A6B800030318BFFFB2012B0ADD022B40F0BE8056
:10A6C800B8F1000F00F0BA801EF0BC0F00F0B680A1
:10A6D8000CF1080CBCF1200FC8D1013F012F00F28A
:10A6E800AD8007F075F9302200215D480CF0FFF9C4
:10A6F8005C4F5D4BD5F800801F605C4B002108F172
:10A708007900C3F80080FDF723FC594B80F0010065
:10A718001870584B07F126021A60574B07F1D402FC
:10A728001A6098F8000005F047FF2868534B00F5B9
:10A73800C5721A6000F0E0FC514B94F8D81107F18B
:10A7480094021A6064224A434E4BC8325A6000226F
:10A758009A60DA601A615A619A61DA6183F8202096
:10A7680083F82120484B2D6807F12C021A60474BCB
:10A7780005F219121A60464B05F289121A60454B08
:10A7880007F108021A60444BDFF848811F60434B09
:10A7980007F1A0021A6007F1AA03C8F80030404B7D
:10A7A800B4F866011E6008F0E9FBC8F80800B4F8C0
:10A7B800680108F0E3FB95F85C3008F1040288F8BA
:10A7C800043095F87830C8F80C0088F8053094F80B
:10A7D800E331286E88F81030324BC8F814501A60EC
:10A7E800314B05F164021A60304908F01FFC01463C
:10A7F8004FF07C5008F0CEFCB5F816412C4B186091
:10A80800204608F0BFFB01462A4808F0C3FC2A4945
:10A8180008F00CFC294A2A4B15602A4A186005F1F1
:10A8280068031360284A05F211151560274A176056
:10A83800274ABDE8F041136008F074BA04F0C8FB79
:10A848004FE700BFD411002000F8030824110020AE
:10A85800A82C00204C1100205E1300208830002016
:10A86800BC0F002018130020F00F0020F40F002068
:10A8780018000020C8070020F00500200010002064
:10A88800CC27002094300020200800201C1B00202A
:10A89800280A0020502B0020542B00203C090020BF
:10A8A800000A00205008002088080020DB0F4940DB
:10A8B80084080020000061444C3D0F4490070020AC
:10A8C80038090020840700202809002030090020CA
:10A8D8007C060020281B002008B5FFF793FDFFF732
:10A8E80037FEBDE808400120FDF7BABB10B508F0F7
:10A8F80049FB0021044608F055FD08B1204601E057
:10A9080004F10040054908F045FC054908F08EFBB4
:10A91800FFF754FC034B186010BD00BF8096184B1E
:10A9280035FA8E3C3C0000202DE9F04105460E46E4
:10A93800078A83899BB21F40002F37D0B7FA87F266
:10A948004FF00043D340DB4399B21F40A2F11B03F1
:10A958002982042BF0D8DFE803F0221F1C1903001A
:10A96800746A24B1013C0023A4B2736201E0AC8D87
:10A97800A4B2D6F82080B8F1000FDDD0D8F80030A6
:10A98800404621469847D8F80480F4E73068A98EF5
:10A9980008E07068298F05E0B068A98F02E0F068C8
:10A9A800B5F84010036889B29847C5E7BDE8F0815B
:10A9B80038B50D4B0D4D99680D4B1A681C465288D9
:10A9C800114203D0FDF764FB286007E0FDF760FB48
:10A9D8002B68984282BFC01A064B186023685A68D1
:10A9E800054B5A6138BD00BF000C0140401B0020D8
:10A9F800980700200400002000040140F8B59C4B93
:10AA080004461B68187818B1012800F06A819AE298
:10AA1800242C984D0CD006D80A2C00F0D9800D2C87
:10AA280000F0D68048E12A2C06D02C2C04D043E133
:10AA380028716871A87150E18F4B69792F790020CE
:10AA48008C4A58542FBB1978D771472921D1597886
:10AA580050291ED19978472907D1D978472904D197
:10AA68001979412901D10121D1719978824A522954
:10AA780003D1D1784D2900F0688299787E4A472918
:10AA880007D1D178532904D11279562A04BF032259
:10AA9800EA71EA79774E022A39D0032A4CD0012A82
:10AAA80040F08580BA1E072A00F28180DFE802F0B4
:10AAB80004080F131A257F2A07F006FDA86076E020
:10AAC8001B78532B73D1AB685B42AB606FE007F028
:10AAD800FBFCE8606BE01B78572B68D1EB685B42A6
:10AAE800EB6064E01B78302B644B1A788CBF42F023
:10AAF800020222F002021A7059E0002007F044FD19
:10AB0800287454E0002007F03FFD68824FE0072FCB
:10AB180006D0082F4BD1012007F036FDF08246E021
:10AB2800012007F031FD41F2184358434FF47A737E
:10AB3800B0FBF3F0B0823AE0022F07D0032F0AD11E
:10AB4800002007F021FD4E4B187030E0002007F080
:10AB58001BFD30762BE02AD93A1F9210337E013242
:10AB6800D2B2013B02EB8303DBB2102B1FD8F91ED4
:10AB7800C2F1010201EB8202D2B2012A0BD0042AEF
:10AB880011D100205E1E07F0FFFC3E4B00229855B5
:10AB98003D4B9A5507E03D4A5E1E0020935507F04D
:10ABA800F3FC3B4B98553B4A136801331360314B18
:10ABB8002A2C18BF9A7907F101074FF000000CBF43
:10ABC800012254402F7168710CBF5A769C7184E041
:10ABD800687E002848D0304B13F8012D2F495A7051
:10ABE8008B42F9D1244A234C13785278402B85BFE5
:10ABF800373B1B011B01DBB298BF03F0F003402A6F
:10AC08008CBF373A303AD2B21344AA79DBB29A42AF
:10AC180027D121230B702249E0790B68012803F121
:10AC280001031E4A0B600AD002281CD1722313703C
:10AC3800A28A1C4B1A80E28A1B4B1A8013E06723F6
:10AC480013700E4B1B789F070ED5184BA2681A601D
:10AC5800E2685A60227C164B1A70628A154B1A8079
:10AC680002E03F230B70002000236B7635E000BF25
:10AC7800BC070020401B0020282D0020C8190020F8
:10AC88006811002099110020891100206911002005
:10AC98007911002030270020C4020020B0020020D3
:10ACA8003C270020CA19002050110020D01900208C
:10ACB800CE190020CC1900206B79687E0E2B9FBF1F
:10ACC800A54A591C5171A54A98BFD454A24A18B92B
:10ACD80093795C40947100E00020003018BF012097
:10ACE800F8BD9D4B0022997E082900F22C81DFE8EF
:10ACF80001F0050B0F15202B475D6700B52C40F0C0
:10AD08002281DA76012239E0622C08BF022235E07E
:10AD180003229A761C775C779C7714E104229A7652
:10AD28005A7F997F2244D2B25A770A449A77DC77BD
:10AD380009E105229A765A7F997F2244D2B25A773E
:10AD48000A449A771C84FEE006229A765A7F997FF5
:10AD58002244D2B25A770A449A771A8C02EB042416
:10AD6800A4B2B4F5AC7F82BF7B4A0121D176002220
:10AD78001C845A84002C40F0E68007229A76E2E090
:10AD88005A7F997F2244D2B25A770A449A775A8CCA
:10AD9800B2F5AC7F3EBF7049891881F82440013272
:10ADA800198C92B291425A84E7D9CCE008229A765B
:10ADB8005B7FA34200F0C780674B0122DA760DE083
:10ADC800674D9A7615F8012D6A70664A9542F9D151
:10ADD800997F614AA14206D03F232B70624A53688B
:10ADE80001335360AFE06148016801310160D07EF2
:10ADF80010B13E232B70A6E021212970D17F0629AE
:10AE080041D004D8022907D0032923D0F8BD12293C
:10AE180059D0302967D0F8BD5021946A2970544917
:10AE28004C60D46A0C60516B4FF47A7491FBF4F166
:10AE3800504C218092F87C114F4A19B1117841F099
:10AE4800020102E0117821F002011170012283F859
:10AE58007D2169E05321297092F82910CE0705D584
:10AE680092F82820D51E6A426A4100E0024602F0A4
:10AE7800010183F87C11002A56D13F490A7822F053
:10AE880002020A7050E04F21297092F82F10CC0767
:10AE980005D592F82E20D11E4A424A4100E00246CA
:10AEA80002F0010183F87C1122B933490A7822F0B3
:10AEB80002020A7093F85310304A1170B3F8501018
:10AEC8002F4A118030E05621946B29702D490C804F
:10AED80042F21074D16B91FBF4F12B4C21800121CB
:10AEE80082F87E1120E04921297092F82810274A1B
:10AEF800102988BF10211170254914780022A24218
:10AF08000ED20E7A234D56554E7A234D5655CE7A8B
:10AF1800224D565511F80C6F214D56550132EEE76A
:10AF280020490A6801320A6093F87D310A4A002BE9
:10AF38003AD092F87E31BBB3002182F87D1182F8B5
:10AF48007E111846F8BD0020F8BD1279432A7FF417
:10AF580094AD0222EA7190E5401B0020282D0020C4
:10AF6800C4020020B00200209C0700203C270020DB
:10AF7800D0190020CC190020C8190020CE190020B3
:10AF880046000020CA190020501100206811002036
:10AF9800641B00206911002079110020891100200C
:10AFA8009911002030270020F8BD0449044B096896
:10AFB800002218705A6199611A777047202D002075
:10AFC8009C070020F8B5101A0D461F4607F0DAFF57
:10AFD8000446781B07F0D6FF174B079E196808F040
:10AFE80025F821460546204608F020F82946074658
:10AFF800284608F01BF80146384607F00FFF0CF00A
:10B00800E7F90E4908F012F808F0FCF9069B294602
:10B01800186004F100400CF04FF8094908F006F8F0
:10B02800084907F0FBFE08F0C7F90028BCBF00F587
:10B038000C40A0303060F8BD3C0000202C7D8E3FD5
:10B04800A00CB34500A00C4644F25063984203DDBF
:10B05800A0F50C40A0387047034B9842BCBF00F5E0
:10B068000C40A030704700BFB0B9FFFFF7B50368C8
:10B07800174C184D23600B68174E63600068FFF784
:10B0880035FC95E80300154B0196009394E80C00F5
:10B09800FFF798FF3668124B60681E606B68114FA7
:10B0A800C01A07F06FFF104B196807F0BFFF08F0D0
:10B0B80083F92A68236878609B1A3B600B4B1E60F3
:10B0C8000B4B1B68DA880B4B1A8003B0F0BD00BF2E
:10B0D800482C0020D0190020542C0020502C00208F
:10B0E800902C0020582C00203C000020882C0020A8
:10B0F80000100020842C002070B50446407907F029
:10B108003DFF1E4908F046F81D4D1E4E2860E07BA5
:10B1180007F034FF194908F03DF8EE606860A0793F
:10B1280007F02CFF184908F035F8184D2860207CE6
:10B1380007F024FF114908F02DF86860A07E07F099
:10B148001DFF134908F026F8EE60A860E07907F0C3
:10B1580015FF0D4908F01EF80E4D2860607C07F0B9
:10B168000DFF064908F016F86860E07E07F006FF54
:10B17800074908F00FF8EE60A86070BD0000C842EB
:10B18800602C00200000FA4400002041702C0020B0
:10B1980000007A44942C002010B50C4C23789B07AF
:10B1A80013D50B4B1B78042B0FD90A4A0A4B10688E
:10B1B800526818605A60FFF799FB084B1A88084BC9
:10B1C8001A80237843F00103237010BDC8190020AA
:10B1D800CE190020D019002054110020C4110020DD
:10B1E800A42C0020164B13B51B681B0325D5154B43
:10B1F800154C1B7815498DF80030154B20681B78C5
:10B208008DF8013007F012FF08F0FCF811498DF8AD
:10B218000200606807F00AFF08F0F4F88DF80300F0
:10B22800A06808F0EFF80C4B8DF804001B780A2092
:10B2380069468DF80530FEF775F802B010BD00BFFD
:10B24800FC2C0020EE2C0020102D002000002041B6
:10B258000C2D002000007A44F22C0020054A1378B7
:10B2680083F001031370044A00231360034A136038
:10B27800B8E700BFF22C0020082D0020042D002084
:10B2880001480249FFF750BB00080040282B002066
:10B2980001480249FFF748BB00040040002B00208A
:10B2A8004FF080400149FFF73FBB00BFD82A00207C
:10B2B80001480249FFF738BB002C0140B02A0020A2
:10B2C80001480249FFF730BB002C0140B02A00209A
:10B2D800254B10B55A43254B254C1B680139B3FB48
:10B2E800F2F20388013AA04289B292B29BB212D01C
:10B2F80004F50064A0420ED0B0F1804F0BD0A4F545
:10B308009834A04207D004F58064A04203D004F525
:10B318008064A04202D123F070039BB2154CA04276
:10B3280006D004F58064A0421CBF23F440739BB28E
:10B3380003800F4B8185984202850FD003F5006387
:10B3480098420BD003F54063984207D003F5806319
:10B35800984203D003F58063984201D10023038605
:10B368000123838210BD00BF40420F00500000201F
:10B37800002C01400010004073B505460068FFF737
:10B38800A7FF2A680124138800269BB243F0010313
:10B398001380EB7A01A88DF804308DF805408DF8FC
:10B3A80006608DF8074006F0A9FEEB7A1B2B0BD13F
:10B3B800192301A88DF804308DF805408DF8066032
:10B3C8008DF8074006F09AFE02B070BD0C4B800A5B
:10B3D80098420CD004D8B0F5801F0CD101207047DA
:10B3E800084B984205D04933984206D003E0022022
:10B3F800704703207047FE2070470020704700BF49
:10B4080001001000020010002DE9F8430468074607
:10B41800204688469146FFF7D9FF03284BD8BA7AC9
:10B428009108B8F1000F06D1A589AEB202258D406A
:10B4380026EA0505A5810A2303FB00131F4A42F8E3
:10B448002380043342F82390B8F1000F07D0BD7A67
:10B45800A189AD080223AB400B439BB2A3812823EB
:10B46800434303F120011144EFF31286502585F37D
:10B47800128803F10C051C331544134455F8047F56
:10B4880017B10F60296804319D42F7D100230B6082
:10B49800F3B283F31188282303FB0020036A23B146
:10B4A800A3899BB243F0010304E0A38923F00103BD
:10B4B8001B041B0CA381BDE8F88300BFB02A002041
:10B4C800FFF776BAFFF774BAFFF772BA014801F0CE
:10B4D800E7B800BFC01C0020014801F0E1B800BF78
:10B4E800141D00200C4B4FF400525A604FF6FE73A7
:10B4F8000A48D0F8082211680B401360D0F8F821E8
:10B50800D0F8FC319A4203D000F5EA7001F0FAB89D
:10B51800012380F81832704700000240401B0020C9
:10B5280037B5044603211E2006226B46F9F788FF2B
:10B5380078BB9DF801309DF80000174D43EA0020C4
:10B5480000B207F01FFD296807F070FD07F034FF0F
:10B558009DF8033020809DF8020043EA002000B2E5
:10B5680007F010FDA96807F061FD07F025FF9DF8B9
:10B578000530A0809DF8040043EA002000B207F0DF
:10B5880001FD696807F052FD07F016FF6080012091
:10B5980000E0002003B030BD200000201FB50446A5
:10B5A80002210C2001220DF10703F9F749FF08B920
:10B5B80000203BE09DF80730DB07F9D50321062280
:10B5C80002AB0C20F9F73CFF0C20092101220DF1F8
:10B5D8000703F9F735FF0028EAD09DF8073013F084
:10B5E8000C0FE5D19DF809209DF808300C2043EA9E
:10B5F8000223C3EB83339B009DF80B2023809DF827
:10B608000A300A2143EA0223C3EB83339B009DF8E7
:10B618000D2063809DF80C3043EA0223C3EB83338B
:10B628009B00A3800122FAF70DF9012004B010BD98
:10B6380007B50A2100220C20FAF704F91420FCF7B8
:10B648004EFD0A210F220C20FAF7FCF80A20FCF71D
:10B6580046FD01AB102103220C20F9F7F1FE0A2068
:10B66800FCF73DFD0A2100220C20FAF7EBF80A202E
:10B67800FCF735FD0DF10303022101220C20F9F737
:10B68800DFFE0DF10303092101220C20F9F7D8FE92
:10B698000A2101220C20FAF7D5F803B05DF804FB63
:10B6A8002DE9FF41604B1B689BB11A681AB15F49CD
:10B6B800886902438A619A889868ADF80420022252
:10B6C8008DF8072004220DEB02018DF8062001F009
:10B6D800B9FB3220FCF703FD002111221E20FAF7E6
:10B6E800B1F8012160221E20FAF7ACF86420FCF7BB
:10B6F800F6FC002402A8FFF713FF274626460A2572
:10B70800022101221E20FAF79DF83220FCF7E7FCFF
:10B7180002A8FFF705FFBDF90820BDF90A10144477
:10B728008A42A8BF0A46BDF90C300F4493421E4412
:10B73800A8BF134613F5805F09DD3D4A013DD36874
:10B7480083F01003D360DBD14FF0010801E04FF024
:10B7580000081E2000211222FAF774F80A25022197
:10B7680001221E20FAF76EF83220FCF7B8FC02A876
:10B77800FFF7D6FEBDF90820BDF90A10A41A8A42BF
:10B78800A8BF0A46BDF90C307F1A9342A6EB030600
:10B79800A8BF134613F5805F07DD254A013DD3682E
:10B7A80083F01003D360DAD101E04FF0000820469F
:10B7B80007F0E8FB01461F4807F0ECFC1E4D20F09F
:10B7C80000402860384607F0DDFB0146194807F0BD
:10B7D800E1FC20F000406860304607F0D3FB0146EA
:10B7E800164807F0D7FC20F00040A860002170221E
:10B7F8001E20FAF727F8012120221E20FAF722F846
:10B808001E2002210022FAF71DF86420FCF767FCCD
:10B81800B8F1000F04D14FF07E532B606B60AB6022
:10B8280004B0BDE8F08100BFA4020020001002406F
:10B83800000C014000406F462000002001C05E4619
:10B84800024640213C20F9F7FDBF024680213C20FA
:10B85800F9F7F8BF012828BF01202DE9F04F064667
:10B86800142000FB06F3704F89B0F918FC586F4B91
:10B878000A691C601E716E4BB1F80880DD69B1F869
:10B888000AA02A43DA61A2884D6822F440721204A1
:10B89800120C4AEA0809A28003A9C5F810900222EE
:10B8A8008DF80E0028460193ADF80C908DF80F2006
:10B8B80001F0C8FA019B00971F464FF0080BAA68D1
:10B8C80018EA020F03D10A20FCF7FEFBF7E70A206B
:10B8D800C5F81480FCF7F8FBC5F810800A20FCF7BF
:10B8E800F3FBBBF1010BEAD1C5F814A00A20FCF761
:10B8F800EBFBC5F814800A20FCF7E6FBC5F81080BE
:10B908000A20FCF7E1FB0222C5F810A0284603A98B
:10B918008DF80F201C228DF80E20ADF80C9001F048
:10B9280091FA444A03A894423A690BBF42F40012C0
:10B9380042F480023A613A610BBF3A693A6922F4EB
:10B94800001222F480023A61A38823F440731B0496
:10B958001B0CA38023889BB243F001032380A58896
:10B9680003F08EFC0599344B25F03F05B1FBF3F34A
:10B978002D042D0C1D43ADB2A5802288002522F090
:10B9880001021204120C22802C4A03A8B1FBF2F126
:10B9980000298AB208BF012242F400414FF496728E
:10B9A80053434FF47A7293FBF2F301339BB223842F
:10B9B800A1832388009A9BB243F001032380238844
:10B9C80023F4816323F002031B041B0C23804FF430
:10B9D80080432381142303FB0626737B01248DF8FF
:10B9E8000C308DF80D508DF80E508DF80F4006F084
:10B9F80085FB337B9DF80F208DF80C308DF80D50AA
:10BA08008DF80E501AB103A806F078FB08E05A0921
:10BA180003F01F039C4002F12003094A42F8234027
:10BA280009B0BDE8F08F00BF449D0108681D0020E3
:10BA3800001002400054004040420F00804F1200A6
:10BA480000E100E0914B70B51A68908A80B2C1B2EB
:10BA5800CE072ED5118821F400610904090C118044
:10BA6800118889B241F48061118000215971997956
:10BA780099B1D97911B9197AFF290ED10121D97152
:10BA8800597A022901BF118889B241F400611180F5
:10BA9800997A41F001011182E2E0997A01F0FE0100
:10BAA80011821A7AFF2A00F0DB80784AFF2151714F
:10BAB800D6E08D073AD5BFF35F8F587AC0B2012818
:10BAC80013D1997989B1D97979B1118821F4806133
:10BAD8000904090C1180BFF35F8F118B1188D8728C
:10BAE80089B241F4007111801BE0118BBFF35F8FA5
:10BAF800587A664902280AD1887940B1C97931B1A2
:10BB0800118821F480610904090C1180A2E0587A97
:10BB18005E49032805D1887918B1C979002940F010
:10BB28009980918889B241F4806198E04C0757D593
:10BB38000121D9729979002938D0D979002935D0CD
:10BB4800597A1088022959791ED920F48060000496
:10BB5800000C1080148ADD68C8B2E4B249B26C5493
:10BB68001188DC6889B241F4007111801968821C5F
:10BB78005A710A8A0130D2B240B222548A8892B2EB
:10BB880042F480628A8026E080B240F4007010801F
:10BB9800148ADD68C8B2E4B249B26C54128A411CF6
:10BBA80049B2D2B203306A54587114E0D97937488F
:10BBB80009B9017C41B1118889B241F40071118041
:10BBC8005A7901325A7106E0118889B241F48071BC
:10BBD80011800122C27119680A88D205FCD43FE09D
:10BBE80001F0400101F0FF04E1B15879168ADD68DF
:10BBF800C4B2611C40B2F6B22E54C9B25D7A597112
:10BC080049B2C81C854201BF908820F480600004B6
:10BC1800000C08BF90805A7A8A4221D11B4A02340C
:10BC280054711DE006061BD5597948B2451C0AD047
:10BC38005C690131205CC9B21082587A597149B2E5
:10BC480088420DD106E0197A5C711182997909B997
:10BC5800597A29B9918821F480610904090C9180E5
:10BC6800597A93F9050001318842084A0CD100211C
:10BC7800D171D17A31B111688A8822F440721204E4
:10BC8800120C8A8000221A7670BD00BF681D002041
:10BC980010B5204C2368998A89B211F4706F1CBFC3
:10BCA8000122627611F4E06F2AD01A8B9A888905EE
:10BCB80022F480624FEA02424FEA12429A801FD46D
:10BCC8001A8892051CD41A88D0050ED51A88D10571
:10BCD800FCD41A8892B242F400721A801A8892052B
:10BCE800FCD42079FFF7B6FD0AE01A8892B242F434
:10BCF80000721A809A8822F440721204120C9A80F8
:10BD08002268938A23F470631B041B0C938200231C
:10BD1800237610BD681D002008B508480AF02BFFDF
:10BD2800C0B209280246054B04DC01302021C0B20C
:10BD38009954F6E700221A5408BD00BF19270020BD
:10BD480008B507480AF017FFC0B21428044B04D8F6
:10BD5800421C20211954D0B2F7E700221A5408BD1A
:10BD6800192700202DE9F74FFCF792F9A64C8046D9
:10BD780026686568A768861BF643451BC71BED4305
:10BD8800FF43F60FED0FFF0F2EB93FB9002D00F05E
:10BD98008782B9462CE04FF0000929E0B14627E038
:10BDA80003EB8A0BBBF802301A050ED413F4805F3C
:10BDB8001DBF964A9BF801101268954A954B14BF0F
:10BDC80052F82120126843F82A20BBF80230D8051F
:10BDD80016D499050AD5904B1B7813F0040F0CBFA5
:10BDE8008E4A8F4A8B4B126843F82A2009F10109C1
:10BDF800207B5FFA89FA8B4982450B68D0D326E00D
:10BE0800894A5046594604F0FBFB884B1B885A0662
:10BE180003D550465946864A16E0580703D550467A
:10BE28005946844A10E0190703D550465946824AB4
:10BE38000AE09A0703D550465946804A04E0DB07D2
:10BE4800D4D5504659467E4A04F0DAFBCEE7DFF8EF
:10BE580008E20093BEF906307822A3F57A735343BB
:10BE68004FF47A7293FBF2F3F34603F22B13019328
:10BE780000225FFA82FE864517D2009B03EB820EF2
:10BE8800BEF802E01EF4806F0DD040F2671ADFF8AA
:10BE98008491019B39F822E09E449EFBFAFC0AFB40
:10BEA8001CEE29F822E00132E3E74DB308F5C3336D
:10BEB800A0336360637B544A13BB9373614B1B6865
:10BEC80013F0020F0AD0DFF894E19EF800E0BEF10B
:10BED800000F03D04FF0010E82F80EE0DA0506D508
:10BEE800594BDB781BB1A37B43F00203A3734A4B86
:10BEF8001B7813F0050F02BFA37B43F00403A37361
:10BF080094F80EE0BEF1000F03D13F4B5B7B002B92
:10BF18004FD094F80DC01CF0010FACF10C031DD1EB
:10BF2800BCF1030F07D8DFF8E8901EF0040F3B4A76
:10BF380008BF4A4600E0364AACF1040CBCF1070FD2
:10BF480005D8DFF81CC11EF0010F18BF6246DBB22E
:10BF5800032B0ED81EF0020F3C4B06E0DBB2032B7E
:10BF680006D82F4B2A4A1EF0020F18BF1A4600E0C7
:10BF7800274A4FF0000C5FFA8CF383420DD20B680E
:10BF880003EB8C035B881B0642BFD2F80090214B61
:10BF980043F82C900CF1010CEDE785B1BEF1000FD0
:10BFA80008D0637B184A0133DBB2142B06D1002377
:10BFB80004E025B1637B002BF3D100E05373002E1E
:10BFC80052D0234A3223B2F90250B2F90020002D90
:10BFD800B8BF6D42002AB8BF524295FBF3F592FBF9
:10BFE800F3F2EDB2D3B2AB4238BF2B46194A13B1C4
:10BFF80092FBF3F300E0134643442360E37B024AD9
:10C0080083BB01232FE000BF841D0020141B0020E8
:10C0180050B40108720E0020E730002058B3010820
:10C0280048B30108181B00206C9D01088C1A0020D9
:10C03800729D0108789D01087E9D0108849D010874
:10C048008A9D0108FC2C00209430002060B3010870
:10C05800CC110020400D0300382D0020141A0020B8
:10C0680068B301080023D3738F4D904B2D78E27B82
:10C07800ADB9002F00F00F818D4B267B1A788D4BC0
:10C0880002F0040293F800C08B4BD2B2D3F800E060
:10C098000B680021894D03EB86060F46B5E01AB9F7
:10C0A800874A1A61002508E0864AFAE70A68AB0061
:10C0B800D6187688760604D40135EBB28342F5D3D8
:10C0C800D7E7814EB6F90060192E25DD12F803E096
:10C0D80094F814C00EF00F09E14526690CDCDFF86E
:10C0E800CCC19CF815C0BCEB1E1FDEBFD6F800C043
:10C0F800DFF8D8E143F80EC012F803E094F816C050
:10C108000EF00F09E14533DBDFF8A0C19CF815C03C
:10C11800BCEB1E1F2CDC26E0193629DA12F803E0E6
:10C1280094F814C00EF00F09E14526690CDCDFF81D
:10C138007CC19CF817C0BCEB1E1FA2BFD6F800C07C
:10C14800DFF888E143F80EC012F803E094F816C04F
:10C158000EF00F09E1450BDBDFF850C19CF817C062
:10C16800BCEB1E1F04DBD6F800E0584E43F806E08F
:10C17800554EB6F90260192E1BDD12F803C094F86B
:10C1880014E00CF00F09F14526690CDCDFF81C916E
:10C1980099F81590B9EB1C1FDEBFD6F80090DFF8B0
:10C1A8002CC143F80C90D25C02F00F0CF4451EDD54
:10C1B80082E7193680DA12F803C094F816E00CF01A
:10C1C8000F09F14526690CDBDFF8E09099F8159026
:10C1D800B9EB1C1FDEBFD6F80090DFF8F0C043F8BB
:10C1E8000C90D25C02F00F0CF445FFF665AF94F8A2
:10C1F80017E0BEEB121FA2BF3668344A9E505BE7B9
:10C208005888000504D404330435B342F8D122E039
:10C218004AB101EB0C0A06209AFBF0F900FB19A0C1
:10C2280001280DDC01E057B9012793F801900EEBC6
:10C2380089003EF829A090F80290C07803E01746DC
:10C24800002081468246013125F802AC85F800902D
:10C258006870C9B2D7E7174A1378013B13F0FF0398
:10C2680008BF06231370124B1B785B0741BFBBF94D
:10C2780006304FF47A72A3F57A7303EBC30348BF11
:10C2880093FBF2F3124A46BF0133DBB2012392FB60
:10C29800F3F34344A36003B0BDE8F04F00F0F4BCEF
:10C2A80003B0BDE8F08F00BF230F0020841D0020DD
:10C2B800E73000202C000020141B0020740E002002
:10C2C80064B3010850B40108CC110020720E00209C
:10C2D800400D0300026B0346C16810B5406942B1C6
:10C2E8001A6C8C1A013A08BF0A46005D1A64C0B27B
:10C2F80010BD1A6A805C01328A4228BF0022C0B28F
:10C308001A6210BD436B13B190F844007047836AFA
:10C31800406A1B1A584258417047036B13B15B6857
:10C32800016C01E0C369016A8B423CBFC2689B187B
:10C33800581AC0B27047426A806A131A5842584164
:10C3480070474171704743799B070AD5436A8269F0
:10C35800D154436A01690133B3FBF1F201FB123393
:10C3680043627047437913F001031FBFC36803F1A9
:10C37800FF32C369006A1DBF181A1040C0B21846C0
:10C388007047437910B513F0010304460DD0FFF749
:10C39800E9FF58B1236A6269E168D05C0133B3FBF5
:10C3A800F1F201FB1233236210BD184610BDF0B53F
:10C3B800046D8279A389467923F4005312F0020FA1
:10C3C8004FEA03434FEA13430CBF00214FF40051D7
:10C3D80012F0040FA38114BF4FF4806E4FF0000ECB
:10C3E80016F0010F8768054614BF04200020B30724
:10C3F800238A48BF40F008029BB223F4405343EA23
:10C4080001032382A18948BF90B289B221F4B051B7
:10C4180021F00C014EEA010140EA0102A281A38A3F
:10C4280087B023F440731B041B0CA38201A802F0FD
:10C4380027FF039B049E264A944218BF1E46A389E1
:10C44800192272431BB2002BB4BF7E00BE00B2FBA0
:10C45800F6F66427B6FBF7F00001010907FB116344
:10C46800A28912B2002AB7BFD9001A013231B1FB32
:10C47800F7F2A7BF3232B2FBF7F302F0070210431C
:10C48800A8BF03F00F03AA79A8BF184380B212F01F
:10C49800010F20812B6D06D00E498B4202BF04206C
:10C4A80001F54841086112F0080F9A8A0BBF22F083
:10C4B800080292B2120442F0080208BF120C9A82D3
:10C4C8009A8992B242F400529A8107B0F0BD00BF37
:10C4D8000038014000440040417168E7816066E728
:10C4E80003460A4690F84602D96A9B7900F0DCBCFC
:10C4F80038B5A0F513746379A579DB0746D594F8A8
:10C50800383205F00105F3B1226B1068838DC3F34F
:10C518004E03838494F83C3223B1B4F84232013399
:10C52800A4F84232917A6A0000F01DFB012384F8D6
:10C538003B32002384F8393284F83A3284F83832AE
:10C54800A4F8403238BD94F83B322046012B04BF92
:10C5580094F8393284F83A3200F0F0FA94F83B2231
:10C56800236B3AB9012284F83B221868997A05FAB4
:10C5780002F207E0002284F83B2295421868997A73
:10C5880008BF0222BDE8384000F0EDBA38BD10B54A
:10C59800A0F5127494F83C22BAB9A36A616A994268
:10C5A80028D0591CA069A162C35C2069DBB25B007A
:10C5B80043F400738142A4F83E324FF00A0384F832
:10C5C8003D3228BFA262012312E094F93D327BB1CB
:10C5D800B4F83E1220464B08A4F83E3201F001019F
:10C5E80000F0D4FA94F83D32013B84F83D3201E082
:10C5F80084F83C3294F83832002B50D194F8393210
:10C608000133DBB2092B84F8393204D12046BDE866
:10C61800104000F093BA0A2B41D194F83B322BB961
:10C62800B4F8403243F00103A4F840326379D907E3
:10C638001CD5B4F84002820501D4C30705D4B4F868
:10C6480044320133A4F8443210E0E36AC0F34700EF
:10C658000BB198470AE0E3696269D054E369E1687D
:10C668000133B3FBF1F201FB1233E361012284F8D9
:10C67800382294F83B220023012A84F839320ED15B
:10C68800A27984F83B32236B12F0010F1868997A6B
:10C698000CBF02220022BDE8104000F064BA10BDB1
:10C6A800026D70B515880446ADB2A90613D5036BA3
:10C6B8008BB9C36A1BB1908880B298470BE0E169D7
:10C6C800928840694E1CD2B2E6614254E169E26840
:10C6D800914228BFE3612B0613D5636AA26A9A4286
:10C6E800236D0AD0511CA069A162825C9A802369DB
:10C6F800994206D30023A36270BDDA6822F0800253
:10C70800DA6070BD836A8169426B1944D160416AFD
:10C71800994297BF0169CB1ACB1A536096BF002381
:10C72800536083624FF0000380F84430136888BF79
:10C73800816243F0010313607047436A8269D154F0
:10C74800436A02690133934228BF00234362436B63
:10C758001BB11B68DB0705D4D4E7026DD36843F02F
:10C768008003D36070472DE9F0431E46944B8DB08B
:10C778009842894690469DF8507051D1914B924A03
:10C7880092491A60924AC3F808805A6102F5807289
:10C798009A614FF48072DA601A618E4A18651A63DA
:10C7A800A2F54842543ADA649A6459638A4B9A6902
:10C7B80042F480429A615A6942F001025A610223A6
:10C7C8008DF803303A074FF40073ADF8003001D507
:10C7D8001C230FE0B30706D51823804869468DF857
:10C7E800023000F02FFBF5070AD54FF48063ADF84F
:10C7F80000304823794869468DF8023000F022FB62
:10C808000E238DF804300022012301A88DF805308D
:10C818008DF806208DF807306A4C05F06FFC4EE065
:10C828006F4B984240F0C7806E4B674AC3F8088048
:10C838001A604FF48072DA601A616B4A18655A619F
:10C8480002F580729A61694A3C079A64DA64624B1D
:10C85800DA6942F40032DA615A6942F001025A6137
:10C868004FF002038DF803304FF00403ADF80030A9
:10C8780001D51C230EE0B00706D518235748694692
:10C888008DF8023000F0DEFAF10709D50823ADF87B
:10C8980000304823514869468DF8023000F0D2FA3A
:10C8A80026238DF804300022012301A88DF80530D5
:10C8B8008DF806208DF8073005F020FC494C00253E
:10C8C800012384F844302562E561A5626562C4F8F5
:10C8D8002C906671C4F80880A7712046FFF767FDA1
:10C8E800F20731D5206B002826D0E36C039501931D
:10C8F8004FF480530A9380230693E36805950493C5
:10C908002023099363690795029308950B9502F014
:10C918003FFC01A9206B02F01DFC226B216D1368FE
:10C9280043F0010313608B8A9BB243F040038B8270
:10C9380053689BB2236407E04FF6DF72236D1A80B9
:10C94800DA6842F02002DA60B3072CD5606B28B3AE
:10C95800A36C002501934FF480530A938023069318
:10C968002369029504931023039305950795089569
:10C9780009950B9502F00CFC606B01A902F0EAFB2B
:10C98800636B1A6842F002021A60226D5D605D6096
:10C99800938A9BB243F08003938204E0226DD368AC
:10C9A80043F08003D360226D204693899BB243F401
:10C9B8000053938100E000200DB0BDE8F08300BF74
:10C9C80000380140141D0020909D010844000240D9
:10C9D8009C1D002058000240001002400008014041
:10C9E80000440040C01C00209C1F0020044400405C
:10C9F80010F80A3C0133DBB20A2B84BF10F8131C71
:10CA0800044A00F80A3C82BF002322F8113000F8DB
:10CA18000A3C7047E02F0020334A70B5136C9068C9
:10CA2800194440F68C23081A98429160D0605160EE
:10CA380013463BD9127893F9451010468A420BD118
:10CA4800111F082908D893F84610182901D8013170
:10CA580003E083F8442002E0002183F8461093F9AC
:10CA680044402149A24219D191F84740B4B10C3150
:10CA78000024944206DA51F8046F1C4D25F814601E
:10CA88000134F6E70C2805D01849002421F8104095
:10CA98000130F7E7164801780131017083F8452025
:10CAA800002201211A7083F8471070BD92F84710D0
:10CAB800C9B140F2DA51A0F2EF248C4208D81178BB
:10CAC8000B2905D80B1D0131117042F8230070BDE8
:10CAD800002283F84720074B03F13002002143F876
:10CAE800041F9342FAD170BDF4000020E02F00200B
:10CAF8001C06002000010020024A136C013319446F
:10CB080011647047F4000020024B53F820301B6872
:10CB180019807047802A0020074BA1F57A7153F8D5
:10CB280020301A681B8959434FF47A7391FBF3F14B
:10CB380089B21180704700BF802A002090F83B32EC
:10CB480010B57BB990F83A3290F83942A34209D22D
:10CB5800B0F8401201229A400A430133A0F840225B
:10CB6800DBB2F3E710BD1FB50123ADF80830ADF80F
:10CB78000410002301A9ADF80A30ADF80C30ADF867
:10CB8800062002F0DEFB05B05DF804FB8379DB07C5
:10CB980048BFB1FA81F1D0F8343148BF49095A6821
:10CBA8001B8909B113617047536170471FB5012391
:10CBB800ADF808300023ADF80C30ADF80A30094B59
:10CBC800ADF804101B7801A9012B08BF0323ADF8A9
:10CBD800062008BFADF80C3002F0B3FB05B05DF8D5
:10CBE80004FB00BFF000002038B510F80E2C0446F6
:10CBF80050F8043C52B9012200F80E2C20F80C1C05
:10CC0800997A18680222BDE83840CFE730F80C2C32
:10CC180020F80A1C891A89B220F8081C074A10F85B
:10CC28000F0C002522F8101004F80E5C1868997A89
:10CC38002A46FFF7BBFF04F8065C38BDE02F00204A
:10CC4800044B53F820301BB107289CBF1B68198080
:10CC5800704700BF1C020020084A13689B020BD5CE
:10CC6800074B002119704FF6FE7306490868034008
:10CC78000B604FF400135360704700BF0000024080
:10CC8800E63000206C0002402DE9F047664D2B6825
:10CC98006649581C0A788E4602F0FF060AB1034618
:10CCA800F6E737462B60687BAB6895F80C80AA7B63
:10CCB80039B2202900F09C80DFF880C10CEB810399
:10CCC800DC789B783CF82110C3F1FF039BB2002B62
:10CCD80065D04FF03C0CB1FBFCF9C3F1FF03634393
:10CCE8001B12B9F1050F5DD8DFE809F0030B1A290B
:10CCF8003A4AE01A4143B1FBFCF0DAB21044C0B240
:10CD080051E0B1FBFCF00CFB101189B2DAB2C1F1B1
:10CD18003C01E31A4B43B3FBFCFC204694442CE053
:10CD2800B1FBFCF00CFB1011E21A89B24A43B2FBCA
:10CD3800FCF25FFA83F84244D2B2204632E0B1FBFB
:10CD4800FCF90CFB191189B2E01AC1F13C01484306
:10CD5800B0FBFCF05FFA83F84044C0B2224621E001
:10CD6800B1FBFCF80CFB1811D8B289B2E31A01FB2D
:10CD780003F2B2FBFCFC224684445FFA8CF412E016
:10CD8800B1FBFCF80CFB181189B2D8B2C1F13C0117
:10CD9800E31A4B43B3FBFCF20244D2B203E022464F
:10CDA800204600E044464FEA042C4CEA004C4CEA8A
:10CDB800020C17234FF0010808FA03F806F11701CF
:10CDC80018EA0C0FA1EB0301DFF8748014BF4FF0D1
:10CDD80011094FF0090989B213F1FF3308F80190DE
:10CDE800E8D218360137B6B2BFB2114BA0465FE79A
:10CDF800AB6001238EF8003040F22A33AA730D4A43
:10CE0800E9800D4985F80C806873AE805360002373
:10CE18008B840B889BB243F001030B80136843F0AB
:10CE280001031360BDE8F0879C210020E630002054
:10CE3800A82100206C00024000040040720E00206F
:10CE4800C5020020F0B5B1F800E000234EFA03F265
:10CE5800D50725D58E784FEAD30CF40648BFCC7891
:10CE680006F00F0203F0070748BF2243BF0050F83F
:10CE78002C500F24BC4025EA0404BA402243282E33
:10CE880040F82C2005D1C46801229A4024EA020205
:10CE980005E0482E04D1C46801229A402243C260AA
:10CEA8000133102BD2D1F0BD2DE9F04F1E464FF4BF
:10CEB80014734343554D85B005F1100480469146DF
:10CEC800E718A24610B92B44514A03E0012805D1BE
:10CED800504A2B441A641032C3F844214FF4147397
:10CEE80003FB08F34C48EC180AEB030203F59C73A8
:10CEF800343253442061E1636262A36200224FF43A
:10CF080080714FF0010BD4F844310320E1612263B2
:10CF1800E2622162A263626384F84C2284F848B218
:10CF280084F84922A4F85222A4F85422C4F818908C
:10CF38006075A67584F8568258681B8904F5A07236
:10CF48004FF0020CADF80C3003A9102301928DF8B4
:10CF58000E308DF80FC0CDF800C0FFF773FF236CBB
:10CF6800DDF800C0597B58681B898DF80E1003A99D
:10CF7800ADF80C308DF80FC0FFF764FF59463846FE
:10CF8800FFF704FE3220FBF7AAF8244B019A1B682E
:10CF9800D2F804B01A46B2FBF9F1B1F5803F03D3D9
:10CFA800012AF8D95208F6E71D4A4FF41474B3FB66
:10CFB800F2F204FB08F8584689B2D2B2FEF7DCF95F
:10CFC80005EB0809174B08F512780AEB080400224C
:10CFD800C9F8583258462146FEF716FAD9F8405093
:10CFE80016F0010F0CBF022200222868A97AFFF769
:10CFF800BAFD0D4B2846C9F85C32211D0022FEF708
:10D0080003FA384605B0BDE8F08F00BF9C21002028
:10D01800B0B30108D0B30108A89D01085000002052
:10D0280040420F0097C50008F9C400082DE9F743EE
:10D038008E460546DFF8A092114699F8B04400687C
:10D04800164698467246631C89F8B034FEF740F9D4
:10D058002B8901A9ADF8043018238DF806306868CB
:10D0680002238DF80730FFF7EDFEAB7A09F2B447DB
:10D07800240127442A6849460C2B00F2F680DFE891
:10D0880013F00D00F400F400F4005100F400F40073
:10D09800F4008A00F400F400F400C200138CDFF8F6
:10D0A8003CC223F001031B041B0C1384138CB2F83D
:10D0B80004E0108B624520F073004FEA00404FEA0D
:10D0C80010409BB21FFA8EFE40F0700014D00CF591
:10D0D800006C624510D00CF5406C62450CD00CF524
:10D0E800806C624508D00CF5806C624504D023F052
:10D0F800020343F0030307E023F00E032EF4407EFF
:10D1080043F003034EF4807EA2F804E01083A2F8F3
:10D1180034801384138B23F008031B041B0C43F087
:10D12800080336E0138CDFF8B4C123F010031B04A6
:10D138001B0C1384138CB2F804E0108B624520F4A6
:10D14800E6404FEA00404FEA10409BB21FFA8EFEBD
:10D1580040F4E04008D00CF5006C624504D023F0A0
:10D16800200343F0300307E023F0E0032EF4406E81
:10D1780043F030034EF4806EA2F804E01083A2F866
:10D1880038801384138B23F400631B041B0C43F4B3
:10D198000063138369E0138CDFF840C123F48073C4
:10D1A8001B041B0C1384138CB2F804E0908B6245AB
:10D1B80020F073004FEA00404FEA10409BB21FFA7C
:10D1C8008EFE40F0700008D00CF5006C624504D06B
:10D1D80023F4007343F4407307E023F460632EF4F0
:10D1E800405E43F440734EF4805EA2F804E09083FE
:10D1F800A2F83C801384938B23F008031B041B0CB8
:10D2080043F0080330E0138CDFF8D0C023F48053D8
:10D218001B041B0C1384108CB2F804E0938B20F4CD
:10D22800005023F4E6431B0400041B0C000C624569
:10D238001FFA8EFE43F4E04340F4405003D00CF54F
:10D24800006C624503D12EF4804E4EF4804EA2F855
:10D2580004E09383A2F840801084938B23F4006346
:10D268001B041B0C43F4006393832B7B43B1B2F87C
:10D2780044306FEA43436FEA53439BB2A2F8443009
:10D2880013889BB243F001031380AB7A0C2B19D897
:10D29800DFE803F0071818180B1818180F181818D3
:10D2A80013000B1902F134000AE00B1902F13800DF
:10D2B80006E00B1902F13C0002E00B1902F14000F4
:10D2C800C3F8B40438460C44A4F8BC64C4F8B824C1
:10D2D80003B0BDE8F08300BF9C210020002C014072
:10D2E80010B5D420FEF7B1FA8020FEF7AEFAA820D8
:10D2F800FEF7ABFA3F20FEF7A8FAD320FEF7A5FA0F
:10D308000020FEF7A2FA4020FEF79FFA8D20FEF7D4
:10D318009CFA1420FEF799FAA120FEF796FAC82085
:10D32800FEF793FADA20FEF790FA1220FEF78DFA4C
:10D338008120FEF78AFACF20FEF787FAD920FEF778
:10D3480084FAF120FEF781FADB20FEF77EFA40200E
:10D35800FEF77BFAA420FEF778FAA620FEF775FA06
:10D36800AF20FEF772FAA620FEF76FFAAE20FEF79E
:10D378006CFA2020FEF769FA0020FEF766FAB02062
:10D38800FEF763FA4020FEF760FA0020FEF75DFA28
:10D398001020FEF75AFA4FF48064013C0020A4B232
:10D3A800FEF74EFA002CF8D18120FEF74EFAC8207D
:10D3B800FEF74BFAAF20FEF748FA012010BD70B512
:10D3C80000EB8000094CA0F1A1059C3825440444D9
:10D3D800074B15F8010F1E787040FEF731FAA54289
:10D3E800F6D13046BDE87040FEF72ABAC09D010864
:10D3F800E930002010B5441E14F8010F10B1FFF7F2
:10D40800DEFFF9E710BD08B55038C0B2FEF71DFAC7
:10D418000020FEF71AFABDE808401020FEF715BAFA
:10D4280010B504465039C8B2FEF70FFA04EB4400B1
:10D43800400000F00E00FEF708FA06206043BDE841
:10D448001040C0F303101030FEF7FFB90028114A4E
:10D45800B8BF404290FBF2F330B50F4C3C2504FBBB
:10D46800030068430D4D90FBF2F22D682D7B25B922
:10D4780003EB830303EB830301E0C3EB031302EB2A
:10D48800830304FB02020B804FF47A7392FBF3F2DE
:10D498004A8030BD80969800806967FFB8190020DF
:10D4A800022803D0431E584258417047064B1B6858
:10D4B8001B7823B1054B1868C0F3C0407047044B74
:10D4C8001878C0F380007047F0050020E8100020AD
:10D4D800E730002010B50A4C5E280146206805D1C7
:10D4E8005D2102F0FCFD20683E2105E05D2903D1A5
:10D4F80002F0F5FD20683D21BDE8104002F0EFBDC7
:10D508001027002010B50446C0B2FFF7E3FFC4F3AC
:10D518000720BDE81040DDE7024B5E21186802F0E5
:10D52800DEBD00BF1027002038B50546054C5E213A
:10D53800206802F0D4FD20682946BDE8384002F092
:10D54800CEBD00BF1027002013B5044601A900680E
:10D55800FFF77CFF1320FFF7E7FFBDF90400FFF793
:10D56800D1FF1B20FFF7E0FFBDF90600FFF7CAFF58
:10D578002320FFF7D9FF2368002BB4BF53204E2088
:10D58800FFF7C0FF01A96068FFF760FF1220FFF7EF
:10D59800CBFFBDF90400FFF7B5FF1A20FFF7C4FF62
:10D5A800BDF90600FFF7AEFF2220FFF7BDFF636855
:10D5B800002BB4BF57204520FFF7A4FF02B010BDD1
:10D5C800674B73B51878FFF76BFF664D04462B78E9
:10D5D800834220D0C8B1644B1B68E3B193F90000C3
:10D5E80002230093614B04211B6800225B780033FF
:10D5F80018BF012301934FF41653FAF7D0FD5C4B83
:10D60800186040B101232B7005E0594E3068FAF7D5
:10D6180025FB34602C70574B574D1878FFF740FFA7
:10D628002B780446834218D088B1544B1B68A3B1A9
:10D638000022012493F9000008214FF49643009436
:10D648000192FAF7ACFD4E4B186028B905E04C4E34
:10D658003068FAF703FB34602C704A4B4A4D18784F
:10D66800FFF71EFF2B78044683422E4643D000283E
:10D6780038D0464B1A68002A3DD0D37992F9000079
:10D68800002B4FF00202424C08BF022300920022F6
:10D6980054F8233001921021FAF781FD3D4B0546DD
:10D6A800186040B33C4C94F84A30022B0BD094F8E5
:10D6B8009620022A01D14C3405E023B1002A04F156
:10D6C8004C0418BF0024354B1C6044B1204600218F
:10D6D8004C2209F00CFA0223256084F84A30012311
:10D6E800337008E02B4E306803F078FE3068FAF7A4
:10D6F800B5FA34602C702A4B2A4D1878FFF7D0FE03
:10D708002B780446834229D000B3274B1B682BB3E0
:10D71800264A93F900001268032352782021002A30
:10D728000CBF08220922009301924FF461430022A2
:10D73800FAF735FD1E4B186080B11E4A012313709D
:10D748002B701D4B1A681D4B1A6007E0184E306885
:10D75800FAF784FA174B34601C702C7002B070BD55
:10D76800F8050020AC110020F4050020B8190020AD
:10D7780010270020F9050020D81900205C1A002085
:10D788004C1A002004060020621A0020000600201F
:10D7980088A00108641A002018280020681A0020B0
:10D7A80010060020781A00200C0600200806002029
:10D7B8007C1A0020801A0020202D0020841A0020C6
:10D7C800642928BF6421F8B501FB00F5642495FBA2
:10D7D800F4F40646E4B20027FBB2A34204D29F2029
:10D7E800FFF7EDFD0137F7E7B4420BD2142195FBA3
:10D7F800F1F5C4EB8410663DC4EB80002844C0B248
:10D80800FFF7DDFD0134E4B2B44201D29A20F7E714
:10D81800F8BD2DE9F743FAF73BFC924C6368C31A4D
:10D82800002BC0F2688300F5433303F5A0736360EF
:10D838008D4B1D78237AC5F38005EB1A18BF012399
:10D8480025724DB1002B00F05683884B5A789A7098
:10D8580001225A701A702BE0844A2BB1D37843F016
:10D868000203D37093785370D67806F0020101F062
:10D87800FF0339B97D498968411A002903DB06F09D
:10D88800010300E0012303F00107784917707BB119
:10D89800F2070DD50A7905230132D2B2B2FBF3F3B0
:10D8A80003EB8303D31A724ADBB20B71D35C4B7060
:10D8B8006E4EDFF8088233787BB3F37823F00203E7
:10D8C800F3706C4B0344AE20B360FDF7BEFF08B1A4
:10D8D800FFF706FD88F80000002800F00C83B02050
:10D8E800FDF7B3FF4020FDF7B0FF0020FDF7ADFFC7
:10D8F8001020FDF7AAFF4FF48067013F0020BFB258
:10D90800FDF79EFF002FF8D13846FFF77CFD7278AF
:10D91800594B53F82200FFF76DFD98F80030002BA3
:10D9280000F0E9827378062B00F2B282DFE813F088
:10D938000700B002180078006A018701EC014F491E
:10D948004F4A504B5048FCF782FB0120FFF75BFD24
:10D958004D48FFF74FFD0220FFF755FD4B48ACE15E
:10D968004B4F3B689B0735D5DFF854810A23B8F83D
:10D978000010DFF85091B1FBF3F203FB121399F892
:10D98800001092B29BB200913F484249FCF75FFBFE
:10D99800FEF7D6F90120FFF736FD3B48FFF72AFDD1
:10D9A8003D4B99F800201868B8F80030067902FB5A
:10D9B800163164234B43C17802208E1B5643B3FBB8
:10D9C800F6F6F6B2FFF71FFD31461520FFF7F8FE11
:10D9D800032600E001263B681F0540F159822F4BC2
:10D9E8002F491F68642397FBF3F2096803FB12733E
:10D9F800009125482B49FCF72AFBFEF7A1F9304690
:10DA0800FFF701FD2048FFF7F5FC01F0DFFE0746B0
:10DA1800701CFFF7F8FC15203946FFF7D1FE37E2F6
:10DA28000120214FFFF7EFFC2048FFF7E3FC3B689C
:10DA3800980749D51E4A1448B2F90210B2F90030C5
:10DA48000091B2F904201B4901921B4AFCF7FFFA26
:10DA5800FEF776F90220FFF7D6FC0B48FFF7CAFC61
:10DA6800032632E010270020E7300020D41A0020D7
:10DA7800BDBF0108404B4C0064A00108C2BF0108AB
:10DA8800CBBF0108D1B5010819270020D2BF010872
:10DA9800FC2C0020E0BF0108B0190020BC190020B0
:10DAA800C0190020F8BF0108C41900200DC00108E2
:10DAB800B611002023C0010832C001083D02002031
:10DAC800B41900204400002002263B68D9071AD563
:10DAD8007B4A7C48B2F90210B2F900300091B2F9E1
:10DAE800042079490192794AFCF7B1FA06F1010854
:10DAF800FEF726F93046FFF786FC5FFA88F871488A
:10DB0800FFF778FC46463B681A0718D5704A6D48F7
:10DB1800B2F90210B2F900300091B2F904206A4952
:10DB280001926C4AFCF793FA771CFEF709F9304624
:10DB3800FFF769FCFFB26348FFF75CFC3E46664AA4
:10DB48006149B2F90030B2F902205E480092634A96
:10DB5800DFF8B091B2F90020771C0192604AFCF717
:10DB680076FAFEF7EDF83046FFF74DFC5548FFF71B
:10DB780041FC5449D9F80000FCF704F9514808F071
:10DB8800FAFFFFB2C1B2092909D84B1CDBB2214404
:10DB980020224A720021E21891721946F3E7DFF851
:10DBA8002481D9F804004144FCF7ECF8FEF7C8F8E2
:10DBB8003846FFF728FC4046FFF71CFC4146D9F8D9
:10DBC8000800FCF7DFF8404608F0D5FF0236F6B249
:10DBD800C7B2092F09D87B1CDBB2274420227A72EE
:10DBE8000021E21891721F46F3E73E4BB3F900009B
:10DBF80005F0C8F908EB0701FCF7C4F8FEF7A0F830
:10DC0800304657E00026384F3B78B34240F2408117
:10DC18000E2E00F03D8170080130FFF7F4FB30460E
:10DC280004F0D8FC3B78B34206D92020FFF7C7FBA5
:10DC3800701CC0B204F0CEFC0236F6B2E3E72B4EFD
:10DC48002B4996F8B0271F48FCF701FA0120FFF787
:10DC5800DAFB1C48FFF7CEFB264B27491F781948EB
:10DC68003A46FCF7F4F90220FFF7CDFB1548FFF719
:10DC7800C1FB0C2303FB0766204996F8B32796F8E7
:10DC8800B2371048FCF7E3F9FEF75AF80320FFF71C
:10DC9800BAFB0C48FFF7AEFB96F8B81796F8B6270C
:10DCA80096F8B737074800911549FCF7D0F9FEF701
:10DCB80047F80420FFF7A7FB0248FFF79BFBE7E0C4
:10DCC800081100201927002023C0010836C00108C8
:10DCD8000E11002081CF0108F42C0020C41100206F
:10DCE8003AC001086C080020B4280020D411002094
:10DCF8003EC00108A82C00204AC001085BC00108EA
:10DD08006CC00108600800207C4B1B681B0640F1B2
:10DD1800BB80236A616A7A4A8B421CBF536292F8BD
:10DD280028304FF001011CBF013303F003034FF00B
:10DD3800000018BF82F82830FFF772FB94F82830EB
:10DD4800704A0026D05CFFF73AFB02200121FFF75A
:10DD580067FB6D4B3620F35C0136C3EBC30393FBC3
:10DD6800F0F0C0B2062828BF06206038C0B2FFF71E
:10DD780026FB102EEDD1654B65491B78654813F0DD
:10DD8800020F654B1A7814BF59234E23FCF75FF92D
:10DD9800FDF7D6FF0220FFF736FB5E48FFF72AFBA8
:10DDA8005E495F4B4E680A685A4892FBF3F25D4938
:10DDB80096FBF3F3FCF74BF9FDF7C2FF0320FFF7DF
:10DDC80022FB5448FFF716FB574B58491A8851480D
:10DDD800FCF73DF9FDF7A0FF0420FFF714FB4D48C1
:10DDE800FFF708FB524B53491A884A48FCF72FF9AA
:10DDF800FDF792FF04210A20FFF712FB4548FFF7C1
:10DE0800F9FA4D49E26A4348FCF721F94B4EFDF710
:10DE180083FF0520FFF7F7FA3E48FFF7EBFA726831
:10DE2800B36847493B48FCF712F9FDF775FF052130
:10DE38000A20FFF7F5FA3748FFF7DCFA3369F2688A
:10DE48004049D21A3348FCF702F9FDF765FF06206E
:10DE5800FFF7D9FA2F48FFF7CDFAB2683A492D48AB
:10DE6800FCF7F5F8FDF758FF06210A20FFF7D8FA66
:10DE78002848FFF7BFFA35491522264808F0A6FEBC
:10DE8800FDF74AFF072015E7F37843F00203F37024
:10DE9800002D30D12E4B002193F820301220052B75
:10DEA80097BF2C4A3F259B181D7FFFF7B9FA2846D4
:10DEB800FFF785FA13200021FFF7B2FA264B1B78EB
:10DEC800002B264B18BF72201B7808BF2120002B7F
:10DED80018BF5220FFF773FA14200021FFF7A0FAA9
:10DEE80094F83050074B585D013505F00305FFF7EE
:10DEF80066FA84F8305003B0BDE8F083FC2C0020AB
:10DF0800102700207EC0010899110020C8190020A0
:10DF180083C0010819270020CE190020D01900203D
:10DF28008096980094C00108CA190020A1C0010871
:10DF380050110020A9C00108B0C001089C070020AA
:10DF4800B7C00108C0C00108C7C00108B00200205E
:10DF58009430002064A00108230F0020880F0020BF
:10DF6800064B1B7803F0040303F0FF001BB1044BBE
:10DF78001888C0F3C01000F001007047E730002097
:10DF88008C1A00202DE9F04F89B00593BE4B00266E
:10DF9800B3F90290B3F90030B9F1000FB8BFC9F175
:10DFA8000009002BB8BF5B429945B8BF9946804627
:10DFB800B2463446B9F5FA7F04910392A8BF4FF4EC
:10DFC800FA79019000960296B04D2B88990754D0A3
:10DFD800AD4B610033F91420AD4B33F9143003EB2A
:10DFE8004202039B5B429A4203DB039B9342A8BF16
:10DFF8001346A84A8F5E059ADB1B32F914001F18D6
:10E00800FFF7AEFF90B1A44B384613F804A004F014
:10E01800B9FFA24905F0BEF80146504604F0E2F8FF
:10E028009E4905F003F805F0C7F9074698F8083047
:10E0380064227B4393FBF2F398F81C206FF0040AE8
:10E048000AFB02FA534504DB02EB820A9A45A8BF91
:10E058009A4642F21072924B53F824003844904288
:10E06800A8BF10468F4A9042B8BF104643F8240014
:10E0780098F812305843031302932D8805F00303D0
:10E08800012B38D0804B884933F91430A60000930F
:10E09800019B51F8247093F801E0844B33F9140084
:10E0A80080EAE073A3EBE073B3F5206F16DC009A07
:10E0B80050235A4392FBFEF3042290FBF2F0181A05
:10E0C8000744B7F57A5F7A4BA8BF4FF47A579F4257
:10E0D800ACBF41F8247041F8243002E0002341F835
:10E0E80024308B597D2693FBF6F6019BDB7A73432C
:10E0F800402693FBF6F6AA0712D5009A09FB06F507
:10E1080009FB02F70298C9F5FA7303FB0A7703FBC8
:10E1180000534FF4FA7297FBF2F193FBF2F505E026
:10E12800EB0755BF354651460099029D5F4B0427C2
:10E1380033F914305F4A93FBF7F3A25C6FF04F0793
:10E14800534393FBF7F398F851204FEA440BCF1849
:10E1580072B13846069204F015FF5749574B01EB48
:10E16800C401069A1B68FBF747FD05F025F9074629
:10E178004E4B534A3BF803003BF9021003B25B1ABB
:10E18800042193FBF1F102F1040E5EF824302BF820
:10E1980002000C3252F8240042F8243098F850203B
:10E1A80018444FEA840C08444EF8241082B1CDF884
:10E1B8001CC0069204F0E6FE4249404B01EBC40144
:10E1C800069A1B68FBF718FD05F0F6F8DDF81CC089
:10E1D8003D4BDFF810E11B5D7A195843202390FB73
:10E1E800F3F3D21A2BF80E20384A5B424CF802306F
:10E1F800019B3748374901334CF801504CF80070FF
:10E20800019375460CB90124DEE61F4B0427B3F9C8
:10E218000440049B244E9B79D6F808E00F335B003A
:10E228006343224C5B11B4F90440002B94FBF7F7CD
:10E23800A3EB0707B8BF5B42322B98F80D400BDC05
:10E2480004FB07E4244BA342A8BF2346234CA34264
:10E25800ACBFB360B46001E00023B36098F803403A
:10E2680004FB07F31E4C9B112478032C3DD9B8F806
:10E278004E40B4F5FA7F38D26742BB4234DBA34242
:10E28800A8BF234631E000BFCC1100208C1A002023
:10E29800E0300020F42C0020BCA001080000204140
:10E2A80044270020F0D8FFFFE029002008110020B3
:10E2B80080C1FFFF682A0020C4290020DC29002033
:10E2C8004C270020102A00207C2A0020482A002001
:10E2D800302A00203C2A0020FEFFFF0F020000F039
:10E2E8007F2A0020282A00203B46B4686FF0FF06EA
:10E2F80044F34F34B4F5807FA8BF4FF48074B44220
:10E30800B8BF344683601E190023AE808C609360CA
:10E3180009B0BDE8F08F2DE9F04F87B00393B44BF7
:10E3280081461D88029105F00205ADB2019295B1B2
:10E33800B04BB3F90250B3F90030002DB8BF6D42AD
:10E34800002BB8BF5B429D42B8BF1D46B5F5007FA4
:10E35800A8BF4FF40075CB460026A64BA64933F953
:10E368001620A64B4FEA460A33F91630520083EAC4
:10E37800E374A4EBE374B4F5206F4FEA860851F810
:10E38800260011DC042493FBF4F3D31A0344B3F5F9
:10E398007A5F9B48A8BF4FF47A538342ACBF41F8D9
:10E3A800263041F8260002E0002341F8263051F8D3
:10E3B80008709BF80B30FF119BF801405F438C4BB2
:10E3C80054431B88BF119B074FEAA41456D08D4BAA
:10E3D8003AF903301A44019B5B429A4203DB019BE2
:10E3E8009342A8BF1346884A3AF902209B1A039A17
:10E3F80032F916201A440492FFF7B2FD049A98B134
:10E40800824B10469B5D049304F0BCFD804904F0E8
:10E41800C1FE049B0146184603F0E4FE7C4904F063
:10E4280005FE04F0C9FF024642F21070794958F817
:10E43800013013448342A8BF034677488342B8BFDC
:10E44800034648F8013099F8081099F81C004A4327
:10E4580000EB8000D21141428A4203DB8242A8BF0E
:10E468000246114699F81220641A53431B13FF1AE7
:10E478006F436C4303EB672701EB64245F4B042273
:10E488003AF9033093FBF2F2644B9B5D534399F8DE
:10E498005120A4EBA31472B12046049204F072FD3B
:10E4A8005F49604B01EBC601049A1B68FBF7A4FBAC
:10E4B80004F082FF044651495B4B3AF801003AF9EF
:10E4C80003E002B2CEEB02024FF0040E92FBFEF222
:10E4D8002AF803009E440C3358F80EC058F803007D
:10E4E80048F80E206044104499F8502048F803C0BA
:10E4F8008C467AB10591049204F044FD4B49494B8E
:10E5080001EBC601049A1B68FBF776FB04F054FF85
:10E51800DDF814C0464BDFF834E19B5DE219434354
:10E528005B11D21A2AF80E2042484349434A5B42FB
:10E5380048F8004048F8017048F802300BF1010B28
:10E5480074460EB9012608E72A4B0427B3F904508C
:10E55800029B294E9B79D6F808E00F335B006B438A
:10E56800BCF904505B1195FBF7F7002BA3EB0707E9
:10E57800B8BF5B42322B99F80D500BDC05FB07E561
:10E588002F4BAB42A8BF2B462E4DAB42ACBFB3605E
:10E59800B56001E00023B36099F8035005FB07F369
:10E5A800294D9B112D78032D0CD9B9F84E50B5F58E
:10E5B800FA7F07D26F42BB4203DBAB42A8BF2B46B0
:10E5C80000E03B46B5686FF0FF0645F34F35B5F5FB
:10E5D800807FA8BF4FF48075B542B8BF35468360C9
:10E5E8005E190023A6808D60936007B0BDE8F08FA8
:10E5F8008C1A0020CC110020E029002008110020EE
:10E6080080C1FFFFE0300020F42C0020BCA00108EE
:10E618000000204144270020F0D8FFFF682A00208E
:10E62800C4290020DC29002060270020102A0020AF
:10E638007C2A0020302A00203C2A0020482A00207A
:10E64800FEFFFF0F020000F07F2A0020282A00208A
:10E658002DE9F04F89B00593AE4B0027B3F902803E
:10E66800B3F90030B8F1000FB8BFC8F10008002BAB
:10E67800B8BF5B429845B8BF98468246B946BB4684
:10E688003C46B8F5FA7F0492A8BF4FF4FA78029096
:10E698000397A14D2B88990757D0022C55D09D4B35
:10E6A800610033F914209D4B33F9143003EB420217
:10E6B800049B5B429A4203DB049B9342A8BF134628
:10E6C800974A8E5E059A9B1B32F914001E18FFF7B5
:10E6D80047FC90B1934B304613F804B004F052FC59
:10E6E800914904F057FD0146584603F07BFD8E49D9
:10E6F80004F09CFC04F060FE06469AF80830642298
:10E70800734393FBF2F39AF81C206FF0040101FBAA
:10E7180002FB5B4505DB02EB82029342A8BF13466E
:10E728009B4642F21072814B53F8240030449042C9
:10E73800A8BF10467E4A9042B8BF104643F824004E
:10E748009AF81230584303130393298801F00303FE
:10E75800012B01D1022C3DD16E4B764D33F914902B
:10E76800029BA00093F801E0734B55F8247033F92D
:10E77800146086EAE673A3EBE673B3F5206F1CDC3E
:10E78800022C14D0502303FB09F292FBFEF304225F
:10E7980096FBF2F69E1B3744B7F57A5F674BA8BF26
:10E7A8004FF47A579F42ACBF2F502B5007E089EAAD
:10E7B800E973A3EBE973642BE4DD00232B505D4B75
:10E7C8007D27C35893FBF7F7029BDB7A7B434027EF
:10E7D80093FBF7F78A0713D5022C11D008FB07F52E
:10E7E80008FB09F60398C8F5FA7303FB0B6603FBED
:10E7F80000534FF4FA7296FBF2F193FBF2F508E03E
:10E80800CB0704D5022C02D0039D594601E03D46B2
:10E81800494663000193484B042633F91430484AAB
:10E8280093FBF6F3A25C6FF04F06534393FBF6F3AA
:10E838009AF85120CE18E2B1022C069230460BD13C
:10E8480004F0A0FB069A530803D09A42A8BF1A46C0
:10E8580000E001223B4905E004F094FB3A49069A9E
:10E8680001EBC401394B1B68FBF7C6F904F0A4FDA2
:10E878000646314B019A0198D15A354B0AB2C05E0F
:10E888004FEA840C121A042092FBF0F20198C1524C
:10E8980003F10801143351F824E053F8240041F837
:10E8A8002420704410449AF8502043F824E082B1A0
:10E8B800CDF81CC0069204F065FB2649234B01EBFA
:10E8C800C401069A1B68FBF797F904F075FDDDF89B
:10E8D8001CC0214B214A1B5D01995843202390FB02
:10E8E800F3F073191B1A8B521D4B40424CF803600E
:10E8F8001C4B01344CF803501B4B032C4CF8030001
:10E90800029B03F1010302937FF4C3AE09B0BDE893
:10E91800F08F00BFCC1100208C1A0020E0300020BE
:10E92800F42C0020BCA0010800002041442700204E
:10E93800F0D8FFFFE02900200811002080C1FFFF68
:10E94800682A0020D4290020C4290020DC290020BE
:10E9580074270020102A00207C2A0020282A002062
:10E96800302A00203C2A0020482A00202DE9F04FB8
:10E9780089B005939D4B80461B880C469B070292E5
:10E988004DD540F2E631129B994AD889B2F9003048
:10E998001B1A03F2F3158D4203D8002BB8BF5B4254
:10E9A80001E04FF4FA73B2F90220101A40F2E6328D
:10E9B80000F2F311914203D80028B8BF404201E0A9
:10E9C8004FF4FA7098F84C503DB39842B8BF1846C7
:10E9D800C0F5FA7004F0D6FA864904F0DBFB4FF074
:10E9E8007E5104F019FA0646642090FBF5F004F015
:10E9F800C9FA0146304604F019FB4FF07E5104F085
:10EA08000DFA0021074604F0AFFC30B938464FF044
:10EA18007E5104F0C7FC20B101E0002701E04FF06F
:10EA28007E57E31C0393CDF800800024039B022C3F
:10EA380013F8015F704E039309D1B6F904000A3543
:10EA4800684304F09FFA6D4904F0A4FB74E036F9BA
:10EA5800140004F097FA8146029804F08FFA654989
:10EA680004F098FB0146484604F0E0FA644B8146FE
:10EA780033F9140004F086FA0146484604F0CEF94A
:10EA8800029B8146584204F07DFA8346484659461F
:10EA98004FEA440A04F068FC48B9029804F072FA94
:10EAA80083464846594604F07DFC00B9CB46554B91
:10EAB80033F90A0004F066FA0146584604F0ACF946
:10EAC800059B814633F9140004F05CFA0146484678
:10EAD80004F0A4F94C4904F05DFB8146FFF740FAC5
:10EAE80028B14A4B4946185D03F07CFB81463F4BF1
:10EAF800B3F800B01BF0010F05D04846D8F8441011
:10EB080004F094FA18E036F90A001435684304F062
:10EB180039FA3A4904F03EFB1BF0020F05460CD0C7
:10EB2800D8F84810484604F081FA394604F07EFACD
:10EB38000146284604F072F9054663000493344BF5
:10EB4800344E33F9140004F01DFA334B196E04F0F7
:10EB58006DFA0146284604F05FF9009B8246196A5F
:10EB680004F064FA2D4B0546185D04F00BFA0146D3
:10EB7800284604F05BFA2A4904F00CFB98F8512067
:10EB8800814692B1022C09D1530803D09A42A8BFFA
:10EB98001A4600E001224846224902E0224901EBD8
:10EBA800C4013368FBF728F8814633685046194694
:10EBB800019304F03BFA009BDFF878B0D96A04F0BF
:10EBC80035FA114904F032FA5BF8241004F026F9FA
:10EBD8001649A500064604F0C7FB68BB3046144931
:10EBE80004F0E0FB48B3124E27E000BF8C1A002067
:10EBF800382D00200000FA43CC11002000004842C4
:10EC0800E0300020F42C002000002041BCA00108C6
:10EC180008110020DC29002044270020C0290020FA
:10EC28000000C842D4290020C429002000007AC36B
:10EC380000007A435C2A0020444E4BF80560DFF858
:10EC48003CB1504655F80B1004F0E6F845F80BA017
:10EC5800069001994FF07E5004F09CFA069B0146FD
:10EC6800184604F0E3F982460BF10C03EA580BF15D
:10EC7800180B104655F80B100793069204F0CEF8BF
:10EC8800514604F0CBF8069A079B45F80B2098F8F4
:10EC98005020014645F803A032B12D49019B01EBF4
:10ECA800C401FAF7A9FF014608462A4904F072FA96
:10ECB800009B996B04F0BAF9274B8246185D04F063
:10ECC80061F90146504604F0B1F9244904F062FAAA
:10ECD8002349824604F048FB38B95046214904F0DC
:10ECE80061FB20B1DFF87CA001E0DFF874A03146B9
:10ECF800484604F093F8514604F090F808F004F9F7
:10ED0800194BB0F57A7FA8BF4FF47A709842B8BF14
:10ED18001846049A154B0134D052484604F04CFB6F
:10ED2800134B5851304604F047FB124B585150468C
:10ED380004F042FB104B032C5851009B03F10403D1
:10ED480000937FF473AE09B0BDE8F08F00007AC37A
:10ED5800102A002000004040C02900200000C842BE
:10ED6800000096C30000964318FCFFFF282A0020E5
:10ED7800302A00203C2A0020482A0020A82700200A
:10ED8800044B00221A605A60034B00221A605A6032
:10ED9800704700BF44270020542A002010B50C4CAF
:10EDA8000123E3704FF48060022384F82030FBF7DE
:10EDB800E7FA084A084BD2F888201B685278642181
:10EDC80001FB0233636123880133238010BD00BF38
:10EDD8009430002044270020202D0020084BDA68BA
:10EDE800D10709D4DA68520708D4DB6813F0100F8A
:10EDF80014BF032004207047012070470220704789
:10EE080000200240704701207047704703788B420A
:10EE180086BF024B33F8110000207047D02700202E
:10EE280008B50021062207F062FE012008BD08B5DA
:10EE38000021062207F05BFE012008BD70B50546DB
:10EE4800F9F726F9324CA369A061C31AB3F5FA5F42
:10EE5800E36182BF002384F8203084F8213094F8DD
:10EE680020302BB9A12D02BF294A012182F8211097
:10EE780094F82110264A31B1D118EDB2013381F846
:10EE8800225082F8203094F8205094F84330AB4256
:10EE98003CD11F4B93F84430052B02D0062B03D0EE
:10EEA8002FE0002003F0C8FE94F823301E2B28D151
:10EEB80000200246C1B26B1E99421ADA214491F829
:10EEC80022300821DBB283EA0206F60744BF83F04A
:10EED8001803C3F3460301F1FF3154BF5B0843F045
:10EEE800800311F0FF01C2F34702ECD101301A464A
:10EEF800E0E7234493F822309A4202D1032003F03A
:10EF08009BFE002384F8213084F8203070BD00BFB8
:10EF1800D027002010B50446B0F9000003F0E8F847
:10EF2800B4F9020003F0E4F8B4F90400BDE81040B5
:10EF380003F0DEB810B50446006803F0D9F860683D
:10EF480003F0D6F8A068BDE8104003F0D1B82DE969
:10EF5800F74F0120F8F770FF002488B3012C2FD851
:10EF68004FF04C0909FB04FA174E06EB0A0808F1A2
:10EF78009007BD7815B10134E4B2EEE790F900309E
:10EF880090F804E01846114B03228DE82400012173
:10EF98002A4653F82E30F9F702F9834660B106F194
:10EFA8004800504429464A4607F0A1FD01231C4465
:10EFB800C8F848B0BB70E4B20120F8F723FFCCE7EB
:10EFC80003B0BDE8F08F00BFD027002088A001085B
:10EFD8000021222210B5104807F089FD0F4B0022AE
:10EFE80019460F480424105C013283F8F60183F8AF
:10EFF800FB4105200024042A83F8FA0183F8FD4127
:10F0080083F8FC0103F10803EBD10123A1F8F831DF
:10F01800522381F8F43110BDC8130020D411002008
:10F02800FCC0010870B50646441E14F8011F89B1DA
:10F03800094D284607F091FD0028F6D005F1080390
:10F0480098423FBF054B401BC018A31B38BF80F830
:10F058008A31EAE770BD00BF8ECF0108D4110020C5
:10F0680007B51C4B03F1E402C3F8E0201A4A92F8F2
:10F0780092215AB1012A14D1032183F8E6100721FD
:10F0880083F8E82083F8E7100C2208E0022183F8CF
:10F09800E610032183F8E82083F8E710072283F8B5
:10F0A800E4200E4A0E4B40201A60F8F7C5FE70B1F6
:10F0B8000122002390F9000040218DE80C00094A44
:10F0C8004FF4E133F9F76BF8003018BF012003B0B3
:10F0D8005DF804FBD0270020D4110020FD29010889
:10F0E80030000020AD2A01080120002102F0C4B937
:10F0F800174AF0B5164692F8E930D2F8ECE0032B3F
:10F1080010D85C1C0EEBC3039D1CE4B208D09A888F
:10F11800D10705D5104203D008E00131042907D1F1
:10F128002346ECE786F8E9300020F0BD9F780021FF
:10F138000C2202FB01F3064D05F1F00C1CF803202C
:10F148009742EAD12B4485F8E940D3F8F400F0BDA2
:10F15800D02700208A6810B50C6A036814430A692E
:10F1680023F4FF4314434A6923F0700314438A6964
:10F178001443CA6914434A6A14438A6A22431343EC
:10F188000360CB6843600B6883604B68C36010BD45
:10F198004FF6FE7302681340036000230360436068
:10F1A8008360C360284B984201D1284A27E0284B46
:10F1B800984201D1254A2AE0264B984201D1234A98
:10F1C8002DE0254B984201D1204A30E0234B98424C
:10F1D80001D11E4A33E0224B984204D11B4A53689E
:10F1E80043F470032EE01F4B984204D1174A53682A
:10F1F80043F0706326E01C4B984204D11B4A5368C5
:10F2080043F00F031EE01A4B984204D1174A536883
:10F2180043F0F00316E0174B984204D1134A5368A1
:10F2280043F470630EE0144B984204D10F4A5368BC
:10F2380043F4704306E0114B984204D10B4A5368DB
:10F2480043F47023536070470800024000000240F6
:10F258001C000240300002404400024058000240B6
:10F268006C00024080000240080402400004024092
:10F278001C04024030040240440402405804024086
:10F28800224A10B5536803F00C03042B03D0082B53
:10F2980004D01F4B14E01F4B5B6811E053685168A2
:10F2A800C3F38343C90303F1020301D41A4906E0F7
:10F2B800516811F4003F1749496818BF49084B4382
:10F2C80003605368154CC3F30313234493F82010C9
:10F2D8000368CB4043605168C1F30221214491F88F
:10F2E800201023FA01F181605168C1F3C221214441
:10F2F80091F82010CB40C3605268C2F38132224497
:10F3080092F83020B3FBF2F3036110BD0010024005
:10F3180000127A003000002000093D0088A0010892
:10F3280010B50446FFF75AFD012806D11CB1FFF7B6
:10F3380055FD013CF8E7052010BD002C08BF05204D
:10F3480010BD0A88F0B54B888E88B1F808E0CC88E3
:10F35800002A3AD1028C43F0010322F00102120480
:10F36800120C0284058B078CADB225F0F30545EA33
:10F378000E1189B241EA06027A49BFB2884212D018
:10F3880001F5006188420ED0B0F1804F0BD0A1F595
:10F398009831884207D001F58061884203D001F591
:10F3A8008061884202D127F0020701E027F00A07AE
:10F3B8001F4302830784038B23F00C031B041B0CDD
:10F3C8000383038B9BB21C4344E0042A44D1028C80
:10F3D80022F010021204120C0284018B058C21F415
:10F3E80040721205120D42EA0E325E4992B242EAAA
:10F3F80006228842ADB292B212D001F5006188426D
:10F408000ED0B0F1804F0BD0A1F59831884207D0CB
:10F4180001F58061884203D001F58061884207D1F7
:10F4280025F0200141EA03139BB243F0100304E0E6
:10F4380025F0A00143F010030B4302830384038BE0
:10F4480023F440631B041B0C0383038B9BB243EA26
:10F458000424A4B20483F0BD082A028C3ED122F40D
:10F4680080721204120C0284828B3E4D92B222F0FA
:10F47800F307018C47EA0E1292B2A84289B242EA17
:10F48800060212D005F50065A8420ED0B0F1804FF3
:10F498000BD0A5F59835A84207D005F58065A84298
:10F4A80003D005F58065A84207D121F4007141EA2F
:10F4B80003239BB243F4807304E021F4206143F4F6
:10F4C80080730B4382830384838B23F00C031B0418
:10F4D8001B0C8383838B9BB21C4341E022F4805234
:10F4E8001204120C0284858B018C25F440752D05BD
:10F4F8002D0D45EA062545EA0E321A4D89B2A84275
:10F5080092B212D005F50065A8420ED0B0F1804F36
:10F518000BD0A5F59835A84207D005F58065A84217
:10F5280003D005F58065A84207D121F4005141EACE
:10F5380003339BB243F4805305E047F6FF5543F489
:10F5480080530D402B4382830384838B23F44063D1
:10F558001B041B0C8383838B9BB243EA0424A4B251
:10F568008483F0BD002C0140CA78F0B5D40648BFAA
:10F578008C780D8802F00F0348BF234315F0FF0F66
:10F588001DD0016800240126A64006EA0507B742F7
:10F5980011D14FEA840E0F2606FA0EF621EA06016B
:10F5A800282A03FA0EF641EA060101D1476102E072
:10F5B800482A08BF07610134082CE4D10160FF2DF7
:10F5C8001FD94168002404F108070126BE4006EA55
:10F5D8000507B74211D14FEA840E0F2606FA0EF638
:10F5E80021EA0601282A03FA0EF641EA060101D1AA
:10F5F800476102E0482A08BF07610134082CE2D1BC
:10F608004160F0BD0F4B1A6842F001021A60596858
:10F618000D4A0A405A601A6822F0847222F4803235
:10F628001A601A6822F480221A605A6822F4FE02CC
:10F638005A604FF41F029A60044B4FF000629A60C0
:10F64800704700BF001002400000FFF800ED00E026
:10F658002DE9F8435B4C0368013AC4F820318388EC
:10F668000D46A4F82431072A42D8DFE802F0040A3C
:10F67800101822292F35B4F820310B80B4F8223124
:10F6880013E0B4F822310B80B4F8203105E0B4F867
:10F6980020315B420B80B4F822315B4205E0B4F8BC
:10F6A80022315B420B80B4F820316B80B4F82431EE
:10F6B8001DE0B4F820315B420B80B4F8223112E02F
:10F6C800B4F822310B80B4F820310CE0B4F82031C2
:10F6D8000B80B4F8223105E0B4F822315B420B808C
:10F6E800B4F820315B426B80B4F824315B42AB80C4
:10F6F800354B1B7A002B62D1B5F9000003F042FCB0
:10F708008046B5F9020003F03DFC0746B5F9040050
:10F7180003F038FCD4F828110646404603F086FC6E
:10F72800D4F834118146384603F080FC0146484637
:10F7380003F074FBD4F840118146304603F076FCA0
:10F748000146484603F06AFB07F0DEFBD4F82C11AB
:10F758002880404603F06AFCD4F8381181463846C0
:10F7680003F064FC0146484603F058FBD4F8441102
:10F778008146304603F05AFC0146484603F04EFBEA
:10F7880007F0C2FBD4F830116880404603F04EFC05
:10F79800D4F83C118046384603F048FC0146404600
:10F7A80003F03CFBD4F848110746304603F03EFC12
:10F7B8000146384603F032FB07F0A6FBA880BDE8F7
:10F7C800F88300BFD02700203000002038B50F4B49
:10F7D8001B689C890E4B186880F31000201A03F0F0
:10F7E800D1FB0C4903F022FC0546204603F0CAFB76
:10F7F8000146284603F0CEFC03F0DEFD6428A8BFCE
:10F80800642020EAE070C0B238BD00BFB019002003
:10F81800C01900200000C84244F6FB71084B1A6862
:10F82800137803EB431300FB03135078C0EB00304D
:10F83800B3FBF0F39078B3FBF0F080B2704700BFF1
:10F84800B019002008B50A480A2290F84D3100EB9B
:10F858004303B3F85C1100F5B47089B220F8041CB6
:10F8680000F040FC80B2FFF7D7FF024B188008BDBC
:10F87800D0270020B41900202DE9F04F89B0059356
:10F88800A04B80461B880492980737D540F2E63291
:10F89800129B9D48DC89B0F900301B1B03F2F3155D
:10F8A800954203D8002BB8BF5B4201E04FF4FA73CE
:10F8B800B0F9022040F2E630121B02F2F31484423F
:10F8C80003D8002AB8BF524201E04FF4FA729342BB
:10F8D800B8BF13460522C3F5FA7393FBF2F30A2265
:10F8E800643B534398F81C20D2105343642293FB83
:10F8F800F2F3134423EAE373DBB200E06423C14666
:10F908000193CB1C03930024039B022C13F8016F73
:10F918007E4F03934FEA440A05D1B7F904301B36EA
:10F928005E4376114AE07A4B37F9142033F91430E4
:10F9380003EB4202049B5B429A4203DB049B934223
:10F94800A8BF1346734A32F90A50059A5B1B32F96D
:10F95800145003EB050BFEF703FB88B16E4A5846BB
:10F96800155D03F00FFB6D4903F014FC01462846B2
:10F9780002F038FC694903F059FB03F01DFD83468A
:10F98800604A1288D10714D437F90A501B366E43DF
:10F9980093074FEA261611D598F812509DF90420BE
:10F9A80005FB0BF35343642293FBF2F306EB231698
:10F9B80004E098F8085005FB0BF52E11584B042568
:10F9C80033F90A30574F93FBF5F5751B99F8016029
:10F9D800E35D6E435E430293642396FBF3F698F867
:10F9E80051B0F611BBF1000F1BD0022C30460CD1E0
:10F9F80003F0C8FA5FEA5B0304D05B45A8BF5B4627
:10FA08001A4600E00122484905E003F0BBFA5A46CD
:10FA1800391D01EBC401FB69FAF7EEF803F0CCFCE1
:10FA28000646424B99F80B7019883E4B01FB05F2CC
:10FA380003F1200E5EF82400D21207FB02073C4AAD
:10FA4800B7F5001FA8BF4FF40017974203F12C0029
:10FA5800B8BF174650F8242040F824504FF6FF70DE
:10FA68000909B0FBF1F1AA1A4A4303F1380103F17D
:10FA780044054EF8247051F824E055F8240045F860
:10FA880024E098F85050921170444FEA840C7F1388
:10FA9800104441F824208DB1CDF818C0079303F025
:10FAA80071FA079B2A4603F1500101EBC401DB6997
:10FAB800FAF7A2F803F080FCDDF818C099F81530C1
:10FAC800F2195843029B013443431846642390FBC0
:10FAD800F3F0184B0012024423F80A2003F108023D
:10FAE8004CF80260032C03F1140203F120034CF8D4
:10FAF80002704CF8030009F101097FF405AF09B061
:10FB0800BDE8F08F8C1A0020382D0020CC11002081
:10FB1800E0300020F42C0020BCA0010800002041A7
:10FB280008110020C0290020D4290020E41000205A
:10FB38000000E0FF282A00202DE9F04F054690F844
:10FB480050008DB008910592099318B13228A8BFCA
:10FB5800322000E0012003F015FA0146AA4803F01C
:10FB680019FBAA4B04461888002808BF012003F097
:10FB780009FAA749069003F059FA0190019920461D
:10FB880003F04CF90146019803F004FBA14B0790E0
:10FB98001B889A0724D5A049B1F90030B1F90200B1
:10FBA80083EAE37280EAE071A2EBE372A1EBE07111
:10FBB80091420C46B8BF1446B4F5E17F12DA91427F
:10FBC80003DD0028D8BF404203E0002BCCBF184615
:10FBD800584203F0D7F9914903F0DCFA064603E0EE
:10FBE800002601E04FF07E564FF00009CA46039503
:10FBF8000024630004938A4B33F9140003F0C2F91C
:10FC0800884903F013FA03F0D7FB03F0BBF98649E0
:10FC180003F00CFA804B029033F9140003F0B2F9A8
:10FC28007C4B07461B889B077ED0014603F0F6F8FD
:10FC38007E4B804633F9140003F0A4F90146404690
:10FC480003F0ECF803F0B8FB059B5B42984203DB3A
:10FC5800059B8342A8BF0346754A0499885E099AA2
:10FC68001B1A32F91400184403F08CF98046FEF789
:10FC780077F970B16F4B40466F4914F8039003F061
:10FC880089FA0146484602F0ADFA6B4903F0CEF90D
:10FC98008046287F03F072F9684903F0C7F9824665
:10FCA800287A03F06BF90146404603F0BFF964492E
:10FCB80003F0BCF903F080FB81460AF1004003F031
:10FCC8007BFB814505DB504603F076FB4845A8BF22
:10FCD800484603F057F9DFF88C910199824640466F
:10FCE80003F0A4F959F8241003F098F855494FEA9D
:10FCF800840B804603F038FB38B94046524903F07C
:10FD080051FB20B1DFF8408101E0DFF8388149F884
:10FD18000B80A87C03F032F90146404603F086F9CF
:10FD28004A4903F083F981463A4BB3F800B01BF017
:10FD3800010F40F099803A4B049ADFF82081D35E96
:10FD4800002BB8BF5B42B3F5206F4FEA84030A93D8
:10FD580003DD002348F824302AE03D49384603F003
:10FD680065F9039B0B90587803F008F90B9A014644
:10FD7800104603F00FFA029903F04EF8019903F0C8
:10FD880055F958F8241003F049F83249804603F031
:10FD9800EBFA38B94046304903F004FB20B1DFF8EC
:10FDA800B88001E0DFF8AC802C4A0A9B42F8038057
:10FDB800039BD87A03F0E2F8284B53F8241003F099
:10FDC80035F9274903F032F91BF0020F80464DD070
:10FDD8003846514603F020F80146304603F026F92C
:10FDE8000146504603F01AF849460746404603F0D4
:10FDF80013F80146304603F019F90146484603F066
:10FE08000DF8804632E000BF83F9223EE41000205E
:10FE1800BD3786358C1A0020CC1100200000E14344
:10FE2800081100200000A03ECDCC4C40E03000205E
:10FE3800F42C0020BCA00108000020410000A040D4
:10FE48006F12033C0000F0C10000F0410AD7A33D47
:10FE58000000A043000040C3000040435C2A00208B
:10FE68000AD7233C542A0020C8465746DFF83CB23C
:10FE78000BF1A803185D03F085F80146029803F01A
:10FE8800D5F8894903F0D2F80146384602F0C4FF94
:10FE980095F85120034642B10BF10401DBF81C3000
:10FEA80001EBC401F9F7A8FE0346804F029807F159
:10FEB800AC0B5BF824100A9302F0AEFF019903F033
:10FEC80069F9029B07F1B4024BF8243052F824B0C8
:10FED8000292594602F0A0FF0146079803F0A6F8DF
:10FEE8000146584602F09AFF029A834642F82400D7
:10FEF80007F1BC02105D03F045F80146584603F0CF
:10FF080095F86B4903F092F883460A9B41461846D8
:10FF180002F084FF594602F07FFF06F0F5FF049BCC
:10FF280007F16802D0520A9B07F170021846029244
:10FF380003F042FA029A07F17C0342F82400404693
:10FF4800029303F039FA029B07F1880843F824006A
:10FF58000BF1004003F030FA039B48F8240001330A
:10FF680003930CB9012444E6089A524B9479B3F9E7
:10FF78000430640028345C434F4B6411B3F9040027
:10FF880003F000F84FF07A5103F050F806F0BCFF88
:10FF9800201A02F0F7FF002CB8BF6442322C064644
:10FFA80002DD0023BB6224E0069803F005FA20F086
:10FFB800030002F0E7FF8046687B02F0DFFF01469E
:10FFC800304603F033F83D490446404603F0E2F872
:10FFD8000146204603F02AF803F0EEF9BB6A1844FC
:10FFE800374B9842A8BF1846364B9842ACBFB86208
:08FFF800BB62BB6A6FF0FF0061
:020000040801F1
:100000005B13B3F5807FA8BF4FF480739842B8BFED
:10001000184602F0BBFF8046304603F0D1F9EB787A
:100020005843801102F0B2FF97F8BF300446032B0B
:1000300011D9B5F84E60B6F5FA7F0CD203F0C0F9CD
:100040007342984203DBB0420346A8BF33461846CA
:1000500002F09CFF044695F8512062B1530803D08A
:100060009A42A8BF1A4600E0012220461849FB69BF
:10007000F9F7C6FD04464146204602F0D3FE03F0E0
:100080009FF900B202F082FF06F042FFA7F86C0071
:10009000204603F095F9B867404603F091F9002334
:1000A000C7F88400C7F890300DB0BDE8F08F00BFEE
:1000B000A69B443BC0290020F7CC9238CC110020ED
:1000C0000811002000803B45FEFFFF0F020000F0FA
:1000D000D42900200368DB68184703689B68184729
:1000E00003685B68184703681B681847B0F902305B
:1000F0002DE9F74F93421CBF0023037090F800A036
:1001000004460E469146BAF1000F40F0AB8010460F
:1001100002F03CFF864902F08DFF864902F08AFF1B
:100120004FF07C5102F086FF06F052FF0146054673
:1001300002F080FF80498346284602F07BFF034699
:1001400058461946019302F06DFE4FF07E5102F0C1
:1001500069FE01464FF07E5003F020F829468046A4
:1001600002F068FF294602F065FF0746014660601D
:1001700002F058FEE7604FF07E572946A0602761E5
:10018000284602F04FFE294602F054FF4FF080410E
:1001900002F046FE0146404602F04CFF019B6061C2
:1001A0001946584602F03CFE394602F03BFE014635
:1001B000404602F03FFF40F2DC53A046274655463A
:1001C00063651023A4F852301823A061A4F85030BE
:1001D0004FF09741D8F8100002F02CFF0021824622
:1001E00003F0C6F828B150464FF07C5102F018FEDB
:1001F00004E050464FF07C5102F014FE03F042F947
:10020000C7E90E014FF09741D8F8040002F012FF41
:100210000021824603F0ACF828B150464FF07C51E3
:1002200002F0FEFD04E050464FF07C5102F0FAFD72
:1002300003F028F90135032DC7E9080108F1040886
:1002400007F10807C4D1A6F2DC531B042367E36758
:100250006367C4F88030A367C4F884300123A4F82E
:1002600002902370D4F85490B4F95280C9EB06067A
:10027000636A06FA08F67343276A4FEAE67B206F43
:1002800007FB0B332667A7FB0667E26F1F44636C0F
:10029000D4F840C053434FEAE27B0CFB0B3ED4F84A
:1002A0008010C4F88020ACFB02237344B61A67EBBD
:1002B0000307E36AA26A43434FEAE07B02FB0B3E7B
:1002C000A2FB00237344B6185F41E36C656F4B4398
:1002D0006067A06C4FEAE17B00FB0B33C4F884102D
:1002E000A0FB01011944636B361A05FB03F3206B75
:1002F0004FEAE57B00FB0B3367EB0107A0FB050131
:10030000801919447941B4F95020A56702F076FDAF
:1003100008F1FF3201239340E067C01841EBE3711D
:10032000424602F06BFD484403B0BDE8F08F00BFC9
:100330006F12833ADB0F4940F404B53F2DE9F843CF
:100340000024254BE0B293F8BF60B0420DD203EB1E
:100350008003224AD3F8C03032F810101BB10B28AA
:1003600001D8DB6898470134EBE71D4B1B685B0342
:100370002FD500242346E2B2B2422AD2DFF85890A9
:100380004FEA840809F1C00757F8242055689D42B8
:1003900017D02846FBF71EF8EFF31283502282F3A2
:1003A00012882821AA8C01FB009092B20132C0F879
:1003B0001421AA8ADBB292B242F00102AA8283F32C
:1003C000118857F8083000221B6801341A802B4628
:1003D000D1E7BDE8F88300BFC02900202811002024
:1003E000FC2C002008B50E4B1B6813F4805F0D4BEE
:1003F00014BFD3F89021D3F8942193F8BF109288BA
:100400000023D8B2884204D2074820F813200133D1
:10041000F7E7FFF793FFBDE808403220F7F763BE28
:10042000FC2C0020C0290020281100200A4B30B5E8
:100430001A680A4B02F48052D3F89041D3F89451D1
:1004400000230AB1A18800E0A988054820F813100C
:1004500001330C2BF5D130BDFC2C0020C02900202D
:10046000AA2C002070B5124D0024214605F29910E7
:10047000702285F8984106F03EFB2146D5F80C32F3
:100480000B4A0B4493F9020088B11E6802F29914DA
:100490000E5108199C88073184809B7970298371DB
:1004A00092F8983103F1010382F89831E6D170BDDA
:1004B000C0290020094B1A680E2303FB0020437A51
:1004C000FF2B07D0064A12789A4203D9054A32F820
:1004D000130000E0808800B2704700BF1C1B0020A2
:1004E000B4280020382D00202DE9F74F304C054668
:1004F000D4F810723846F9F765FE06463846F9F723
:10050000EEFDD4F8147281463846F9F75BFE01908F
:100510003846F9F7E4FDD5F804A0074631465046C1
:1005200002F088FDD5F8088083464946404602F02F
:1005300081FD0146584602F073FC019B2968834601
:10054000184602F077FD49460546504602F072FD16
:10055000394602F06FFD0146284602F063FC394639
:100560000546404602F066FD314602F063FD014655
:10057000284602F057FC0146584606F0A1FD0D49F9
:1005800002F058FD0C4902F009FED4F8181202F0EE
:1005900049FC0A4902F002FE06F0BAFC83B21A04D2
:1005A00044BF00F5B47083B218B203B0BDE8F08F59
:1005B000C02900200000E144DB0F49400000204139
:1005C00001380A4B042804D8DFE800F00507090BBE
:1005D0000D00074A08E0074A06E0074A04E0074A18
:1005E00002E0074A00E0074A1A607047480000200E
:1005F00059E6000881F8000875E900081FE30008C3
:100600008DDF000841FB000810B54B88DC0641BFB8
:100610002F4B14791B6853F8244044BF2D4B43F8EB
:1006200020404B889B0641BF294B54791B6853F8E7
:10063000244044BF274B43F820404B881C070ED56D
:10064000254B0C781B78B3EB141FA1BF204BD4783B
:100650001B6853F82440A4BF1E4B43F820404B882E
:100660009B070ED51D4B0C781B78B3EB141FDFBF17
:10067000174B54781B6853F82440DCBF154B43F8E4
:1006800020404B88DC070FD5154C0B78247803F0FD
:100690000F03A342DFBF0E4B14781B6853F82440AE
:1006A000DCBF0C4B43F820404B885B070FD50B7821
:1006B0000C4903F00F0309788B42A1BF044B9278D9
:1006C0001B6853F82220A4BF024B43F8202010BD22
:1006D000141B0020720E00209B1D0020991D00207D
:1006E000981D00209A1D0020254A0023F0B51568AA
:1006F0001C461A462348244903700B702E1976882D
:100700004EB92F5D3FB9037000230A704B70077814
:100710001C461A460CE0360548BF013204F10404B9
:1007200003F1010348BFD2B2802CDBB2E6D1EAE785
:10073000E0B2B8420CD215F82400013406099E42FA
:1007400000F00F00A8BF731C9042A8BF421CEFE747
:100750008A704B70C2F3470102F001020A444C1E3A
:100760000A490B480A70C3F3470203F0010313441C
:1007700004700849501E084A08701370F0BD00BF8D
:10078000181B0020901D0020DC2B00209A1D00204B
:10079000981D00209B1D0020991D0020924B2DE9E3
:1007A000F04FDA68914D1A612A6891B0DA60904A88
:1007B0000295136843F0200313608E4B1A78012AC8
:1007C0000CBF002201221A708B4B1A78910740F15E
:1007D0004D838A490978042940F248838849097879
:1007E00001F0040101F0FF0011B922F001021A70BA
:1007F0001B78DB0702D408B1FAF7D2FC8149CA782A
:10080000531C052293FBF2F202EB82029A1A7E4BF2
:10081000CA701F7892000023DFF81082DFF8109270
:1008200058F82310794C91FBF9FE04F1080040F8C8
:1008300023E0774844F8231000FB0E1142F21070B9
:1008400091FBF0F004F1100680B226F813004FF08F
:10085000140C04F114060CFB036C04F13C0A5AF866
:1008600023605CF802504CF80210761B31440526D8
:100870004AF8231091FBF6F109FB0E114434012FC5
:1008800044F823104FEA830B444605D10238B0F5F3
:10089000797F98BF4BF808100BB90123BCE7594E7C
:1008A000029BB2461868336DC01A02F06BFB5949BF
:1008B00002F074FC029B4FF07E511B6807463365C3
:1008C00002F056FD08B94FF07E574B4BCAF85470F2
:1008D0001B78514E13F00103504D12D00DAA009217
:1008E0004F4B0EAA01920CCB94E80300FAF76EFB73
:1008F0000D9A6421B2FBF1F20E9B328093FBF1F36F
:1009000000E033802B809AF858303E4D002B35D0D4
:10091000696D4FF07E5002F041FC0746EB6D206898
:10092000C01A02F033FB394602F084FB02F048FDA6
:100930002B6E86B2606836B2C01A02F027FB394BC4
:10094000196802F077FB394602F074FB02F038FDBB
:10095000B5F9662000B28118B5F964200220B318F9
:1009600091FBF0F193FBF0F389B29BB2A5F86A100A
:10097000A5F86830A5F86610A5F8643001238AF858
:100980005830294B61681B88206803F030031D4EE6
:10099000264DCAF86010CAF85C00002B00F0668291
:1009A00006F17403009306F178030193F26E336F3E
:1009B000FAF70CFB6B68306FC01A02F0E7FA194BBC
:1009C000196802F037FB02F0FBFCF36E2A68C6F8E8
:1009D00080009B1AF3670C4B1B78012B2AD0022B4B
:1009E00000F0E68042E200BF9C070020202D00209E
:1009F000C419002052110020C8190020CE1900206F
:100A0000E7300020DC2B0020FC0F0020E02B002032
:100A1000806967FF00007A44421A0020441A0020CF
:100A2000541100203C0000208C1A0020D019002016
:100A300080969800D6F88430D6F8A0400293D6F875
:100A4000943004F100400393D6F89830776D059305
:100A500002F0B6FC8146204602F0B2FCD6F89C308B
:100A6000BB4C0493BB4B06901B684FF0000B0793E5
:100A7000B94E4FEA4B0356F82B80A6F114024046BC
:100A800032F81B50089302F081FA029902F0D2FA70
:100A900002F096FC401B1FFA80FA283626F81BA0AD
:100AA0000FFA8AFA504602F071FA039902F0C2FA7C
:100AB00002F086FC86B20AEB080002F067FA05999C
:100AC00002F0B8FA394602F0B5FA216802F0AAF944
:100AD00002F076FC484504DB069B9842A8BF184606
:100AE00000E0484602F052FA206002F069FC079BE1
:100AF000304486B2987802F045FA984902F09AFAA2
:100B000001464FF07E5002F049FB394602F08AF967
:100B10000146384602F042FB09906068D4F808A00C
:100B2000C0EB080002F032FA394602F037FB5146BA
:100B300002F076F9099A0146104602F07BFA014666
:100B4000504602F06FF93135ADB2622D0146206199
:100B5000C4F80480A0600ED9049802F06BFA02F089
:100B60002FFC7F4AB0F5FA6FA8BF4FF4FA609042AD
:100B7000B8BF104600E0002040F6B832064436B256
:100B80009642A8BF1646774A089B9642B8BF1646BB
:100B9000754A54F8140B9E52142202FB0BF273494F
:100BA0005050BBF1000F40F061814FF0010B5FE747
:100BB000684BB6F8A8401F68736F3D8902935B08C5
:100BC0009D4228BF1D4623B29D4202DC1FFA85F9D3
:100BD0000AE06749706D02F02DFA02F0F1FB204443
:100BE0001FFA80F9A6F8A890DAF87860DAF8AC4035
:100BF000341B2046FAF72CFA41F293130028D8BF91
:100C000040429842CCBF0020012078B3204602F039
:100C1000BDF9584902F00EFAF9F761FA0446029854
:100C200002F0B0F90146204602F004FA02F0C8FBD7
:100C300040F6B83380B2AAF8B00000B29842A8BF1C
:100C40001846484B9842ACBF3018F01848F6A043FD
:100C5000984203DDA0F50C40A03804E00028BCBF9A
:100C600000F50C40A030CAF8B40001E0CAF8B46046
:100C7000DAF8B4300026C3F50C502830039302F0A4
:100C800085F93C4902F0D6F90446F9F79BFA0F9032
:100C90002046F9F724FADAF8B830DAF8C4400593B8
:100CA000DAF8BC300E9004F10040089302F088FBA3
:100CB0000490204602F084FBDAF8C030DAF8548061
:100CC0002A4C09900793730048460A9302F05EF994
:100CD0000EAB53F8261002F0ADF9DFF8A0A00546E0
:100CE0003AF9160002F052F90146284602F098F847
:100CF00002F066FB05B2204BB5F57A7FA8BF4FF432
:100D00007A759D42B8BF1D460AF13C0AA8B22AF87E
:100D1000160000B202F03AF90599824602F08AF90B
:100D200002F04EFB089983B25046069302F082F916
:100D3000414602F07FF9216802F074F802F040FBAE
:100D4000049B98421CDB099B9842A8BF184618E0F8
:100D50003810002000100020582C0020DB0FC94064
:100D600030F8FFFF48F4FFFF0A1000206010002059
:100D70000000C842D302373918FCFFFF442C002082
:100D8000049802F003F920608346B87802F0FAF87C
:100D9000384902F04FF901464FF07E5002F0FEF95B
:100DA000414602F03FF80146404602F0F7F90B9049
:100DB0006068D4F808A0281A02F0E8F8414602F06A
:100DC000EDF9514602F02CF8DDF82CC001466046E2
:100DD00002F030F90146504602F024F86560014601
:100DE0002061A060079802F025F902F0E9FA069B5D
:100DF0001434034458469A4602F0E2FA40F6B832F8
:100E0000504400B29042A8BF10461B4A0A9B904231
:100E1000B8BF1046194A1A4998521422724342F830
:100E200001B00EB901264EE73B792BB1039A64233A
:100E300092FBF3F3134A13803B88029A124C9A42B6
:100E40000DD9D4F8AC30A06FC01AFAF701F942F20C
:100E5000107380EAE072A2EBE0729A4206DD0B4B5F
:100E600001221A70B4F8C820064B1A8011B0BDE8F0
:100E7000F08F00BFDB0FC94048F4FFFF0A100020CD
:100E800038100020F80F0020DC2B0020FC0F002081
:100E9000F0B5974D87B02B78023B082B00F2958177
:100EA000DFE813F009002E004E0063007B008D0088
:100EB00009016E0179018F4B8F4C1A6863686433A6
:100EC0009A4240F2828100268C4B8D4A1B789E42CA
:100ED0000ADA2368884FD05C30B101F05DF83B68D6
:100EE000013601333B60EFE72168834B525C002AF7
:100EF00040F06B811A604FF0FF325A60032354E1D7
:100F0000262300937F4B492003F10C0201930292A8
:100F10005021A3F10A020233F8F724FD002840F023
:100F20005481794B4FF0FF311B6813F08002724BF4
:100F300003D083E80300042337E11A6059602AE0F4
:100F4000724A02230021009301910291482002F18C
:100F50000803F8F707FD002840F03781664B4FF093
:100F6000FF3218605A6005231FE107230093684B86
:100F7000472003F10C02019302920021A3F1080221
:100F80000433F8F7EFFC002840F01F815A4B4FF074
:100F9000FF3218605A60062307E15E4A05230021EC
:100FA000009301910291532002F10803F8F7DAFC53
:100FB000002840F00A81504B18600723F5E04E4CA2
:100FC000236813B96360012323604C4B1A7863686C
:100FD0001344402BA8BF4023132B636040F3F580DC
:100FE000454B1B680D2B00F2E780DFE803F060073C
:100FF0000B0E121923282D3134404B51464800F076
:10100000A9FF51E0454846493FE046484649474A1E
:1010100048E0474B474893F8D61793F8D72741E065
:10102000434B0C2193F8B027434801FB023393F85C
:10103000B2172AE03E4B4148B3F8441125E03C4B3F
:101040003F48B3F8461120E03E4B3F4819691CE089
:101050003E483F4B18E03F4B1B68D80404D5344B47
:101060003D4893F87C1110E00C2323601FE0304BC7
:101070003A4893F8801193F8812193F87F3100F07A
:1010800079FF11E03648374B198800F073FF0BE009
:101090001D4B1B6819050AD5254B3348B3F884113D
:1010A000B3F9822100F066FF6368181A6060236854
:1010B0000133236089E02D4B1B689A0114D52C4B1A
:1010C0001B888BB92B4B0E201B6804A904932A4B59
:1010D0001B680593F8F72AF9284B4FF480521A80C1
:1010E00009232B70F8F79CF9F8F702F96DE000BFBF
:1010F0005C2D0020202D00201C2F002054000020FB
:10110000C0A001082AA10108FC2C0020E8A20108C7
:1011100000A301084CA3010800C101081DC101087A
:10112000D1B5010835C10108BCB50108C8B5010831
:10113000D41100204CC1010860C101086DC1010833
:101140007FC101089427002091C10108A4C10108B2
:101150001A000020042F0020B1C10108C1C10108FC
:10116000DDC10108002F0020EBC10108E8100020BC
:10117000102F00200C2F0020CC300020242F002026
:10118000134B1B78002BADD0124B1B689B01A9D4CD
:1011900008232B70A8E7104B1A68104B5B68C83304
:1011A0009A4204D900F0AEFE01232B700DE000F04E
:1011B000C3FE0028F6D108E000F0BEFE28B1084BBF
:1011C0004FF480521A800923EFE707B0F0BD00BF4B
:1011D000082F0020E8100020202D00201C2F0020C8
:1011E000242F002007B5064B06490093064B074AFB
:1011F00001930748074BF8F743FF03B05DF804FB82
:10120000C8B50108D2BF0108D1B50108CBBF01089C
:101210000BC30108BCB5010808B5037833B90C4B02
:101220000C481978BDE80840F8F72ABF05F0FCFC27
:1012300002280CD8064B0C221870074B02FB00301A
:10124000064B0230186000F0C7FB0548E5E708BD13
:10125000A82C00202BC30108841900204C11002069
:1012600083B5010808B503783BB90B4B0B4893F8DD
:10127000B017BDE80840F8F703BF05F0D5FC022819
:1012800008D8054B83F8B007F9F7C0F8F9F764F907
:101290000348E8E708BD00BFD41100202FC30108B0
:1012A00083B5010838B5037803BB214B1B680133B4
:1012B0000F2B07D81F490C2202FB031295681C460E
:1012C0002DBB00E01C4601340F2C01DD002400E0A2
:1012D00005D818490C2202FB04129568BDB99C423E
:1012E000F1D11548BDE83840F8F7CABE05F09CFCBE
:1012F0000F28044605D80F4A0C2303FB00239D68E2
:101300002DB92146BDE838400C48F8F7B9BE084B66
:101310001C60F6F775FE21462A460948F8F7B0FE2C
:101320000C235C43034B185DBDE83840F6F77ABEEA
:101330004000002074A301083CC3010852C3010807
:101340006AC3010873B5037813B9F6F7D5F93DE020
:101350001F4901AA05F0C9FC00240146264625467E
:1013600099B134B1012C08D1084605F05DFC064660
:1013700003E0084605F058FC05461549002001AA7F
:1013800005F0B3FC01340146EAE70B2D02D9114800
:101390000C220BE0022C10D1A6F57A73B3F57A7FFC
:1013A00007D90D484FF47A714FF4FA62F6F721F934
:1013B0000CE00A4B03EB45035E80084B084803EB47
:1013C00045032946B3F90220F8F75AFE02B070BD72
:1013D000A6B90108E4B7010809BD0108A82C00203E
:1013E00081C3010838B50D4C05462368834206D1F8
:1013F000F6F738FC204600214C2205F07CFBE36C1C
:10140000AB4209D12846F6F72DFCBDE83840044828
:1014100000214C2205F06FBB38BD00BF182800200A
:1014200064280020034B1A68D379591C1344D171E6
:10143000187A70476C1A002010B5FFF7F3FF84B2DA
:10144000FFF7F0FF04EB002080B210BD10B5FFF7EE
:10145000F3FF0446FFF7F0FF04EB004010BD10B5AA
:101460000446054B21461868FEF73DFE034B1B68FA
:1014700098796040987110BD701A00206C1A002095
:1014800038B504460D462420FFF7E9FF4D20FFF74D
:10149000E6FF002C084C14BF21203E20FFF7DFFFA1
:1014A0002368002228469A71FFF7D9FF236893F832
:1014B0004900BDE83840D2E76C1A00200146002000
:1014C000DEE710B50446C0B2FFF7C9FF200ABDE849
:1014D0001040C4E710B5044680B2FFF7F2FF200CBD
:1014E000BDE81040EDE737B58288836804461006F2
:1014F0000D4641BF29494FF4CC7091F8B01700FB5D
:101500000133D10542BF26490C20097802F03F0281
:1015100048BF00FB0133042A12D006D8012A0DD09F
:10152000022A2FD193F900102DE0102A0AD0202A88
:101530000AD0082A26D1B3F9001024E0197822E055
:10154000198820E019681EE069461868F8F71EFC43
:1015500001461448F8F794FDF5B1E06801F016FD76
:101560006946F8F713FC01460F48F8F789FD206932
:1015700001F00CFD6946F8F709FC01460A48F8F746
:101580007FFD09E000210948F8F77AFD25B10848F8
:10159000E1682269F8F774FD03B030BDD411002072
:1015A000A82C0020BFB80108B8B80108ADC00108D8
:1015B00090C30108024B0146D869FEF794BD00BFF5
:1015C000A82C002010B5441E14F8011F21B1034BB4
:1015D000D869FEF788FDF7E710BD00BFA82C0020F2
:1015E000F7B52A492A4B08782A4D1C682A4B05EB87
:1015F00080001A88D0F8C010284B29481B78009129
:101600004FF47A71B4FBF1F1F8F73AFD254B264817
:101610001968264B0026B1FBF3F1F8F731FD244B96
:101620001F68F3B205EB8302D2F8D010E9B10124B0
:101630009C403C4217D0220715D01E4A0B20D25C9A
:1016400000FB0323134A1C4802EB8303D3F8F0206A
:10165000F8F716FD022C06D1184B93F8281011B19B
:101660001748F8F70DFD0136DBE71648FFF7AAFF2C
:10167000154B16481A88164B92B2198840F2DC7343
:1016800003B0BDE8F040F8F7FBBC00BF141A00201F
:10169000202D002074A30108B4190020440000206C
:1016A00097C3010850000020DAC3010840420F0030
:1016B000C41900204C000020EAC30108A82C002017
:1016C000F2C301083AC40108E6100020F6C301087D
:1016D000E41000202DE9F0410024804625460F4EFD
:1016E0004146A759384605F087FA58B139460C48A3
:1016F000F8F7C6FC30190021FFF7F5FE0948FFF79F
:1017000061FF013540F6BC4314349C42E7D11DB95A
:10171000BDE8F041044855E7BDE8F08114A5010893
:1017200028B901083AC401083BB801082DE9F74F70
:10173000824605F024FA054628B1012819D19AF805
:1017400000302A2B15D15948FFF73CFF0024584E92
:101750005848A159F8F794FC30192946FFF7C3FE01
:101760005548FFF72FFF40F6BC4314349C42EED19E
:1017700098E050463D2105F0F4F9002800F08D80F6
:1017800003461D4613F8012D202AFAD0441C20469A
:1017900005F04AFA81462046F8F762FA0746CAEB96
:1017A00005054FF0000B142404FB0BF4DFF8208137
:1017B00008F5D073E6580193304605F0E0F9844609
:1017C000314662465046CDF800C005F0E1F9DDF83B
:1017D00000C0019B002856D1EAB2624553D11D19C1
:1017E0004444D4F8AC0101F0D1FB0146384601F085
:1017F000D3FD002845D0D4F8B00101F0C7FB014665
:10180000384601F0BFFD00283BD0B4F8A4319A0659
:1018100058BF4F46142202FB0B881C0648BF2748BE
:10182000D8F8A82142BF90F8B0074FF4CC7404FB5D
:101830000022D80542BF22480C24007803F03F0361
:1018400048BF04FB0022042B39460BD004D8013BCF
:10185000012B0CD817700AE0102B05D0202B05D0D7
:10186000082B04D1118002E0176000E017603146B8
:101870001448F8F705FC2846002103B0BDE8F04FF6
:1018800031E6114805E00BF1010BBBF1A30F8AD142
:101890000E4803B0BDE8F04F94E6504603B0BDE8F3
:1018A000F04F17E703B0BDE8F08F00BF28C4010870
:1018B00014A5010828B901083AC40108D411002070
:1018C000A82C00203DC4010848C401083BB8010809
:1018D00074A3010870B50546284605F050F9064680
:1018E00058B9194B19485A79194BBDE8704003EBA8
:1018F0008203D3F8581EF8F7C3BB28461549324671
:1019000005F046F960B91448FFF75CFE134C54F833
:10191000041F19B11248F8F7B3FBF8E7114805E0C6
:101920000024114B53F8241019B91048BDE8704039
:1019300048E62846324605F02BF901340028F0D15C
:10194000014B0B4D5C71C7E7D411002068C401083E
:1019500074A30108D6B8010874C40108CCB1010809
:10196000D2B801083AC40108D0B101083BB8010857
:1019700083B5010808B50748FFF724FE064BD86970
:10198000F6F75DFCFEF72EFDF8F716FD034A044B53
:10199000DA6008BD87C40108A82C00200400FA05FD
:1019A00000ED00E008B50548FFF70CFE00F05AF81E
:1019B000F8F72CFDBDE80840DCE700BF93C4010840
:1019C00008B50448FFF7FEFDF8F720FDBDE8084024
:1019D000D0E700BFA9C4010810B50E4C2068F6F787
:1019E0007DFA20680022047A02FB02F3193B63436C
:1019F00003F6C4135343192193FBF1F3064921F86D
:101A000012300132072AEFD1BDE810400349F6F742
:101A10001DBA00BF4C1100208810002018130020B0
:101A20000E4B1A78692A16D140F2DC72598891421D
:101A300011D11A79BE2A0ED193F8D9270020EF2AA6
:101A40000BD113F8012B5040054A9342F9D1B0FA5B
:101A500080F04009704700207047704700F8030885
:101A6000DCFF03082DE9F74FEA4C002140F2DC725D
:101A7000204605F040F8E84B04F53A721A60E74B4F
:101A800000221A70E64B04F2B271196069232370C8
:101A9000032363714FF48073A3604FF41673A4F8AB
:101AA0006631FA23A4F86831BC23A4F864314FF4FA
:101AB000FA73A4F86E31012384F8623184F87E3120
:101AC00084F88631052384F8273240F2DC53A4F8E9
:101AD000983140F24C43A4F89A3140F26C73A4F868
:101AE0009C3140F27533A4F89E3140F64303A4F8CC
:101AF000A0312346202184F86A116E2184F87C11DC
:101B00000A2184F87D112B2184F87F11212184F88A
:101B10008011232184F881114FF4C871A4F8821137
:101B2000032ACCBF0121002102F1010283F8A21196
:101B300014BF1E217521122A83F8A31103F1020399
:101B4000EED140F27E41A4F8441140F23A71A4F87B
:101B5000461140F27E51A4F84C1140F2EA5140F295
:101B6000DC50A4F84E1140F2B4514FF4FA63A4F8DB
:101B7000C831A4F8CC31A4F8D031A4F8D43105236D
:101B800084F8E231C82301264FF47A774FF0320B04
:101B9000A4F8E631DFF880924FF4C8734FF01E0AC4
:101BA0001922A4F8EA31A4F84A01A4F85011A4F8C3
:101BB000C671A4F8CA71A4F8CE71A4F8D27184F8E1
:101BC000E46184F8E56184F8E861A4F84871A4F858
:101BD00052B184F895A184F8E32100920190A4F811
:101BE000543184F8E16184F8EE61A4F856B184F8C8
:101BF000F161FDF7F1F9D9F80030009A00254FF0B6
